:100000000C9457100C947F100C947F100C947F105C
:100010000C947F100C947F100C947F100C947F1024
:100020000C947F100C947F100C9483160C94746DB8
:100030000C94C5710C94C36D0C947F100C940C1728
:100040000C9471160C947F100C947F100C947F10FC
:100050000C947F100C947F100C947F100C947F10E4
:100060000C9448720C9452170C94286E0C94927253
:100070000C947F100C947F100C94E16A0C947F1008
:100080000C947F100C947F100C947F10E818EC18DF
:10009000B118B718BD18BD18BD18E018E418E81855
:1000A000EC18F918F918F018952395239523952342
:1000B000C223B923B923B923B923B923B923B92357
:1000C000A523AA23AA23522F5C2F722FBF2FFE2F06
:1000D0005C3067306A30C430C83008341D34B934FD
:1000E0004236CB364935043A49384C375437DC3739
:1000F0004B394343164319431D43234327432C43A2
:10010000B84BC74BD24BE84BEF4BF64B054C1C4C56
:10011000344CFF4C2A4D324D3A4D464D6B4D7B4D84
:10012000A54DF24DFE4D394E514E624E6C4E7A4EFB
:10013000864ED951EB5CAD54205A2D55EB5CEB5CEF
:10014000F058EB5C855BEB5CEB5CEF53E9513156AF
:100150005B694A6944694C695069546947695869DF
:100160005E69AB70AE70C570E070E070C570C57050
:10017000C473C673C973CE73DF73EE73FC730674F6
:10018000167426742B744174447448744A744C7405
:1001900051745574607464746C7473747774797486
:1001A0007D747F748174837487748B749074957478
:1001B0009A749F74A47420454550524F4D20697322
:1001C0007420766572616C746574202020544553E8
:1001D00054452045494E5354454C4C2F4B414C49B6
:1001E0004200416C61726D20697374206465616BBB
:1001F0007469766965727400454550524F4D207799
:10020000656E6967205370656963686572004C416B
:10021000454454000553746F70706564006D5374E9
:1002200061636B206F666C6F7700536368616C74F9
:100230006572205761726E756E671F536368616CDB
:1002400074657220617573736368616C74656E00A8
:10025000476173206E6963687420696D2052756808
:10026000657A7374641F7365747A6520617566209E
:100270005374616E64676173004E41434852494351
:1002800048540054617374652064727565636B65CE
:100290006E0062656C2E2054617374652064727503
:1002A00065636B656E004F4646414E20476173475C
:1002B0006125000000642810070301000000000110
:1002C000010102020202010103002D2D2D2D00204B
:1002D000414C41524D0000010203000201030301A1
:1002E0000200030201000453656920486F6520473E
:1002F0006173205175652000414E20004155530027
:1003000003474153534549484F45494430494431D7
:1003100049443251554546574B54524E4C31204C6E
:1003200032204C33204C34204C35204C36204C3776
:10033000204C38204C39204C41204C42204C43204A
:10034000001B1E272D36394B4E636C7278878D93B8
:100350009CB1B4C6C9D2D8E1E453706C6173680033
:1003600080400000000000000000000000000000CD
:10037000000000000000000000000000000000007D
:10038000000000000000000000000000000000006D
:10039000000000000000000000000000000000005D
:1003A0000000000000000000000000000080C0E02D
:1003B000E0F0F8F8FCFCFCF8F8F8F0400000000071
:1003C00000808080000000000000000000000000AD
:1003D0000000000000000080C0C0E0E0E0F0F0F0AD
:1003E000E0C00000000000C0F8FFFF9F8783838308
:1003F00083838383838383838383838383838383CD
:10040000838383038380838383838383838383833F
:1004100083838383838383838383838383C3E3731C
:100420003F1F0000000080E0F0F8FCFEFFFFFFFF30
:100430007F3F1F1F0F0783C3E1E1E0E0C0000E1FF5
:100440003F7F7FFFF3E0E08000000000000000003D
:10045000000080F0FCFEFFFFFFFF7F3F0F03010164
:100460000100000080F0FEFFFFC7C1C1C1C1C1C1D2
:10047000C1C1C1C1C1C1C1C1C1C1C1C1C1C1C1C16C
:1004800001C1F0FEFF3F0F070F0D0D0D1D191919CA
:10049000193131313171616161E1C1C1C181000046
:1004A0000080E0F8FCFFFFFFFF2F170F038180C0E3
:1004B000E0F0F8FCFEFFFFFFFFFFFF7F0100000000
:1004C0000000000001010307070E1E1C3870E0F059
:1004D000F8FEFFFF7F1F0F03000100000000000077
:1004E000000000000000000000000000000000000C
:1004F00000000000000000000000000000000000FC
:1005000000000000000000000000000000000000EB
:1005100000000000000000000000000000000000DB
:100520007EFFFFFFFFFFFFFBF8FCFCFEFF7F3F1F8E
:100530000F07C3FFFFFFFFFFFF7F07000000000062
:10054000000000000000000000C0E0F8FEFFFF7F98
:100550001F0F1F3D7CF8F8F0E08000000000000055
:10056000000000000000000000000000000000008B
:10057000000000000000000000000000000000007B
:10058000000000000000000000000000000000006B
:10059000000000000000000000000000000000005B
:1005A000000001010101010307070703010000002A
:1005B000E0FCFFFFFFFFFF1F030000000000000042
:1005C00000000000C0F078DE2713090E07030000CA
:1005D00000000000000001030F7FFFFC7878F800A6
:1005E000000000000000000000008080808080800B
:1005F000808080008080008080000000000000007B
:1006000080808080808080808080808080808080EA
:1006100080800000000000000000000000000000DA
:100620000000000000000000000000000080F0FE5C
:10063000FFFFFFFF3F0F010000000000000000C0AF
:10064000E0381E0F03000100000000000000000061
:100650000000000000000000000000000003030193
:10066000000000000000000000000E0E0202020266
:10067000020303000F0F000F0F08080808080808FE
:100680000F0F08080808080F0F000000000F0F00E8
:10069000000000000000000000000000000000005A
:1006A0000000000000000000000000C0F8BFFFFFD5
:1006B000FF1F7F010000000000000000F0FCFF7F32
:1006C0007830000000000000000000000000000082
:1006D000000000000000000000000000000000001A
:1006E000000000000000000000000000000000000A
:1006F00000000000000000000000000000000000FA
:1007000000000000000000000000000000000000E9
:1007100000000000000000000000000000000000D9
:10072000000000000000000000301C070E0F070151
:1007300000000000000000000000000000000000B9
:1007400000000000000000000000000000000000A9
:100750000000000000000000000000000000000099
:10076000000000564552533A2056312E3735322D6F
:100770004D696B651F444154453A2033302E313169
:100780002E323031361F54494D453A2031333A34F8
:10079000323A35331F2053564E3A20657239782D40
:1007A000723832301F204D4F443A20202020202024
:1007B000003C0606414E2020202041555320202099
:1007C000424549444520313553656B2033305365EC
:1007D0006B20363053656B20456967656E65005642
:1007E00053000720382053656B2031322053656B4E
:1007F0002031362053656B20001E030153415658AB
:10080000004E756D6D657220546F6E2053636800E5
:10081000534943484552484549545320534348009F
:100820004B4F504945205452494D205B4D454E5544
:100830005D000D416E00494E442E20534348414C0B
:10084000544552003C010A5A6165686C2072756E0D
:10085000745A6165686C20686F63680054696D65DF
:10086000721F5369676E616C411F5369676E616CDB
:10087000421F54696D65721F52657365742053770A
:1008800069746368003C01023136203800205479D5
:1008900070651F204368616E731F20436F756E740F
:1008A00072791F42696E641F52616E6765003C0277
:1008B000094C50342F4C5035202044534D326F6E2C
:1008C0006C792044534D322F44534D580044534DBE
:1008D0002054797000014E59000B4F7074696F6E8F
:1008E0000004486967684C6F7720003C00044E6F35
:1008F0006E65003C040750574D4942555350504DCA
:100900004942555350574D5342555350504D5F53E4
:10091000425553003C0206484F4E5441494A4A5200
:10092000435831202058354331003C0405574C488A
:10093000303858363030205838303020483236443D
:10094000204530313020003C03024D544837595A7D
:100950004C53003C02054347303233594438323956
:1009600048385F3344003C0707475245454E202036
:10097000424C5545202020444D3030372020513204
:1009800038322020204A333031355F314A3330311C
:10099000355F324D4B3333303431513234322020D5
:1009A00020003C010753594D4158202053594D41D7
:1009B000583543003C0106574C544F59534645495E
:1009C0004C554E003C040759443731372020534BD7
:1009D00059574C4B5253594D4158342058494E5851
:1009E000554E204E494855492020003C03074453AA
:1009F0004D322D323244534D322D313144534D5806
:100A00002D323244534D582D3131003C0105486997
:100A1000736B79484B333130003C010543485F31FB
:100A20003643485F3820003C0306466C79736B7987
:100A300056397839202056367836202056393132CA
:100A400020200006466C79736B7948756273616E7D
:100A50004672736B79444869736B792056327832E9
:100A6000202044534D2020204465766F2020594497
:100A7000373137204B4E2020202053796D6158208C
:100A8000534C5420202043583130202043473032EB
:100A90003320426179616E674672736B79584553B2
:100AA0006B7920204D54393978784D4A587120207F
:100AB0005368656E71694659333236205346485340
:100AC00053204A3650524F20465137373720415332
:100AD00053414E204672736B7956484F4E544149EC
:100AE0004F706E4C72734146484432530050726FDF
:100AF000746F636F6C1F547970651F506F776572E8
:100B00001F42696E6420202020204175746F626945
:100B10006E641F52616E676500660103504F534E4D
:100B20004547005369676E616C6172740050504DA7
:100B3000204C61656E67650D6D53656B000C456DEE
:100B40004E756D00043443482036434820384348EE
:100B50002031304348313243483134434831364301
:100B60004800137553000650504D202020584A5419
:100B700020202044534D32202050504D31362050FB
:100B8000504D53494D4D554C5449205342555320D7
:100B90002000312E204B616E616C1F50726F746F9C
:100BA00000024578706F1F1F014475616C2052610F
:100BB00074651F1F4472536368311F447253636826
:100BC0003200003804445220486F636804445220C5
:100BD0004D697474044452205469656600660404C7
:100BE0002D2D2D2D313230203132305831343020FE
:100BF00039302020005461756D656C7479701F4B1D
:100C00006F6C6C656B7469761F416E7363686C61A1
:100C1000671F484F4520556D6B6568721F515545DC
:100C200020556D6B6568721F434F4C204469726597
:100C30006374696F6E005348475131323300540476
:100C4000064578706F6E2045784665696E46656921
:100C50006E20204D697474656C47726F62202000AD
:100C60005472696D20496E6B1F5472696D20536315
:100C7000681F48692E52657320536C6F772F446547
:100C80006C61791F547261696E65721F506965707D
:100C90002043656E005A01062020456E642043659E
:100CA0006E74726500452E204772656E7A651F541A
:100CB00068722E2044656661756C741F4761737598
:100CC0006D6B6568721F5468726F74746C65204F29
:100CD00070656E1F472D5472696D1F472D457870E2
:100CE0006F2D4472006607032D2D2D503120503298
:100CF00020503320475634475635475636475637E7
:100D000000537464722E536368616C741F4375736F
:100D1000746F6D53746B4E616D65731F4175746FA5
:100D20006772656E7A651F5468726F74746C6520A3
:100D300044656661756C7400546F6E6672657120EF
:100D4000114D454E5500411691169C168916841674
:100D50007D16AC1447166C165F16A6141018FB14FB
:100D60005616564100566F696365004D454E552035
:100D70004C4F4E470044656C65746500566F69635F
:100D8000652046696C65005402062D2D2D2D2D2DF4
:100D90004E756D62657220417564696F006601046D
:100DA000506C61794D757465005402064E6F2020B9
:100DB00020204265666F7265416674657220004E40
:100DC00003072D2D2D2D2D2D2D4861707469633154
:100DD00048617074696332486170746963330007F5
:100DE00076603D76616C20763D76616C2020000750
:100DF000280D2900506C617920536F757263651F4F
:100E00004F6E206E6F2054656C656D657472791F2E
:100E100046696C655479706500536F757263651F20
:100E200046756E6374696F6E1F56616C75651F53EE
:100E300077697463681F526174651F4861707469D3
:100E40006300566F69636520416C61726D000342F7
:100E500045574720535449434B532F504F54530049
:100E600005534554204D495450554E4B5400035B97
:100E70004D454E555D205A554D2053544152540016
:100E80006607044E4F4E454558543145585432502C
:100E90004330205047322050423720504735204CB5
:100EA0002D575200454C45207377697463681F4184
:100EB000494C207377697463681F504231207377FF
:100EC000697463681F504232207377697463681FC6
:100ED00050473220496E7075741F50423720496E5A
:100EE0007075741F4C2D575220496E7075740042F6
:100EF000616E644C7565636B65004B616C004D758C
:100F00006C7469706C696B61001802036175732001
:100F10002B3D203A3D00036D6F64650A25207175F5
:100F200065207363680007536C6176650012424761
:100F300000414E41000F504232000F5042310054E8
:100F400072696D2D202B004C696E6B731F526563A7
:100F500068741F20486F63681F52756E74721F207B
:100F6000457869741F4D656E7565004449414700B9
:100F7000537469636B5363726F6C6C00506F74537E
:100F800063726F6C6C005374617274204E616D6596
:100F900000537461727462696C6473636869726D22
:100FA00000416C61726D205761726E756E670053FF
:100FB00070656963686572205761726E756E67004F
:100FC000476173205761726E756E67004261747479
:100FD00065726965205761726E756E671F496E6133
:100FE0006B74697669746174616C61726D136D0004
:100FF0004B7265757A5472696D1F476173756D6BBD
:101000006568721F416B746976696572652050501E
:101010004D53494D1F4B616E616C20526569686587
:101020006E666F6C67651F4D6F6475730048617005
:101030007469736368652053746165726B650042FF
:10104000040A5069657065722020202050694C6147
:101050007574737072655069657072546F6E20207C
:101060005069654C617574546F6E4D656761536F5F
:10107000756E6420005406064C6175746C7354736D
:1010800074417573784B75727A204B75727A202093
:101090004E6F726D616C4C616E672020784C616E92
:1010A0006720004C61757473741F506965706572B8
:1010B0001F536F756E646D6F6475731F546F6E6828
:1010C0006F656865004C69636874736368616C740C
:1010D00065721F4C6963687420756D6B6568726515
:1010E0006E1F4C6963687420617573206E6163685C
:1010F00013731F4C6963687420616E2053746B62B4
:101100006577656713731F426C69747A206265693D
:101110002050696570004B6F6E74726173740014B7
:1011200015C914EB14FB14E214D5140C150415BFE7
:1011300014B714F21422047C5E0345787078466577
:101140004665694D697453746B0011544F541F0107
:10115000544D45115453571F0153544B11535425AB
:1011600000035B4D454E555D20746F2072656672BD
:1011700065736800746D72314C6174206D61781212
:1011800075731F746D72314C6174206D696E1275C8
:10119000731F746D7231204A6974746572127573AD
:1011A0001F746D61696E126D7300535441540009D0
:1011B00066726569004D4F44454C5741484C0020CC
:1011C000464D300A52455441004241434B55502050
:1011D000444F4E45004241434B55500052455354F5
:1011E0004F52454400534156494E470052455354CF
:1011F0004F52494E47004C4F4144494E47005265BB
:1012000073746F7265004261636B75700020464DA8
:1012100000536368616C7465721F5472696D6D650B
:10122000721F4661646520496E1F46616465204FE8
:10123000757400464C204D4F4455530052414E4763
:101240004520434845434B20525353493A000642F8
:10125000494E44494E47004B6F7069657265204D99
:101260006F64656C6C004C4F4553434845204D4FAF
:1012700044454C4C004B4F5049455245204D4F443E
:10128000454C4C0054656D706C61746573104D4530
:101290004E5500012B2A5200202020202020202003
:1012A000202020202020004C4F4553434845204D0E
:1012B0004953434845523F00436C65617220414C9D
:1012C0004C206D697865733F00034A41200B4E4501
:1012D000494E1F035B4D454E555D0B5B45584954C8
:1012E0005D004D6178206D69782065727265696373
:1012F00068743A2033321F1F5B455849545D207A89
:10130000756D2041626272656368656E004E020809
:1013100048696E7A7566676E20204D756C746970C9
:101320006C697A6945727365747A656E2020000D68
:101330004469666600114578706F00015573652039
:101340004F757470757420202000015175656C6CA8
:10135000651F014475616C20526174651F014F6601
:10136000667365741F01466978204F6666736574FD
:101370001F01456E61626C654578706F44521F01B4
:101380005472696D6D656E1F1F1F01536368616C38
:101390007465721F014D4F4445531F015761726EB2
:1013A000756E671F014D756C7470781F01566572FC
:1013B0007A2E2072756E7465721F015665727A2ED0
:1013C00020686F63681F014C616E6773616D2072E6
:1013D000756E74721F014C616E6773616D20686F6A
:1013E0006368004265617262204D4953434845522B
:1013F00020004F5000566F726C6167656E0053435A
:10140000092B0D2A122F00044C314C324C334C3432
:101410004C354C364C374C384C394C414C424C4393
:101420000048010546697273744C6173742000535F
:101430006F757263651F1F4F66667365741F4D7508
:101440006C7469706C6965721F44697669736F7238
:101450001F556E69741F5369676E1F446563696D1C
:10146000616C731F4F6666736574204174005B2D59
:101470003E5D004B5600564F5245494E5354006A4C
:1014800001032D2D2D554D4B0053575220003C028A
:10149000034431364438204C52503C0203416D65C0
:1014A0004A6170457572566F696365004C2E5377BB
:1014B0006974636865730044696167416E610044E3
:1014C000696167537774636800417564696F486147
:1014D00070746963004B616C696272696572756EE4
:1014E0006700436F6E74726F6C7300416C61726D54
:1014F000730048617264776172650047656E65725A
:10150000656C6C0056657273696F6E005472616928
:101510006E657200446973706C6179005B4D454E75
:10152000555D2057454E4E2046455254494700458B
:1015300044495400424541524245490053454C2FCD
:1015400045444954004B4F50494552004245574588
:101550004745004C4F45534348004241434B55508B
:1015600000524553544F524500424541524245496D
:101570000045494E46554547004B4F50494552009E
:10158000424557454745004C4F4553434800434C5F
:1015900045415220414C4C000473494478735448EF
:1015A000527352554473454C457341494C734745FA
:1015B000417354524E0012081200081C0808081CFF
:1015C0000800000822004900220800000000002254
:1015D0007F220000000822004900220800000822A3
:1015E0000049002208000000227F220000000000C5
:1015F000082200490022080000081C0808081C08EE
:1016000000534300475600054665657420566F6CCD
:1016100074734465675F434465675F466D41682046
:1016200020416D7073204D657472655761747473D9
:1016300000465643466D416D5718242F2F0033380E
:101640003B4D6978657200566F726C6167656E001C
:1016500001534847510050726F746F636F6C0047BD
:101660004C4F42414C4520564152530053616665F0
:10167000747920537773004B55525645004B757261
:1016800076656E004D4F4449004578706F2F447267
:101690000048454C492045494E5354004752454E59
:1016A0005A454E004D6F64656C2053656C656374DC
:1016B000004D6F64656C205365747570004C6173E8
:1016C00074204D656E7500526164696F20536574B6
:1016D0007570005374617469737469637300506941
:1016E000657020436F756E74646F776E004D696E20
:1016F0007574656E746F6E00032D2D2D53746D48D7
:10170000746D47746D51746D52454E536569486FE1
:101710006547617351756550312050322050332038
:1017200000042020414E2041555342454944204168
:101730004C4C4F4E434500072D2D2D2D202020765B
:101740003E76616C2020763C76616C20207C767C35
:101750003E76616C7C767C3C76616C414E44202008
:1017600020204F522020202020584F52202020207F
:1017700076313D3D7632207631213D76322076310C
:101780003E7632202076313C763220204C617463E4
:10179000682020462D466C6F702054696D654F6639
:1017A0006676603D76616C20004E616D650006577F
:1017B00061726E31205761726E32204368656170CC
:1017C0002052696E672020536369466920526F6218
:1017D0006F742043686972702054616461202043F3
:1017E0007269636B74536972656E20416C6D436CF2
:1017F0006B5261746174615469636B20204861703D
:10180000746331486170746332486170746333008B
:1018100054696D657200545245303132414747007A
:1018200003536E3D5377720020414243444546477F
:1018300048494A4B4C4D4E4F5051525354555657B0
:1018400058595A6162636465666768696A6B6C6D52
:101850006E6F707172737475767778797A30313211
:10186000333435363738395F2D2E00FEFFFDF6F75D
:10187000F8F9FAFBFC042D2D2D2D54494D31544916
:101880004D32414B4B55477672314776723247762F
:1018900072334776723447767235477672364776BA
:1018A000723700032D2D2D783E30783C307C787CCB
:1018B000663E30663C307C667C6331206332206358
:1018C0003320633420633520633620633720633848
:1018D0002063392063313063313163313263313316
:1018E0006331346331356331360004503120205088
:1018F0003220205033202048414C42564F4C4C431C
:10190000594331435943324359433350504D315079
:10191000504D3250504D3350504D3450504D355045
:10192000504D3650504D3750504D3843483120437C
:10193000483220434833204348342043483520432D
:10194000483620434837204348382043483920430D
:1019500048313043483131434831324348313343D1
:10196000483134434831354348313653574348476B
:1019700056312047563220475633204756342047A9
:10198000563520475636204756372054484953008D
:10199000536368616C746572205761726E756E670F
:1019A00000536368726569626665686C657200669B
:1019B0006F726D61746965726520454550524F4D77
:1019C0000066616C7363686520454570726F6D20B9
:1019D000446174656E00434845434B204D4F444578
:1019E0004C2054494D45525300434845434B204DEC
:1019F00049582F445220534F5552434553004D4FA1
:101A000044454C4C202020200049434820202020E1
:101A100020202000454550524F4D206F666C6F7757
:101A200000E2AEA1A6A4A2C02F25AF0000000000D6
:101A300000000000000000000000000000000000A6
:101A400000000B07000000C0C0C0C0C0C0C0000044
:101A50000000000000000000000000000000000680
:101A6000060000000080E0781E06181E0701000036
:101A700000F8FC8EC66EFCF8070F1D181C0F070837
:101A80000CFEFE00000018181F1F1818000C0E8610
:101A9000C6EE7C381E1F1B1918181806C6C6C6EEDF
:101AA000FC38181818181D0F07C0E0B0988CFEFEFF
:101AB00001010101011F1F7E7E6666E6C686060CD7
:101AC00018181C0F07F8FCE666E6CC88070F1C18F0
:101AD0001C0F07060606C6E67E1E001C1F0300003C
:101AE0000038FCEEC6EEFC38070F1D181D0F0778F6
:101AF000FCCE86CEFCF8040C1D191D0F070000005B
:101B00003030000000000003030000E0F89C869CD9
:101B1000F8E01F1F0101011F1FFEFEC6C6EEFC38C4
:101B20001F1F18181D0F07F8FC0E060E0C08070FD4
:101B30001C181C0C04FEFE060E1CF8F01F1F181CBF
:101B40000E0703FEFEC6C6C606061F1F1818181885
:101B500018FEFEC6C6C606061F1F0000000000F8DD
:101B6000FC0E06CECCC8070F1C18181F0FFEFEC0B7
:101B7000C0C0FEFE1F1F0000001F1F0606FEFE065F
:101B8000060018181F1F18180000060606FEFE069D
:101B90000E1E18181F0F00FEFEF0381C0E061F1F29
:101BA00003070E1C18FEFE00000000001F1F18187F
:101BB000181818FEFC187018FCFE1F1F0000001FEC
:101BC0001FFEFC70C080FEFE1F1F0000030F1FF8E9
:101BD000FC0E060EFCF8070F1C181C0F07FEFEC6B5
:101BE000C6EE7C381F1F0000000000F8FC0E060E39
:101BF000FCF8070F1C1B1E0F1BFEFE86C6EE7C3872
:101C00001F1F03070E1C18387CEEC6C68E0C0C1C5A
:101C100018181D0F070606FEFE06060000001F1F0F
:101C2000000000FEFE000000FEFE070F1C181C0F47
:101C300007FEFE000000FEFE01070E180E0701FE63
:101C4000FE008000FEFE1F0F0603060F1F1E3EF063
:101C5000E0F03E1E1E1F0301031F1E7EFEC0C0FEDD
:101C60007E0000001F1F0000000686C6E6F67E3ECE
:101C70001F1F1B191818180000000000000018187A
:101C800018181818180060606060E0C0060F1F1B6D
:101C90001B1F1FFEFEE060E0C0801F1F1C181C0FF2
:101CA00007C0E0E06060E0C00F1F1C18181C0C802B
:101CB000C0E060E0FEFE070F1C181C1F1FC0E060A4
:101CC0006060E0C00F1F1B1B1B1B01C0F8FCCEC6D1
:101CD0000E0C001F1F00000000C0E0703070E0C05C
:101CE00003C7CECCEE7F3FFEFEC0E0E0C0801F1FEA
:101CF0000100001F1F000060E6E600000000181F42
:101D00001F180000000000E3E300307060607F3FB8
:101D100000FEFEC0E07038181F1F03070E1C1800DD
:101D20000006FEFE00000000181F1F1800E0E06023
:101D3000C060E0C01F1F0001001F1FE0E0C0E0E026
:101D4000C0801F1F0100001F1F80C0E060E0C08036
:101D5000070F1C181C0F07E0F0703070F0E0FFFF59
:101D60000E0C0E0F07E0F0703070F0E0070F0E0C55
:101D70000EFFFFE0E0C06060E0E01F1F0000000019
:101D800000C0E06060606060191B1B1B1B1F0E60C1
:101D900060FEFE60600000000F1F181C0CE0E000F9
:101DA0000000E0E0070F1C1C0E1F1FE0E000000019
:101DB000E0E001070E180E0701E0E0000000E0E09F
:101DC0000F1F180E181F0F60E0800080E060181CC5
:101DD0000703071C18E0E0000000E0E007CFCECCCE
:101DE000EC7F3F6060606060E0E01C1E1E1B1B1902
:101DF0001900000000000000006F0000070007004D
:101E0000147F147F14242A7F2A1223130864623655
:101E1000495522500005030000001C2241000041EA
:101E2000221C0014083E081408083E080800503020
:101E3000000008080808080060600000201008047E
:101E400002003E49453E0000427F40006251494643
:101E50000041494936001814127F002745453900D2
:101E60003E494932000179050300364949360006EA
:101E700049291E00003636000000563600000814BE
:101E800022411414141414412214080002015109AF
:101E90000600060909067E0909097E7F4949493677
:101EA0003E414141227F4141221C7F494949417FB6
:101EB000090909013E4149497A7F0808087F004124
:101EC0007F41002040413F017F081422417F404074
:101ED00040407F020C027F7F0408107F3E41414159
:101EE0003E7F090909063E4151215E7F09192946B5
:101EF000264949493201017F01013F4040403F1FCF
:101F00002040201F3F4030403F63140814630708FF
:101F10007008076151494543007F414100020408B0
:101F200010200041417F0004020102044040404073
:101F300040080408100820545454787F484444381A
:101F40003844444420384444487F38545454180892
:101F50007E0901020C5252523E7F0804047800446C
:101F60007D40002040443D007F1028440000417F18
:101F700040007C041804787C080404783844444405
:101F8000387C14141408081414187C7C0804040801
:101F90004854545420043F4440203C4040207C1C82
:101FA0002040201C3C4020403C44281028440C5039
:101FB00050503C4464544C44000836410000007FBB
:101FC000000000413608000808221C08081C2208EE
:101FD0000804027F020410207F20101830180C061D
:101FE00001020408102040804080080420100201F3
:101FF0009CCE003264E2F1003264645A505A64505C
:10200000463C46649C141E465A536572766F2054B3
:1020100065737428382900536572766F2054657390
:102020007428313629004779726F2045696E7374C0
:102030000048656C692045696E73740044656C7472
:10204000615C4E7572666C7565676C657200562DC5
:102050004C6569747700646175657220476173200F
:1020600061757300476173206175730045696E6621
:102070006163686520342D4348006C20642056203D
:102080004E203C20312026201720092000008911F5
:1020900012239B322446AD573665BF74488CC19DD0
:1020A0005AAFD3BE6CCAE5DB7EE9F7F8A2761124FD
:1020B0001FBECFEFD0E1DEBFCDBF11E0A0E0B1E0A9
:1020C000ECE2FFEE02C005900D92A231B107D9F704
:1020D0001EE0A2E1B1E001C01D92A238B107E1F714
:1020E00010E2CEEAD0E204C02297FE010E945F77A0
:1020F000CC3AD107C9F70E9450750C9494770C9490
:102100000000E0916B0694E0E99FF0011124E80FD4
:10211000F11DEA52FD4F84918F5F0895F8948091EC
:10212000760D9091770D78940895E82FF0E0E654BD
:10213000FD4F849108952AE0829FC00111248B599C
:102140009D4F089590916D0691708091BC0586FB1E
:10215000882780F9892708950F93022F24FF03C051
:102160000F7E9DE201C094E2411104C024E04AECDC
:1021700052E00EC04530A0F49091BC0594FF0BC016
:10218000006194E0499FA00111244B57594F24E06E
:102190000E94CA640DC02FEF240F46EE52E006C025
:1021A000941730F02BEF240F4AEE58E10E94EE64B2
:1021B0000F910895442311F04C5E01C040E0CCCF54
:1021C000CF93DF93E5E8F1E080919906108291E0EA
:1021D000918381FF09C092E2928393E29383EF019E
:1021E000259694E2948304C0EF01239692E09283B3
:1021F00082FF09C09FE1988390E29983FE013396A4
:1022000091E29A8304C0FE01319693E0988394E0B2
:10221000908395E0918396E0928384FF09C095E2D4
:10222000938396E29483EF01269697E2958304C008
:10223000EF01249697E0938385FF09C098E2988385
:1022400099E29983DE0113969AE29A8304C0DE0133
:10225000119698E0988399E09C93FD0186FD02C059
:10226000319604C032969BE2ED01998387FF03C04B
:102270008CE280833196DF018AE08D938F5F863117
:10228000E1F78487CF01895791408093570127E177
:10229000258740E099270196242F30E08217930785
:1022A00054F0F901EB57FE4FE081F0E0E85AFE4FA1
:1022B00040834F5FF1CF90919D0690FF0AC08091BF
:1022C00064008B7F809364008091650084608093BC
:1022D000650091FF02C0BF98C79ADF91CF91089522
:1022E00087FF03C0819591E001C090E0E82FFF27B0
:1022F000E7FDF095E85AFE4F808191118195089590
:1023000087FF03C0819591E001C090E0E82FFF278F
:10231000E7FDF095EB57FE4F80819111819508956F
:102320000F931F93CF93DF93D62FC42F022F16E066
:10233000180F442339F0463141F04A3E81F44CEF06
:1023400052E005C04BEC52E002C048EF52E06D2F66
:10235000812FDF91CF911F910F910C94006547FF62
:1023600004C041E20E943D64C1952FEF2C0F27313C
:1023700014F026EF2C0F40E053E06D2F812F0E94C8
:10238000EE64DF91CF911F910F9108950F931F93EA
:10239000CF93DF93D82F162FC42F022F4D3234F056
:1023A0004DE682E18D0F0E943D64CC52202F4C2FD0
:1023B000612F8AEF8D0FDF91CF911F910F91B0CFD9
:1023C000DF92EF92FF920F931F93CF93DF93D82F5B
:1023D000162FF42E27FF03C0E5E0F2E002C0E0E094
:1023E000F2E0C281D3802370E22E81E0821718F1DF
:1023F000C4306CF483E0C802A00111244A555D4F3B
:102400000F2D23E0612F8D2F0E94CA6418C0CD5F6D
:102410000F2D2C2F43EA58E1612F8D2F0E94EE647F
:10242000C0310CF4D6502F2D45E2612F82E18D0F83
:102430000E943D6404C082E028130AC004C0E11079
:1024400007C0C13029F42F2D4D2D612F8D2F9EDF18
:10245000DF91CF911F910F91FF90EF90DF90089542
:10246000873038F4E82FF0E0EE0FFF1FE05CF74F05
:1024700024C08C3050F18431C0F4482F50E0DA0190
:10248000AA0FBB1FA45FBE4F2D913C91803148F431
:10249000FA01EE0FFF1FEF5BF94F80819181281B3E
:1024A000390BC901880F991F0895843248F4E82F29
:1024B000F0E0EE0FFF1FE850F84F80819181089502
:1024C0008E3218F484520C94442380E090E00895F6
:1024D0000E944C75882311F0A895FACF1092A60D92
:1024E00008951F93CF93DF93EC01162F0E94F163A1
:1024F000BE0188E10E94256512FF04C067E182E108
:102500000E94B97410FD11C011FF06C062E972E0AB
:1025100080E30E94256506C043E852E068E38CE151
:102520000E943B654FEC52E002C049E752E024E0D4
:1025300060E086E1DF91CF911F910C94006561E02E
:10254000D0DF0C943F680F93262F00E040E053E06B
:1025500060E10E94EE640F9108951F93CF93DF9383
:10256000C6E110E08C2F0E942569110F182BC15075
:10257000CE30C1F78091990682FF12C08FE10E9490
:10258000CF6924E0829FE0011124137CC12B84E0F9
:102590000E94CF6920E1829FC00111241C2F182BBB
:1025A000812FDF91CF911F91089570E0882399F0DA
:1025B00090E0019725E0289FF001299FF00D11245C
:1025C000E60FF71FEE0FFF1FE05FFA4F808191814A
:1025D0008B509E4F0895FB01E35DFB4F808199274F
:1025E00087FD909508951F93CF93DF93D82F162FD3
:1025F000C4E0DD2391F0612F8D2FD7DF9C01253FB3
:1026000081E0380764F08BE0820F8D1710F08CE0CA
:10261000820FC15029F0D82FECCFC0E001C0CD2FE0
:102620008C2FDF91CF911F910895CF93C62FDBDFC1
:102630006C2FCF91BACF8E3791053CF483382FEFB2
:10264000920734F483E89FEF03C08DE790E008958C
:102650000895FF920F931F93CF93DF938A01C62FA4
:10266000D0E08823D9F0BFDFF82E8823B9F0C80165
:10267000E2DF2F2D30E02150310945E0429FF0018B
:10268000439FF00D1124EC0FFD1FEE0FFF1FE05FC5
:10269000FA4F855F91409183808305C0C801CBDFED
:1026A000C35DDB4F888386E0DF91CF911F910F914F
:1026B000FF900C945E5EAF92BF92CF92DF92EF924A
:1026C000FF920F931F93CF93DF938C017B016A01DD
:1026D000A22EB0900B029B2D9F7D943439F08091F7
:1026E0001E08882309F498C0933479F4B19906C080
:1026F00080913E01E801C80FD11D02C0E80121967A
:1027000083E10E94AF7485E010C0953419F09234D3
:1027100009F088C0B19983C080913E01E801C81BCF
:10272000D10984E10E94AF7484E00E94256981117F
:1027300068C0E114F104F9F481E0C816D104D9F4B9
:1027400080E6B81619F08EE2B81211C010921E0879
:10275000C1E00115110509F0C0E0D0E08B2D0E9409
:10276000F0698EE2B81206C01092540803C0C1701E
:10277000DD2701C0B12C4091410150914201C41BA1
:10278000D50B80915408813071F440911402B199B5
:1027900005C084E14802A001112403C0552747FD6C
:1027A0005095C40FD51FCC16DD0644F48B2D0E9426
:1027B000F06983E10E94AF74E6010AC0CE15DF051F
:1027C0003CF48B2D0E94F06984E10E94AF74E70114
:1027D000C017D10749F1B19903C08FEF8093B406B8
:1027E000209751F48B2D0E94E06917FF02C083E10E
:1027F00001C084E10E94AF748A2D83700E945E5EE6
:1028000013C0CC27DD27C01BD10B85E00E94F069E7
:1028100084E00E94F0698DCF953421F47BCFE801EC
:1028200021977FCFE80185CFCE01DF91CF911F9116
:102830000F91FF90EF90DF90CF90BF90AF900895F1
:10284000552747FD5095772767FD7095992787FD98
:10285000909531CF20911708F3CF462F209117087C
:1028600060E0EECF462F50E02091170860E070E066
:1028700022CF90914A01911103C0811106C00895A1
:10288000811103C08FEF890F01C080E080934A015E
:102890008EEB809349010895E0914A01F0E0EE0F3C
:1028A000FF1FE55BFE4F918380838FEB809349018F
:1028B000089580916F062AEF829FC0011124880F2E
:1028C000991F20913A0130913B012817390720F4D4
:1028D00090933B0180933A010895EBE4FEE037A129
:1028E000303180F420A541E0420F40A7DF01A20F64
:1028F000B11DA20FB11D8D939C93403108F010A61D
:102900003F5F37A3089590E08C5F9E4FE6CF90E045
:10291000E4CF8093160290E04097DFCF0F931F9390
:10292000CF93DF93EC018091760681FF07C1809100
:10293000870686FF89C012E001E00E94CF6A8F3FC0
:102940002FEF920781F029A9211104C08F31A9F737
:1029500009ABF3CF213011F419ABEFCF223069F777
:102960008AAB19AAEACF8EA1813041F53FA133236A
:1029700009F452C029A5FE01E20FF11DE20FF11D7D
:10298000808191812F5F203108F020E029A731500C
:102990003FA32091C60121FDE0C097FD02C021E1C7
:1029A00001C028E22BA32FE12AA722E02BA78CA7A6
:1029B0009DA718AA84E08FA72EA32EC0811106C060
:1029C0008091750D8D3340F186E025C0823021F174
:1029D0009AA99078833049F4992329F08BA18150EA
:1029E0008BA3811119C084E016C0843021F499238F
:1029F00099F083E00EC0853039F48BA181508BA310
:102A000081110AC081E007C0863031F4992321F09A
:102A100084E18BA385E08EA38EA1823009F49DC052
:102A20008BA98F5F8BAB8A3008F497C01BAA8DE10E
:102A30008AA781E08BA798A1911101C080E08CA7A3
:102A400018AA83E08FA789C098A189A1992311F0C2
:102A5000846001C08B7F89A38EA1813081F5C79AE4
:102A60002FA1222349F189A531E0380F39A7FE01B2
:102A7000E80FF11DE80FF11D808191819DA38CA3CA
:102A8000303108F019A621502FA32091C60121FD55
:102A900064C097FD02C021E101C028E22BA329A157
:102AA0002C7F97FD226029A389A18BBBC7988FE15A
:102AB0008AA382E08EA351C089A18BBB4DC0811136
:102AC0000CC0C79A89A1836089A38BBB8091750DC7
:102AD0008D3308F441C086E02FC0823009F43DC038
:102AE00089A18BBBC79ABF9800C0000000C086B305
:102AF0008078BF9A9EA1933049F4882329F08BA156
:102B000081508BA3811128C084E016C0943021F439
:102B1000882311F183E00EC0953039F48BA18150E8
:102B20008BA3811119C081E007C09630A9F48823D6
:102B300099F084E18BA385E08EA30EC080919D0661
:102B400081FD0BC08091730686FB882780F998A1D0
:102B5000981711F0C79A01C0C798DF91CF911F91C4
:102B60000F91089590916B0690FD02C093E0892724
:102B7000E82FF0E0E25BF74FE081E7FDE95FE595E4
:102B8000E595E5951E1624F0EE2321F0E19502C0AF
:102B900080E801C080E0E83008F0E7E0F0E0ED54C4
:102BA000FD4FE491EE2319F099E0909355018E2B9F
:102BB0000895853030F46FEF680F8091040735DD9C
:102BC00024C08D3080F4E82FF0E0EE0FFF1FEC5CA6
:102BD000F74F8081918197FD079653E095958795F2
:102BE0005A95E1F712C08D3170F4E82FF0E0EE0F46
:102BF000FF1FEA5FF74F808191816AE070E00E94D9
:102C00000C77CB0102C080E090E015CD482F8330D7
:102C100021F0882321F0E82F03C0E0E001C0E3E0C9
:102C2000F0E0EE0FFF1FED5EFE4F8081918144309A
:102C300080F42091880630E002C0359527954A95AA
:102C4000E2F720FF06C020E038E0A901481B590B3D
:102C5000CA0108951F93CF93DF9310E0C0E0D0E046
:102C6000812FD4DFC80FD91F1F5F1430C9F7C05898
:102C7000DF4F8D2F90E0DF91CF911F910895CF937B
:102C800080916B068170C2E0C81B8C2FBFDF6C2F58
:102C90000E944C3D2091BC0525FF05C00F964F9723
:102CA00028F080E004C081319C4FDCF781E0CF91B7
:102CB0000895E3E1F1E040E0842F806487B9369A1B
:102CC0003699FECF24B135B1369A3699FECF84B10C
:102CD00095B1820F931F819391934F5F483061F7B5
:102CE000089578941F920F920FB60F9211248F932C
:102CF000809112018F5F809312018F910F900FBE10
:102D00000F901F90189578941F920F920FB60F9204
:102D100011242F938F939F93CF93DF93EF93FF9380
:102D2000F89487B78F7B87BF78942091CA018091F0
:102D3000CC0190917606882359F090FF07C08091CE
:102D4000810E820F8093810E87FF02C01B9A01C003
:102D50001B9891FF50C08091870686FF22C0EBE44C
:102D6000FEE087A5882309F446C080910A028111FC
:102D700042C080919B0085FF0DC080A991E0980F13
:102D800090ABEF01C80FD11D8AA580939C0087A549
:102D9000815087A787A581112EC086A1823059F561
:102DA00026C080915F09811126C0EBE4FEE086A178
:102DB000823009F583A1882311F081501BC021A125
:102DC000C79A82A180FD09C02D7F84A195A196FD9F
:102DD0002260880F991F95A384A381E082278BBB73
:102DE00081A3C79882A1815082A3811104C083E08E
:102DF00086A385E083A3F89487B7806487BF78941F
:102E0000FF91EF91DF91CF919F918F912F910F9033
:102E10000FBE0F901F90189578941F920F920FB6C7
:102E20000F9211242F933F934F935F936F937F9350
:102E30008F939F93AF93BF93EF93FF9381B7845684
:102E400081BF88EC91E00E94F6720E94FF69809138
:102E5000AE0D82608093AE0DE2E0F1E080818150A2
:102E600011F0808304C084E6808381E081838281C5
:102E7000815011F0828305C08AE082838381816062
:102E80008383FF91EF91BF91AF919F918F917F913C
:102E90006F915F914F913F912F910F900FBE0F90C7
:102EA0001F90189578941F920F920FB60F921124CD
:102EB0002F933F934F935F936F937F938F939F9342
:102EC000AF93BF93EF93FF932091800030918100E7
:102ED000F89480917D008F7D80937D00789480911F
:102EE000B1069091B206A901481B590BCA019695EB
:102EF00087953093B2062093B106409123019C013F
:102F0000215A3F402F3D3E4230F12FEF240F283011
:102F100028F59C012152334027373540F0F424E650
:102F200020931502E42FF0E0EE0FFF1FEE5DFE4F41
:102F30009C012C5D354050917106565F529FC00137
:102F4000539F900D11246AE070E00E940C7771830A
:102F500060834F5F03C041E001C040E04093230124
:102F6000F89480917D00806280937D007894FF9139
:102F7000EF91BF91AF919F918F917F916F915F91F1
:102F80004F913F912F910F900FBE0F901F9018956A
:102F900092EC980F81E0973008F080E00895FC01F2
:102FA0008081882359F0843218F085520C94732361
:102FB000815056DA40E060E00C94C17408959C01A1
:102FC00055E0359527955A95E1F7280F391FAC0143
:102FD000440F452F441F550B241B350B892F990F88
:102FE000990B8595820F931F08959DE7980F9B3F3E
:102FF00088F08E57E82FF0E0EE0FFF1FEE5FFA4FDC
:10300000808186171CF46083862F0895481714F476
:103010004083842F089544E66CE9E7CF982F809190
:103020005C0284FF03C081E0923009F080E00895E3
:1030300049E284029001112435952795359527950D
:1030400087FD815C86FB880F880B80F9A901481BEE
:10305000510987FD5395CA0108954F925F926F926F
:103060007F928F929F92AF92BF92CF92DF92EF9218
:10307000FF920F931F93CF93DF93782E642E8823B4
:1030800009F4D6C086E1781621F09AEE791203C0D1
:10309000D1C081E0D5C0872D992787FD909597FFF6
:1030A00003C0919581959109873191056CF00E943B
:1030B0006569982F81E017141CF49111C1C0BAC042
:1030C000992309F4BDC0B6C0872D87FD81958A304C
:1030D00040F4825F0E94256917140CF4B1C091E09E
:1030E000A5C08A50E82EF12C6701CC0CDD1CE6014E
:1030F000CE0DDF1DCF55DB4F8A818F7009F49AC04A
:1031000094E0961530F4F701E256F94F90819170F2
:103110008AC05880498009D8811107C08FEF850D7A
:103120009FD98C01898184DF0EC0823041F48FEFFA
:10313000850D96D98C018981815092D904C080E097
:1031400090E000E010E02A812F70822E912CF40193
:103150003197EE30F10508F071C0EA5BFF4F0C9437
:103160005D7717FF35C011950195110931C017FF23
:1031700033C01195019511092FC001E0060D402FB4
:1031800060E0852D6ADF182F402F60E0842D65DF19
:103190002A812F70253061F4112309F44FC0882350
:1031A00009F44CC08A8182958F7059F591E031C045
:1031B000263019F41111F6CFF2CF982F91271EC0A7
:1031C00008171907D9F5EECF0817190759F736C0B0
:1031D000801791073CF332C0081719071CF32EC063
:1031E000F601E255FE4F91819095991F9927991FFD
:1031F00005C0F701E256F94F908191709111D2CF3D
:1032000008C089300CF08F5F41E0460D60E025DF9B
:10321000982F2A812F7030E02C30310524F4F701EB
:10322000E256F94F908317143CF081E0892708C0DB
:10323000862F06C080E004C0892F02C090E0E9CF4D
:10324000DF91CF911F910F91FF90EF90DF90CF9082
:10325000BF90AF909F908F907F906F905F904F90B6
:10326000089540E060E0F9CE80915806FADF8111C0
:1032700013C080913A0190913B01892B69F410921F
:103280006B0E8091750D9091B306981749F080935D
:10329000B3068BE49EE042CB81E080936B0EF1CFCE
:1032A0000895CF93DF93C62F20914802222339F04F
:1032B00090934A0280934902DF91CF91089564E090
:1032C00010D90E943F68C11103C08091550601C00A
:1032D00089E10E940D68FCD8D1E00E944C758823DA
:1032E00019F0DF91CF91F4C88091AE0D833019F4BD
:1032F000A8951092AE0DCC2319F0D0936B0E02C09E
:1033000010926B0EB1DFE9CF60E0CBCFE0914A01C4
:10331000E43018F08DE192E0F7CF2FEB20934901D4
:10332000EF5FE0934A01F0E0EE0FFF1FE55BFE4F19
:1033300091838083089580916A0680FD16C0B9DC70
:103340009EDC811112C066E080E592E0CAD80E943E
:103350003F68BED8AEDC88DFA89591DC811105C03E
:103360000E944C758823B1F3B3C80895DF92EF92A1
:10337000FF920F931F93CF93DF9380916A0681FD95
:103380008FC0C091FA04F0900C068091990682FDDE
:103390000CC08C2F8873883041F0803131F080323E
:1033A00021F0C77CC860C093FA04E12CDD24D394DB
:1033B000D4D8182F85E20E94CF69082FD12FDC279F
:1033C0006E2D62608AE292E08CD8D0FF03C060E08C
:1033D00082E0B9D8D1FF03C061E087E1B4D8809121
:1033E000990682FF1AC08D2F8C7051F0612F70E00A
:1033F000759567957595679563706B5E8CE2A3D83C
:103400008D2F8073F9F0612F70E044E0759567951A
:103410004A95E1F763706D5F13C0D2FF03C062E0AD
:103420008CE291D88D2F887369F013FF02C063E09E
:1034300007C014FF02C064E003C015FF03C065E0CD
:1034400081E481D88091990684FF0AC0802F8F255E
:10345000837061F0602F6370655E86E574D806C086
:10346000D6FF03C066E086E56ED80F2DD7FF03C0F8
:1034700067E08BE668D80E943F68DD2021F028D8FD
:1034800034E0E32E01C0E12C1C1302C00F1541F003
:103490000E944C75811104C0E7DEA895D12C88CF1D
:1034A000DF91CF911F910F91FF90EF90DF900895E2
:1034B0008111FFD980913A0190913B01009709F069
:1034C000019720913901222361F0209177064AEF7C
:1034D000249F90011124220F331F8217930708F4B1
:1034E000C90190933B0180933A01BECE1F93CF93C5
:1034F000DF93C8E1D5E090E0888111E0190F8823BF
:1035000029F0AFDE882311F0812F05C0912F2A9674
:10351000143091F780E0DF91CF911F9108958F9241
:103520009F92AF92BF92CF92DF92EF92FF920F9352
:103530001F93CF93DF93EC01A62EB12C6501CC0C29
:10354000DD1CF601E95EFD4F008111818981882330
:1035500009F457C08D809E80888181500E9430126E
:103560007C018981853038F4833050F4813079F0E2
:10357000823091F039C08530A1F0863071F134C0CD
:10358000F7FE03C0F194E194F108833029F481E05F
:103590008E149F043CF125C081E0E814F90414F175
:1035A00020C08881F5DC882369F08AE09701829F3A
:1035B0007001839FF00C1124F4018E9F40018F9FB6
:1035C000900C1124E818F908FFE1EF0EF11C81E0DE
:1035D0002FE3E216F10430F004C081E0E814F904AE
:1035E00009F080E0E82EF12C8A81811104C0EF28D7
:1035F00029F081E01BC035DE8111F9CF00E010E039
:1036000014C08A81882331F02CDE81110BC00FEFAA
:103610001FEF0CC08B81843040F09C81907681E05C
:1036200029F403C080E091E002C080E090E0892BA3
:10363000F501E95DFD4F5F01F080209105019B815F
:1036400021FD2EC0933059F48A810E94CF69F8166B
:1036500089F1FF24F394F80E00E010E02CC08130D3
:1036600041F4F11003C0292F2D7FB1F0913089F47E
:1036700021C0F1E0FF120CC08FEF890F823040F4BF
:1036800080E000E010E09230B1F4E2E0FE2E13C0E2
:1036900080E0913219F40CC000E010E0F82E0BC06D
:1036A000FF24F394913209F0F12C0FEF1FEF03C0C8
:1036B0000FEF1FEFF12CF50180838C8187FD03C094
:1036C000F1100AC07BC088818532D0F38552C4D7FF
:1036D000882309F473C0F4CF17FF04C08B818330B3
:1036E00028F46CC00115110509F055C08C81807655
:1036F000803211F4CE0153DC8C81877059F1813016
:1037000021F52F81822F98858C3FF1E09F0740F0B3
:1037100040E050E060E070E084E0820F23D70DC00D
:10372000853F21E0920748F0FC01EE0FFF1FE85EA5
:10373000FE4F8081992787FD90952F2D30E02150F5
:103740003109820F931FC9D805C060E070E08F81F6
:103750000E94B4748C818076803411F4CE011FDC19
:103760008C81282F287181F08695869586958370A7
:1037700090E0029724F0283121F48FE003C08DE01F
:1037800001C08EE00E94AF748B8183508E31A0F017
:103790000FEF1FEF13C01016110684F40F5F1F4FB9
:1037A0008B813AE0839FC0011124439708171907C2
:1037B0002CF000E010E002C001E010E0F601E95E4C
:1037C000FD4F11830083DF91CF911F910F91FF90E7
:1037D000EF90DF90CF90BF90AF909F908F90089523
:1037E0001F93CF93DF93C4ECD5E010E0612FCE019F
:1037F00096DE29961F5F1830C9F7DF91CF911F9190
:1038000008959F92AF92BF92CF92DF92EF92FF9274
:103810000F931F93CF93DF9310925308809112015F
:1038200002B7909112018913F9CF10E0182B41DAF9
:103830008EE587B91BBA8FE18ABB00C099B38FEFC1
:103840008ABBECE0F2E08781882311F080E202C0BD
:10385000892F807E8483292F207C8081281759F02E
:103860008074880F90783181891711F0315001C030
:103870003F5F3183208382819381891711F0838395
:1038800081838091760D9091AD06282F291B20937E
:103890003C018093AD0680910A02811106C060E070
:1038A00086EF97E00E94024801C0A89580913C01F4
:1038B000882309F4CCC2C4E3D1E080911C0888239A
:1038C00019F0815080931C08C5D92B813C81821747
:1038D000930741F09C838B831A82198281E0809345
:1038E00039012DC060916C06665F49F180913D0100
:1038F000823328F188818F5F8883803100F189814C
:103900009A8101969A838983188247E751E0649FE0
:103910009001659F300D11242817390780F48F71AD
:103920009927019761F48091C6018D7F8093C6012C
:1039300086E00E9489146DE280E10E94B9740E94C1
:10394000CB310E94E63080911502882319F0815016
:103950008093150280E00E94B05E0E94F1630E9495
:10396000B968D82E80910A028111B4C13D2D3F70F3
:10397000A32E4AEFA40EC0915D02C43021F0C330E3
:1039800019F4C4E001C0C8E057E05A1508F495C026
:103990008D2D807F803209F490C08A2D86950E94FB
:1039A00081109091870690FD04C0CC24CA94C80E63
:1039B00003C0E4E0CE2EC81A6C2D809104070E944B
:1039C000F312B82E6C2D0E9415137C01C1110CC08E
:1039D000EC0197FF04C0CC27DD27C81BD90BD59578
:1039E000C795D595C795CF5F82E0C8120FC080916B
:1039F0005C0280FD02C0912C03C099249394C2E024
:103A00000E94A210882319F0C19501C0912CDD27D6
:103A1000C7FDD095A0FE03C0CE0DDF1D04C0F70189
:103A2000EC1BFD0BEF01209721F08D2F8F2587FFD9
:103A300011C091100FC0EF2869F040E050E06C2DEC
:103A40008B2D0E9429138D2D0E94F06986E10E9422
:103A5000AF74C8C39E0124583F4F293F310548F435
:103A6000AE016C2D8B2D0E9429136C2FC7FF18C03F
:103A700016C01C161D061CF44DE750E002C043E8BA
:103A80005FEF6C2D8B2D0E942913CE0183589F4F21
:103A90008B3F910508F0A6C36C2F1C160CF46195A2
:103AA00067FD6D5F65956595772767FD7095645C2B
:103AB0007F4F85E10E94B47495C38D2D8F7B71F487
:103AC0008091B406B1998AC38F3F31F08F5F883CF3
:103AD00019F48FEF6DEBD62E8093B406EFE3F1E08F
:103AE00080914C0890914D0820813181281B390B21
:103AF00037FF02C0215E3F4F55E0359527955A9517
:103B0000E1F72115310561F024813581281B390B3E
:103B100037FF02C02F5F3F4F3595279591838083F4
:103B20009583848380916D0685FD04C080911A0879
:103B3000882311F020E030E033832283CCE0D2E010
:103B40002D818981821B8F3F09F480E087FD8F5F83
:103B500085958887982F990F920F9D838D29A8DCD2
:103B6000F0908306F7E0FF0EE0914A01F0E0EE0FDF
:103B7000FF1FE55BFE4F208131812E59354409F04E
:103B800040C08091760881113CC02885222371F0C5
:103B90008E81332727FD3095F901E80FF11D87FD50
:103BA000FA95CF010E941B138E831886E091C704FB
:103BB0008E2F807E31F1E295E695E770F0E0E430FB
:103BC000F10554F4EE0FFF1FEA5BF74F20813181BE
:103BD0003C5F60E078E00CC0EE0FFF1FE050FB4F51
:103BE0002081332727FD309523583F4F6AEF70E03F
:103BF00047E0429FC001439F900D11240E94F87638
:103C0000F62E80911602F81619F08F2D0E94891455
:103C10008091730687FF3CC0809156018823C1F1D3
:103C2000809155018823B1F18091AC0687FD03C0D6
:103C30008F5F8093AC0682E00E94B215982F9F7729
:103C400089F02091AC06921728F51092AC06D1109D
:103C500021C0D82ED094DD1CDD24DD1C83E68D1917
:103C6000D82E18C083E00E94B215982F9F7791F04C
:103C70002091AC06921770F41092AC06D1100AC0D5
:103C8000D82ED094DD1CDD24DD1CF4E6DF0E02C04E
:103C90001092550181E080935601E0901202FF24BA
:103CA000E7FCF094C3E0D5E08881882371F085308B
:103CB00031F00E94D915992787FD909501C0C70161
:103CC0000E941B13FE0131978083229625E0C131AB
:103CD000D20751F78091490290914A020097B1F0C2
:103CE00060E00E9471120E944C759091AB0699237E
:103CF00039F0811128C010924A021092490223C063
:103D0000882309F181E08093AB061DC01092AB06B9
:103D1000C0914901CC2331F01092490187E10E9402
:103D2000AF74DC2E84E180933E01D0920B02E091CF
:103D30004A01F0E0EE0FFF1FE55BFE4F0190F081BE
:103D4000E02D8D2D09950E943F68C091650088EC9B
:103D500091E00E94E272882311F084E105C0809115
:103D6000800E882321F081508093800E06C08091C0
:103D700063008695817080937F0E80917F0E809383
:103D80004702882309F42CC28091730685FD28C25E
:103D9000CF7EC09365008091750D8F71823009F0E0
:103DA00054C08091210190912201AC01A4E0440F04
:103DB000551FAA95E1F797FD0796BC01F3E07595AD
:103DC0006795FA95E1F720915706332727FD30953F
:103DD0002A5F3F4F629FC001639F900D729F900DBD
:103DE0001124840F951F20916D0626FD05C060915A
:103DF00000017091010102C060EF70E00E94F8764E
:103E000080913D01680F711D6F5F7F4F75956795BC
:103E100060933D018091AA06805F8093AA0681117C
:103E200014C080915606681780F4623370F06EE219
:103E300081E10E94B97480916D0683FF06C082E320
:103E400090E090933B0180933A01109239018EE506
:103E500087B9369A3699FECF84B195B19093010116
:103E6000809300018091AE0D833019F4A8951092D3
:103E7000AE0D2091120182B7909112012913F9CF52
:103E800090E0922B801B910B209108013091090149
:103E90002817390720F49093090180930801809135
:103EA0000501882309F419C10091AF061091B006ED
:103EB0000F5F1F4F1093B0060093AF068091C704A9
:103EC0008F7150E1B52EB81AF7E1FB1508F477C0F1
:103ED000EB2CF12CE701CC0FDD1FC853DB4F3FE08B
:103EE0003B1528F4E701CC0FDD1FC45DDA4F888154
:103EF000C82EC294C69427E0C222D98045E04C1552
:103F000050F05AEF5D1538F4ED2DF0E0EE0FFF1F85
:103F1000EE5EFC4FD0808F7109F44FC0A2D9A82E5D
:103F200080910501F701E15DFD4F7F0181FD43C0F7
:103F30008C2D857049F48081811106C0AA2021F062
:103F40008D2D90E00E946D148FEF8C0D823058F40F
:103F5000F7018081813079F5A1102DC0F2E0CF12F8
:103F600026C0D39424C025E02C1548F4F7018081A5
:103F7000811121C0AA20F9F08981B5D31CC0F2E0DB
:103F8000FC15C8F4AA20B9F024E0C21631F035E0DF
:103F9000C31631F066E970E005C06CE271E002C062
:103FA00068E572E0C8010E94F876892B21F48D2D16
:103FB00090E00E946D14F701A082B39485CF01EACE
:103FC00014E0BEE9AB2EB6E0BB2ECEEACC2EC1E0AB
:103FD000DC2EE12CF12CF8019280892D8F700E944B
:103FE00095108330D9F5F601C081D181209771F405
:103FF000F801C081C7FD06C0C095FAE0CF02E0011C
:1040000011241BC0DD27C7FDD09517C0D7FF14C0F2
:10401000219699F4F701EE55FB4FC081C7FD06C00C
:10402000CF5F2AE0C202E001112406C0DD27C7FDF0
:10403000D095C095D09501C02197892D807F59F0EA
:10404000892D82958F7089300CF08F5F0AD981118C
:1040500002C0CFEFDFEFF601D183C083F501C0814D
:10406000F80182818F708C3071F48081FAD88111CF
:1040700009C0F701EE55FB4F8081F3D8882319F072
:10408000C0E001C0C1E0F80182818F708D3091F4F1
:104090008081E7D8882359F0C1FD0CC0F701EE55A7
:1040A000FB4F8081DED8882321F0C3E003C0CD7FA1
:1040B00001C0C2E0F501C1935F010D5F1F4FF3E046
:1040C000EF0EF11C22E0C20ED11C34E2E316F10423
:1040D00009F081CF85DB10920501809103018823CF
:1040E00009F482C02091AE062F5E822F8F7090E07F
:1040F0000C970CF0207F2093AE068091C7048F713F
:10410000A0E1FA2EF81ACBE4D2E0E12C422F407362
:10411000D42E522F5F70C52E822F8077B82E207F2D
:10412000A22EEF1409F450C08E0103581D4FF80160
:104130008081982F907C9034A9F4D11013C0880FFF
:10414000880F859585958DD8882361F080917606B6
:1041500080FF05C0FE01E258FD4F808101C081E073
:104160000E94AF74F8018081982F907C903849F5B7
:10417000880F880F859585958731B4F087518130F8
:1041800039F018F0823039F01CC0B1101AC006C0E6
:10419000C11017C003C0F0E2AF1213C0FE01E25815
:1041A000FD4F8081A0D20DC0D1100BC05AD88823FA
:1041B00041F0FE01E258FD4F8081805890E00E945E
:1041C0006D14E3942296ADCF1092030180915501B6
:1041D000882351F081508093550106C080E07CCC4B
:1041E000C061D7CDD12C6CCCDF91CF911F910F91B5
:1041F000FF90EF90DF90CF90BF90AF909F90089589
:10420000282F30E0883058F02850310949E0429F8B
:10421000C001439F900D1124875A9B4F089545E09C
:10422000429FC001439F900D11248F5C9B4F0895C6
:10423000813641F40E94F06981E00E94391486EAD7
:104240009EE464D862EE72E180E10C942565CF9320
:10425000C82F8091AC0D80FF03C06EE472E102C0F4
:104260006CE372E188E10E942565C13641F481E684
:104270000E94F0691092AC0D80E00E943914809188
:10428000F40881508093F408811103C081E00E94FA
:10429000AF74CF910895CF93DF93EB01E3E7F8E09C
:1042A0008F3B19F49091730803C08E3B21F49081E9
:1042B0009150988310829281992321F091819F7768
:1042C0009083128290819923A9F0813219F08E385F
:1042D00009F047C020911E08211108C09150988311
:1042E00010820E94F06987E10E94AF7410921E084C
:1042F00080E037C09881843681F4292F30E048303F
:1043000031F050E024173507FCF427E004C02730D3
:104310003105D4F428E0920F17C0853629F4292FEF
:1043200030E0483099F417C0803611F08E3261F4D5
:104330009F5F9083906891830E94F06910920B02B6
:104340001092F50790E080E098830BC0273031058C
:10435000DCF327E004C028303105B4F328E0921BD9
:10436000F3CFDF91CF9108951F93CF93DF93182F51
:10437000D62FC42F662329F06FE0842F0E942D14BE
:10438000C82F80915C024C2F83FF02C0440FD06283
:1043900050E02D2F612F80E60E9428678C2FDF913F
:1043A000CF911F910895FF920F931F93CF93DF93A7
:1043B000182FF62E0AE08AE0189FE0011124CB594D
:1043C000DD4F2FE130E0211B3109029FA001039F47
:1043D000500D1124BE01CE010A960E946C77FF2079
:1043E00049F0BE016A5071094AE050E0CE010E94D6
:1043F0006C770DC0FE0111920A95E9F780910009D2
:104400008883898384E68A838F8188608F83109371
:10441000020982E0DF91CF911F910F91FF900C94E0
:104420005E5EAF92BF92CF92DF92EF92FF920F93B8
:104430001F93CF93DF93EC01C62ED42E88E0681330
:104440000AC0FE013E964591549160E085E40E94C9
:104450003B6508E001C007E010E07801EE0CFF1CAE
:1044600098E0A92EB12CFE01659174918A2D0E94CD
:104470002565BC1448F4FE01EE0DFF1D45915491D5
:104480006A2D85E40E943B65B394229688E0A80ECD
:1044900087E0B812E8CF4FE360E083E40E94DB6579
:1044A000DD20F1F087E06D2D8D1540F4601B660F67
:1044B000660F660F20E04BE385E406C0660F660FCB
:1044C000660F20E042E480E0DF91CF911F910F91D1
:1044D000FF90EF90DF90CF90BF90AF900C9461650C
:1044E000DF91CF911F910F91FF90EF90DF90CF90D0
:1044F000BF90AF9008950F93443051F490915A02B9
:104500009F70913029F449E854E10F910C940065B3
:10451000022F242F45E758E10E94EE640F91089581
:104520009C01220F331F280F391F9595879595956C
:104530008795280F391F959587959595879595951A
:104540008795820F931F0895429643E7489F9001F5
:10455000499F300D1124C901E6E095958795EA95AC
:10456000E1F70895CF92DF92EF92FF920F931F939E
:10457000CF93DF937B018A01D090530895E09D157E
:1045800008F45FC091E09D0D90935308EBE08E9F7F
:10459000E0011124C257DA4F8881882349F0815005
:1045A0000E9430129C01442737FD4095542F03C0D0
:1045B00020E030E0A901D0925308DE80FD2DF87094
:1045C000CF2ED3FC0AC089819A81AA2797FDA09596
:1045D000BA2F280F391F4A1F5B1FAB81B0E011961D
:1045E0000E94CA762C8130E02F5F3F4F442737FD71
:1045F0004095542F0E944177CC2051F089819A81B7
:10460000AA2797FDA095BA2F280F391F4A1F5B1FB5
:10461000D0FE07C050954095309521953F4F4F4FA4
:104620005F4FE114F10419F08D81F70180830115CA
:10463000110529F08E8186958370F8018083C90168
:1046400002C080E090E0DF91CF911F910F91FF9029
:10465000EF90DF90CF90089581E00895E82FF0E08B
:10466000E559F74EE491862F992787FD9095835859
:104670009F4FEE5FE23038F42AE0AC01249FC00186
:10468000259F900D11240895E82FF0E0E559F74E8D
:10469000E491E03F29F1ED3F4CF4EE0FFF0BEA5EB1
:1046A000FA4F8081992787FD90950895ED3FA1F0FD
:1046B000BCF0EF3F09F0A4F48E2F992787FD909569
:1046C00002962FE0289FF001299FF00D1124EB5A4C
:1046D000F74F83859485089580913D0190E008957A
:1046E00080E090E00895CF92DF92EF92FF92CF9317
:1046F000DF9300D0CDB7DEB7F82E1A821982C4DF5F
:10470000EF2DF0E0E559F74E2491422F552747FD54
:104710005095652F752F415F5F4F4F30510590F5D4
:104720004C5A5F4FFA010C945D77AE014F5F5F4FBB
:10473000BE016E5F7F4F8FE0820F14DFEA81F0E0F1
:10474000E75CF94EE491EA831DC024E22A8321E06C
:10475000298318C06CE370E00E940C776B017C0128
:1047600046E260E0C6010E94C174C70125E32A83C6
:1047700009C0E22FEE0FFF0BEA5EFA4F8081992706
:1047800087FD90954A8169810E94C1740F900F90B6
:10479000DF91CF91FF90EF90DF90CF9008950F932E
:1047A0009FE0499FF0011124EB5AF74F4385548550
:1047B000022F0E9466670F9108958F929F92AF9289
:1047C000BF92CF92DF92EF92FF920F931F93CF93FE
:1047D000DF9300D0CDB7DEB7F82ED62EC22EB32E83
:1047E000102F80E28A83E42FFF27E7FDF095E5593B
:1047F000F74EA4908E2D8170982EE0FE20C0AFE081
:10480000AA0DA43008F08CC08BE0A89FD001112421
:10481000FD01EB56FA4F8081882309F481C0AF0176
:1048200000E124E08F2D0E94CA6412FD03C008E15C
:104830000F0D06C00CE10F0D88EFD80E01C00F2D33
:104840008E2D8870882EE3FC1F7B81EFA8160CF458
:104850003DC084EF8A152CF482E08A0D8230F8F096
:1048600035C0AE014F5F5F4FBE016E5F7F4F8FE07F
:104870008A0D78DE2981213011F4106203C02230C4
:1048800009F41063EA81F0E0EF5CF94EE491EA8309
:10489000E7FE02C08C2D9B2DC82EB92E17C012FD2D
:1048A00002C08CEF01C082E0800F9110865F17700C
:1048B000012F212F4C2D5B2D6D2D83500E9466679B
:1048C000E3E3EA0DEA838AEFF80E0AC0882071F16B
:1048D0008DE38F0D212F4C2D5B2D6D2D0E942867B0
:1048E0008E2D867069F0E2FE04C08AE08F0D1B7F7A
:1048F00002C08091620D212F4A816D2D0E943D647E
:104900008A810F900F90DF91CF911F910F91FF90AF
:10491000EF90DF90CF90BF90AF909F908F900895D1
:104920004F5F20E06D2D8F2DE6DD7FCF802FD2CF22
:104930000F931F93CF93DF93C82FD62F042F122FDF
:1049400044E056E10E94006540E3400F212F6D2FA7
:104950008CE08C0FDF91CF911F910F910C943D64EF
:10496000EF920F931F93CF93DF93C42F122F2E2D0F
:10497000DE2DD3709DE7940F9B3F80F043E84C0FF2
:104980008251D6DFDD2359F122E042E850E06EE7A4
:1049900070E08C2F90E00E945B130CC0552747FD00
:1049A00050950E942867DD23D1F0402F612F8C2F76
:1049B0000E942A14C82F80910B028D3B81F48DE751
:1049C0008C0F8B3F40F0EC2FF0E0EE0FFF1FEA5F03
:1049D000FB4FC08101C0CEE782E00E945E5E8C2F5B
:1049E000DF91CF911F910F91EF900895EF920F9368
:1049F000E22E0DE723E8B4DF0F91EF900895CF93F7
:104A0000DF939EE0899FE0011124CB50DC4F8C8521
:104A10000E943119882339F08D850E943119811146
:104A200004C081E003C080E001C082E0DF91CF914B
:104A30000895942F9695691B242F891B0C94CC679D
:104A40009091140281E0191624F0911101C080E0C8
:104A5000819510921402089521E0AC0160E080E09D
:104A60000C9400650F931F93CF93C62F0E94286765
:104A7000B8018C2FCF911F910F910C942565FF9257
:104A80000F931F93CF93DF93182FC42FD22F61154D
:104A9000710591F0FB018491AB014E5F5F4F319640
:104AA000F490222319F00091180801C000E02C2F87
:104AB000612F0E94EE6414C0442329F042E8682F5D
:104AC00087E60E94C864DD2311F004E601C000E01F
:104AD00027E047E0612F86E60E94D767FF24F39422
:104AE000DD23A1F080911608882321F080911E0813
:104AF000882361F0209117084F2D60E08C2FDF9103
:104B0000CF911F910F91FF900C9420148C2FDF9167
:104B1000CF911F910F91FF900895982F862F242FEA
:104B2000492F60E070E0ABCF0F931F93CF93DF93DB
:104B3000182FD62F022FBA018D2F0E942565C1E0B4
:104B4000402F6D2F8C2F811BE8DFC81B8C2FDF912E
:104B5000CF911F910F910895982F862F242F492FC1
:104B60006FE774E18CCF0F9390915A029F7021E010
:104B7000913009F020E000E040E258E10E94EE644C
:104B80000F910895442321F050E0805F0C94286732
:104B90004CEF52E00C940065EF92FF920F931F933D
:104BA000CF93DF93EC01062FF42E1091F507A0911F
:104BB0004808B091490820914A0830914B08EFE32A
:104BC000F1E0868197818A1B9B0B97FDCF9666E06B
:104BD000959587956A95E1F7482F80931B08808506
:104BE0009185821B930B97FDCF9656E095958795FF
:104BF0005A95E1F7982F80931908442311F0B78351
:104C0000A683992311F03187208780911A0881119A
:104C100004C080916D0685FF06C010921B0810929B
:104C2000190810921A0880911B08811108C0809100
:104C30001908811104C082819381892B11F00E948F
:104C40005914E09005098FEFF81609F44DC08091D2
:104C5000540881112DC08091FD08882319F010920D
:104C6000FD081E2DEDDE18166CF41E1510F41F5FE6
:104C7000C9F488818F1518F48F5F888301C018826A
:104C800010E010C0882371F011110BC088818823B7
:104C900019F08150888301C0F88281E08093FD087B
:104CA00001C011500E3271F481E0809354080AC0A3
:104CB000813041F40E3221F080911E08811102C032
:104CC000109254088091F407B1990BC08F3F19F0EE
:104CD0008F5F8D3338F091E090931E0890935408C5
:104CE00001C080E08093F407E092160880911E08CE
:104CF00081112CC0809119088823A1F04881481B9C
:104D000047FD40E08F2D90E0242F332727FD30957D
:104D1000281739070CF04F2D4883E11608F41E2D93
:104D2000109219088881882389F080911B088823B4
:104D300069F0181B17FD10E08E2D90E0212F33270E
:104D400027FD3095281739070CF01E2D003679F114
:104D500090F4023409F46BC028F40132E9F10E3208
:104D600031F184C0043409F442C008F46EC0053443
:104D700009F44DC07BC0053609F44BC040F403363E
:104D800009F466C0B0F5023609F454C06FC00E389D
:104D900001F10F3B39F0013809F068C010921E088C
:104DA00081E022C0188210921E0810E05FC08FEFD1
:104DB000F81609F45BC081E090911E08911180E023
:104DC00080931E08882309F451C081E08093540821
:104DD0004DC08EE80E94F06980911E08882319F06A
:104DE00010921E0843C080E00E9439143FC01E1577
:104DF000E9F1EE20D9F180911E08811137C01E150E
:104E000010F41F5F01C010E010920B022FC011239D
:104E100069F1EE2059F180911E08811127C01123FC
:104E200019F0EE24EA94E10E10920B021EC0888164
:104E30008F15E1F080911E08811118C088818F15AF
:104E400010F48F5F0DC018820EC08881882371F026
:104E500080911E0881110AC08881882319F0815031
:104E6000888301C0F882E11608F41E2D20911E08E7
:104E700021110AC031E08091410190914201892BBA
:104E800009F430E0832F01C081E080931D08109366
:104E9000F507222311F082E001C081E08093180819
:104EA00010920509DF91CF911F910F91FF90EF9024
:104EB0000895AF92BF92CF92DF92EF92FF920F933D
:104EC0001F93CF93DF93C82F8FE596E1C5DD4AE0AE
:104ED0006C2F88EF98E060DEC090F808B090F5077E
:104EE00086E0CE3211F0C03671F48C1578F489EF7B
:104EF0008C0D809306098C2F0E94F0698FE59BE44E
:104F00000E94861962C08C1508F45FC081E080930E
:104F10000509E12CF12C18E064E076E1812F0E9474
:104F20002565AE2C41E34E0D612F8CE00E94C864D4
:104F3000E701CC0FDD1FCE5FDA4FD12CCA1005C0C0
:104F4000BD1003C00091180801C000E080911E0848
:104F5000882309F486C0D1101BC0002329F062E227
:104F600089810E942D14898329812D3018F448EFFE
:104F700056E105C02D3140F42D5F4AEE58E1612F16
:104F80008CE30E94EE6415C02D5147E054E1F7CF49
:104F9000002331F04DE763E888810E942A1488835A
:104FA0004881552747FD5095202F612F8CE60E94A0
:104FB0002867D39482E0D812C1CF185F8FEFE81A28
:104FC000F80A103409F0A8CF41C089EFC80E0EE8E6
:104FD00015E071E3E72EE8E0FE2E6EEF73E18F2D12
:104FE0000E9425654E2D6F2D8CE00E94C864E8015B
:104FF00020E048816F2D88E10E94AC1049815A81E0
:105000006F2D8BE40E9456674B8150E04F5F5F4FDE
:105010006F2D80E60E9456674C8150E04F5F5F4FD6
:105020006F2D8EE70E94566788E0F80EE394055FC7
:105030001F4F88E2F812D1CF6C2D660F660F660FF6
:10504000685F20E04EE780E00E946165DF91CF91CC
:105050001F910F91FF90EF90DF90CF90BF90AF9096
:105060000895D1109DCF80CF1F93CF93DF93C82F8A
:10507000D62F142F47E16BE2DCDC43E06AE28C2F91
:105080000E94DB6543E06BE28FEF8C0F0E94D965D5
:10509000812F69EF0E94EB76382F375D8D2F67E007
:1050A0000E94EB768C0F25E045E0632F8250DF9164
:1050B000CF911F910C94AC67CF92DF92EF92FF9249
:1050C0000F931F93CF93DF93CEE4D8E0498168819B
:1050D0008AE2CADF4A816B8186E5C6DFC0E4D8E098
:1050E0002896AAE3FA2E0DE510E0B7E3CB2E8991BE
:1050F00099919C5FB8010E940C77DD24D394D60E61
:10510000EC2CE61A4D2D6E2D8F2D0E94DB654D2D5A
:105110006E2D81E08F0D0E94DB654D2D6E2D82E09E
:105120008F0D0E94DB6585E0F80E89E4F812DFCF71
:10513000DF91CF911F910F91FF90EF90DF90CF9073
:1051400008954EE654E168E388E60C943B650F93BE
:105150001F93CF93DF93D82F162FC42F022F47FF13
:1051600008C041E28AEF8D0F0E943D6486E08C1BEF
:10517000C82F2C2F43EA58E1612F8D2F0E94EE6437
:10518000DF91CF911F910F9108950F931F93CF93AC
:10519000DF93162F042FC62FD0E0AE014F5F5F4F75
:1051A000202F682F86E60E942867002329F06FEFE2
:1051B000CE010E943214182F812FDF91CF911F91C1
:1051C0000F9108950F93CF93DF93C42FD02FD270F8
:1051D00001FF03C00E94C61102C00E94901100FF8F
:1051E00041C0DD23B9F1CD3274F084ED8C0F0E9403
:1051F00070112091570130E0280F311D87FD3A953D
:105200002150310907C08C2F0E947011282F33279D
:1052100027FD309580915701482F440F4250C1E03F
:105220006C2F681B822F0E942A1490915701482FDF
:10523000552747FD5095292F30E0421753073CF082
:10524000C91B8C0F0E948011CCE2C80F0BC00E94BA
:10525000801107C040915701642F61958C2F0E94E7
:105260002A14C82F8C2FDF91CF910F910895FF92B0
:105270000F931F93CF93DF93182FF62EEA01022F7F
:105280004981453249F4298522952695277048E9B8
:1052900055E10E94EE6411C020610E94AC1089812A
:1052A0008551803150F48F8186FF07C0202F42EF57
:1052B00053E16F2D812F0E940065DF91CF911F91E7
:1052C0000F91FF90089580919B03882329F088E136
:1052D00091E20E94861981E00895CF93DF93C82F51
:1052E00088E00E94256569EC72E188E20E942565EC
:1052F000C13671F028F4CE3269F0C03659F012C0D0
:10530000CE3831F0CF3B71F480E00E94AF740AC018
:10531000D2E001C0D1E08C2F0E94F06981E00E94B0
:10532000391401C0D0E08D2FDF91CF910895CF9334
:105330009091F2079F3F19F468EB72E102C067EAAF
:1053400072E1CBDF813019F0823019F127C0C091B2
:10535000F207CF3F19F40E94586B1BC08C2F0E949C
:105360009B102FE130E02C1B3109CAE0C29FA00145
:10537000C39F500D1124BC01665F7F4F0E946C7764
:10538000EBE9F3E0DF011D92CA95E9F782E00E94A4
:105390005E5E86EA9EE4CF910C948619CF910895C3
:1053A0000F93CF93C82F4FE06AE778E08091EF0723
:1053B0000E94A35D00E12AE04AE758E060E181E055
:1053C0000E94CA644FE360E182E40E94C864809155
:1053D000F007882319F065E772E102C066E672E122
:1053E0008C2F7BDF813019F08230F9F024C080915E
:1053F000F0078823A9F087E592E10E949F1280912F
:10540000EF070E94EB5D882339F087E10E94AF74BB
:1054100082E08093F00709C080E00E94AF7405C06D
:105420008091EF078F5F0E94986183EB9AE2CF91A2
:105430000F910C948619CF910F910895DF92EF92FE
:10544000FF920F931F93CF93DF93EC01062FD42E7F
:10545000F62E18E0E12CFF20B9F0F0FE0EC02D2D45
:1054600048E952E1612F82E10E94FB64AE01612FA5
:1054700088E10E943B65E394185FF694FE018491F5
:1054800021968111FBCFE7CFCD2DCC0FCD0DCC0FC9
:105490002AEF210F4C2F67E082E10E94CC6744EF96
:1054A0004C0F60917708660F660F660F685F20E00B
:1054B00088E10E946165C4DA282FC6E7D8E09981A7
:1054C0008B81882351F03091750D36FF08C08150D3
:1054D0008B83811104C018821CC08FEF8B83809155
:1054E0000B02813681F028F4803249F08E3239F097
:1054F00012C08336C9F088F08E3829F00CC01882AB
:105500001B8281E01AC00E94F06910920B0218827F
:105510001B8282E012C012162CF4EA949E1530F41D
:105520009F5F04C0222339F0911191508B81882311
:1055300011F08FEF8B83998380E0909177089F5FC4
:1055400020E000FF02C0915021F006952F5F283027
:10555000C1F720937808DF91CF911F910F91FF90B1
:10556000EF90DF900895DF92EF92FF920F931F93D9
:10557000CF93DF93C82F85EB91E16EDAF090EE08C0
:1055800080917608811105C04FE06C2F8EEE98E077
:1055900003DB6FEA71E180E00E9425650E94BE6036
:1055A000AC0160E086E60E9456671091EE0880919B
:1055B000F007823021F41092ED081092F0078091EC
:1055C0001F0891E0980F191728F4123068F08FEF38
:1055D000810F0BC094E0980F911738F48CEF810F76
:1055E0008B3018F08AE001C080E080931F08082FFC
:1055F000D0E1EE24E3941013E12CDD24D394D00EFB
:105600002E2D4D2D6D2F82E10E94586780915406FA
:10561000081305C04AE26D2F81E00E94C8644FE084
:105620006AE778E0802F0E94A35DEE2031F0809140
:10563000ED08882311F001E101C000E12FE04AE705
:1056400058E06D2F88E10E94CA64D85FD03411F011
:105650000D2DCFCF80917608882309F475C08091F5
:10566000EE0890915406981302C0D9E501C0DEE718
:105670000E94D45D811101C0D6E98091760682FF37
:10568000DF734AE06D2F8FE295E1D8DE813009F0BB
:105690009AC0D0917808D11105C084E891E50E94A4
:1056A0004C1491C09FEF9D0F923050F50091EE0881
:1056B000009354068093AB0D8C2F0E94F0690E94DA
:1056C0005A5F802F0E94695F8091050182608093FC
:1056D000050181E00E945E5E0E945A5F0E949B1954
:1056E0000E94B619809155020E9483140E94347260
:1056F00080917608823089F2D23009F055C0CDCF42
:10570000D53031F48C2F0E94F0691092F00704C05C
:10571000D33049F48093F0071093EF0780ED99E2BE
:105720000E94861950C0D63019F480937E0804C0B8
:10573000D73039F410927E08109382088EE09FE2F1
:10574000EFCF8093ED083FC0C63638F4C43688F4F6
:10575000C036C1F0C13641F036C0C13829F1CF3B67
:1057600039F1CE3681F50EC08091ED08882359F1CC
:105770000FC0909154068091EE08981709F48DCFD0
:1057800082E00AC010921E088091ED08882319F06B
:105790001092ED0818C081E0809376088C2F0E944B
:1057A000F069109277080FC081E00E9439140BC095
:1057B0001092ED0810927608809154068093EE08BE
:1057C00081E00E94B05E8091ED088823F9F0CF2D32
:1057D000DD27C7FDD095812F90E0C817D907B1F01C
:1057E00061E0610F81E08F0D0E9477618091540626
:1057F000181303C0F092540606C090E0C817D907EA
:1058000029F41093540681E00E945E5EDF91CF91EF
:105810001F910F91FF90EF90DF900895CF92DF924C
:10582000EF92FF92CF93DF93FC01EB019C01DC012F
:105830000E94AB769B01AC01DE010E94C076272F4F
:10584000382F492F5527DF010E94C0766B017C015C
:105850003CE0F694E794D794C7943A95D1F724E6C0
:1058600030E02C1B3D0B0E94AB766E5C7F4F8F4F60
:105870009F4F6C0D7D1D8E1D9F1D24E630E040E086
:1058800050E00E941F77C901DF91CF91FF90EF9008
:10589000DF90CF9008951F93CF93DF93611571052B
:1058A00019F1192F111F1127111F19F091958195C9
:1058B000910977FF0FC0719561957109C0E0D4E03F
:1058C0009E01281B390BC901A9DF9E01281B390B3A
:1058D000C90101C0A3DF112329F022273327281B88
:1058E000390B01C09C01C901DF91CF911F9108952F
:1058F000EF920F93CF93DF93382F862F642F922F41
:10590000332319F02091180801C020E0C091030949
:105910004EE0C49FE0011124CB50DC4F933629F4B4
:10592000032F4C854FDC8C8725C0923629F4032F3A
:105930004D8548DC8D871EC0E02FF0E0E90FF11D9A
:10594000E90FF11DEE0FFF1FEE0DF11DEC0FFD1F16
:10595000EF01011106C0E22E04E62CE9488100D8CF
:1059600008C048814C59E22E04E620E00E94B02491
:1059700084568883DF91CF910F91EF90089590E046
:10598000E92FF0E0E85DF74EE491E81721F0EE230F
:1059900021F09F5FF5CF892F089580E0089582342C
:1059A00030F4E82FF0E0E85DF74E8491089580E24E
:1059B0000895DF92EF92FF920F931F93CF93DF939F
:1059C000F82E162FEA01E22ED02E69EA77E1812F18
:1059D0000E94256500E12E2DAE01612F82E40E9418
:1059E000CA64DD2099F18F2D880F8F0D880F2091CB
:1059F0001E0846E0612F8E5B0E9461654E2D440FAC
:105A00004E0D440F4C5F6FEF610F29E080E40E9460
:105A1000CC6780911E088823C9F0CF0DD11D8881E5
:105A20008111ADDF2D2D41E460E00E942014B7DF2D
:105A3000488150E0282F332727FD30954217530720
:105A400029F08883809117080E945E5EDF91CF91D4
:105A50001F910F91FF90EF90DF900895FF920F93A9
:105A60001F93CF93DF93C82FD62FF42E122F622FC0
:105A7000842F0E94D512FC01E53F81E0F80774F005
:105A80009BE09E0F9F1510F09CE09E0F40E3490F96
:105A9000202F6D2F8C2F0E943D6407C0212F40E5E1
:105AA00056E16D2F8C2F0E94EE64DF91CF911F91F4
:105AB0000F91FF9008957F928F929F92AF92BF9225
:105AC000CF92DF92EF92FF920F931F93CF93DF93CA
:105AD000182FC09106092AE0C29FE0011124C05F7F
:105AE000DA4F83E392E10E942C2543E0612F83EF9C
:105AF00098E052D8409106094F5C60E080E30E9434
:105B0000C864B090F30878E0C72ED12CE3E0AE2E45
:105B1000BD1003C09090180801C0912C81E0D816E8
:105B2000D1F0D81640F08985192D106292E0D9166F
:105B300009F461C072C061E172E18C2D0E9425659B
:105B400001E0911001C000E0292D48856C2D80E313
:105B500039DB88877BC09110A09205096CE3762E13
:105B6000812C8091F507881511F000E001C0092D06
:105B7000409106094F5F282D6C2D872D6FDF9920EE
:105B800099F18091F50788112FC080911D08882315
:105B900059F18E01080D111D080D111DF801E0804D
:105BA000F180FBE0EF1AFEEFFF0A24EFE21621E09E
:105BB000F20624F454EFE52EFF24F39422E048EF9C
:105BC00051E064EF71E0C7010E945B138E159F05E1
:105BD00059F0843FE1E09E0711F480E090E0855F9A
:105BE0009140F801918380838394F6E07F0E24E056
:105BF0008212B7CF2BC0992049F06FE08F700E94BE
:105C00002D148F709985907F982B998749854F70B7
:105C100085E0489FA001112414C0992059F06FE03D
:105C200082958F700E942D148295807F99859F7038
:105C3000982B9987498542954F7095E0499FA0011F
:105C40001124212F6C2D86E60E942867D394E8E06A
:105C5000CE0EF4E0DF125CCFDF91CF911F910F9158
:105C6000FF90EF90DF90CF90BF90AF909F908F907C
:105C70007F9008951F93CF93DF93C82FD62F142FB3
:105C80004EE052E10E943B6540E3410F6D2F8CE0F6
:105C90008C0FDF91CF911F910C94C864BF92CF926B
:105CA000DF92EF92FF920F931F93CF93DF93C82F52
:105CB00084E896E10E942C2543E06C2F8FEE98E05B
:105CC0000E94CC25B090EF08C03611F0CE3649F4D2
:105CD000B09206098C2F0E94F0698BE59DE20E942C
:105CE00086196FEB71E180E10E942565F0E1EF2EEE
:105CF000F5E0FF2EA8E1DA2E10E0CC24C3941B11AE
:105D0000C12CE7018985882331F02C2D4AE26D2DC5
:105D100089E70E943D641F5F412F6D2D86E0AADF59
:105D20002C2D48856D2D88E10E949011DCE3C0E0A8
:105D30000C2D2C2F412F6D2D8D2F90DECF5FDA5F34
:105D4000C430B1F78AE0E80EF11C88E0D80E1430B8
:105D5000A1F60E94761A682F660F660F660F615FC4
:105D600029E04AE180E0DF91CF911F910F91FF90F0
:105D7000EF90DF90CF90BF900C94CC671F93CF93A0
:105D8000DF93162FEC01112329F089910E94C86A34
:105D90001150F9CFDF91CF911F910895CF93C82F64
:105DA0000E94CF6A8F3F21F08C13FACF81E001C0AF
:105DB00080E0CF910895CF93C82F81E00E94C86AF8
:105DC00080E00E94C86A8C2FCF910C94C86AEAE7E1
:105DD000F8E01382128282E08093FF0884E40C943E
:105DE000C86A0F93209180083091810842E3429F56
:105DF000C001439F900D11246EEE71E00E94F87671
:105E0000062F28E044E660E38EE00E94D7670F91FA
:105E10000895AC0168E184E20C943B659F92AF92D7
:105E2000BF92CF92DF92EF92FF920F931F93CF9387
:105E3000DF93B82ECAE7D8E08C81882319F086E07A
:105E400092E102C08EEF91E10E942C25A89521E6F7
:105E5000B21659F08FEBB81217C00E94B66A1092B2
:105E6000FF0819821092F2080FC08AE50E94C86AE2
:105E7000809154060E94695F89E08093FF08109228
:105E80001E0881E60E94F069C090F2084091FF0868
:105E900050E04A30510508F084C1FA01ED59FF4F36
:105EA0000C945D778BE10E94C86A8BE10E94C86AFE
:105EB00018821B8281E09FC08B81853030F48EE395
:105EC0006DDF8B818F5F8B836CC18C81882341F068
:105ED0001D8287E08093FF0882E40E94C86A61C146
:105EE00076DF5FC127E08C2D622F0E94DF76829FD4
:105EF000202D1124298386EF91E18BDF1CE00AE03D
:105F00000E94CF6A8F3F09F44CC12091F008309174
:105F1000F1082F5F3F4F3093F1082093F008833052
:105F200009F469C08D3009F480E02A819881FE016E
:105F3000129FE00DF11D1124E90FF11D81878111E0
:105F400016C09B818981981750F081E0820F8A8367
:105F5000883028F088E50E94C86A83E04CC08EE44F
:105F60000E94C86A8B818F5F8B831882C9CF81E0C2
:105F7000890F8B3010F48883C3CF0883C1CF8A8107
:105F8000982E883010F017E0912E4981480F41502B
:105F90006B2D82EF98E00E94CC258981C81A8C2D48
:105FA000873008F09DCF7E0199E0E90EF11C00E0FA
:105FB00010E0B8E0AB2EDD24C7FCD094091598F4AE
:105FC00021E0C016D10609F020E02061A7016A2D6A
:105FD0008CE00E94006528E0A20E0F5F1F4F8CE04E
:105FE000E80EF11CEBCF90E6B912DBC082E50E940F
:105FF000C86A1D8284E08093FF08D3C08CEE91E1D3
:1060000008DF8D81811120C01F821E8282E7C6DEDB
:10601000882309F44FC08DE0CEDE8C2D90E02981DD
:10602000821B91092CE0289FF001299FF00D11247B
:106030003996EC0FFD1F8CED838783E084876DE03C
:10604000CF019CDE188264C08130A1F50E94CF6A26
:106050008F3F2FEF920771F1988121E0290F28835C
:10606000FE01E90FF11D818788818F3078F38E81E1
:106070009F810CED13E0081B190B0D30110510F07A
:106080000CE010E0A80166E878E0855B9D4F0E9477
:1060900063778E819F81800F911F9F838E838C3DBC
:1060A000934008F48AC085E08093FF0885E60E944B
:1060B000C86A188296DE75C085EE91E1AADE8885F1
:1060C0000E945D5D882309F46CC086E094CF8CED5E
:1060D00091E15CC085ED91E19CDE8D8181111AC05A
:1060E0001F821E8282E65ADE882321F388850E9461
:1060F000D65D8DE060DE6AE08BE492E03FDE8BE00F
:106100000E94C86A8CED0E94C86A83E00E94C86A37
:1061100081E02FC0813049F483E640DE882351F2CC
:1061200082E08D831F821E82C5CF8230D1F48E81A2
:106130009F818C3D934028F083E00E94C86A84E0F0
:1061400018C08CE038DE8E819F816CE0855B9D4FAE
:1061500015DE83E08D838E819F810C969F838E83D5
:10616000A9CF833041F484E619DE882309F4A2CF55
:1061700082E08D839FCF86E011DE882309F49ACFD9
:1061800088E08093FF0896CF89EC91E142DE09C058
:106190008AE704DE882329F00E94C06A80E00E941A
:1061A0003914DF91CF911F910F91FF90EF90DF9005
:1061B000CF90BF90AF909F9008958EE678CF21E06A
:1061C000411101C020E0405D0C943D640E948E109E
:1061D0002091EB083091EC08AC01421B530B9A0163
:1061E000283E334088F09093EC088093EB08809130
:1061F0005A028F70823041F485E10E943119882360
:1062000019F087E00C94AF7408950F9300E020E03C
:106210000E9466670F9108951F93CF93DF93182F05
:106220008AEA91E10E942C25163628F4143630F4BF
:10623000113659F00FC01E3841F00CC08091EA08A9
:1062400091E089278093EA0805C01092EA0880E06F
:106250000E9439148091EA08882309F43FC0C6E0FF
:10626000D1E0103641F48FEF888319821B821A82A5
:1062700087E10E94AF7464E771E188E00E942565C0
:106280004981469550E068E086E60E94566748815D
:10629000469550E060E186E60E9456674981888114
:1062A000481B469550E068E186E60E9456678A8161
:1062B0009B8129E1289FA001299F500D112456950B
:1062C00047955695479520E360E286E60E94286749
:1062D00061E671E188E30E94256529C0C5E5D8E043
:1062E0006AE471E180E00E9425654091E8075091E1
:1062F000E90768E08AE289DF4C815D8168E08EE42D
:1063000084DF4F81588560E18AE27FDF49855A85C5
:1063100084E0569547958A95E1F760E18EE475DF54
:106320004091E6075091E70760E08EE46EDFDF9171
:10633000CF911F910895CF93DF93282F30E095E000
:10634000899FE0011124C050DE4F4C818FE0829F75
:10635000F001839FF00D1124EB5AF74F988189814A
:1063600095878687442311F090E080E093878487A7
:10637000108617821582148212861186118210826D
:10638000DF91CF9108951092E9071092E80780E01D
:10639000D2CF81E0D0CF5F926F927F928F929F9207
:1063A000AF92BF92CF92DF92EF92FF920F931F9323
:1063B000CF93DF9306EE17E0F8018F0186818F5FA0
:1063C000868375E5A72E78E0B72EE4E0EE2EE2E0B6
:1063D000FE2E812C55245394E501811003C0809139
:1063E000BA0502C08091BB05882309F48FC18D32A4
:1063F0004CF08C520E9431199E81891709F486C194
:106400008E8302C00E943119882309F47FC1811054
:1064100002C0B9DF01C0BDDF66246394F701329783
:106420009080F701319770808EEF890D823028F4CB
:10643000C0904408D090450802C0C12CD12C809156
:106440005208882319F0C12C6CEFD62EF3E0F91511
:1064500048F4E92DF0E0EE0FFF1FE251F84FC08045
:10646000D18002C0992059F12CE2271504F5F801DA
:106470008481958128813981822B932B2B81822BDA
:106480002681822B2A81822B892B09F41A8284EDA2
:10649000870D0E943119882341F09A81911105C01E
:1064A00091E02B81211190E09B838A8308C07720A3
:1064B00029F0872D0E9431198B8301C05B828B816B
:1064C000882379F061100DC0FCEFDF1AD7FE03C0FE
:1064D0002FE3C20ED11C46E0D594C7944A95E1F74C
:1064E00001C0C12C888199818C0D911D998388836D
:1064F0000E948E10F801C480D5808C199D098436C5
:10650000910508F46AC0668170E0888199810E94D3
:106510000C77462F99838883F80181100DC0208164
:1065200031812F5F3F4F31832083228133812F5F61
:106530003F4F3383228307C01682F4E6CF0ED11C6F
:10654000F801D582C482442331F02F8138852F5F32
:106550003F4F38872F83611009C02B81222331F0F0
:106560002C813D812F5F3F4F3D832C83772775958D
:10657000679589859A85680F791F7A876987F701FA
:106580003497808191819C878B879920E1F0F1E09D
:106590009F1209C0711004C0F801628173810EC09E
:1065A0006C817D810BC0F2E09F1203C06F81788502
:1065B00005C024E0769567952A95E1F79C01261B96
:1065C000370B3C872B87F7012081222331F02B8565
:1065D0003C85821B930B9C878B878394FFE0AF0ED7
:1065E000B11C25E0E20EF11C32E08312F5CE05E588
:1065F00018E0F8018F01F090040280910002909160
:106600000102C385D485258536852C173D0709F4FD
:106610007FC0D687C5872381222309F479C0FF2054
:1066200021F09C012C1B3D0BE90120916D0622FFFE
:106630002DC0892B59F1CE31D10519F469E289E1D8
:106640000BC0C431D10519F46AE28AE105C0CA3031
:10665000D10529F46BE28BE10E94B9740AC0C630FF
:10666000D1052CF4D7FD05C06C2F8CE1F5CF80E06F
:1066700001C081E090916D0693FF08C0882331F03E
:1066800082E390E090933B0180933A01D7FF05C0ED
:10669000FF2019F0F801C385D4856CE370E0CE01CA
:1066A0000E940C77DC01CB0140916D0641FF1AC0BE
:1066B000AB2BC1F44091760641FF07C0009741F033
:1066C00046E260E00E94C17403C080E00E94AF74A3
:1066D00080916D0683FF06C082E390E090933B01BA
:1066E00080933A01F801838594850A960A9780F48D
:1066F0008CE10E94AF7480916D0683FF09C082E334
:1067000090E090933B0180933A0102C0612C86CEC9
:10671000DF91CF911F910F91FF90EF90DF90CF907D
:10672000BF90AF909F908F907F906F905F900895F3
:106730000F9304E12AE04BE452E0682F88E10E94C5
:10674000CA640F9108950F931F93CF93DF93D82FAF
:10675000162FC42F423049F48091990682FF12C04F
:106760008FE10E94CF6925E10AC0463059F480913B
:10677000990684FF07C085E20E94CF692BE1280FAC
:1067800000E006C081E08C0F0E943119082F2C2FE9
:1067900040E053E0612F8D2F0E94EE64DF91CF9196
:1067A0001F910F9108956F927F928F929F92AF9257
:1067B000BF92CF92DF92EF92FF920F931F93CF93EE
:1067C000DF9391E0909317089091C60190FF02C06B
:1067D00044E001C043E066EE78E00E944B21F82ED1
:1067E000409107094150682F86EE98E00E94CC2521
:1067F000E090E608D09018080091730810E00C3083
:10680000110508F0C6C6F801E359FF4F0C945D77F7
:1068100087EC96E10E942C258091C60180FF02C082
:106820006BE001C06AE06093070941E04E0D6750DC
:106830008FE191E10E941122ACC684E195E10E94B2
:106840002C2586E080930709EE2011F0C0E001C0FE
:10685000CD2D4091550650E006E111E12C2F68E066
:1068600086E70E943225CC2351F04DE26AE0809108
:1068700055060E942A14809355060E941A6865ECFA
:1068800070E180E10E94256581E0E8120CC0409132
:106890005701642F6195809158060E942A148093B5
:1068A00058062D2D01C020E04091580660E180E699
:1068B0000E94901141E092E0E91240E0809173065D
:1068C00068E186FB882780F90E948D2590917306E8
:1068D00080FB96F990937306C0916F06E3E0EE1289
:1068E00007C068E78C2F0E942D14C82F2D2D01C0E2
:1068F00020E04C2F440F440F4C0F60E286E60E94CC
:10690000C225CC2329F043E760E288E70E94C864EF
:10691000C0936F06C0917706F4E0EF1206C068E7F7
:106920008C2F0E942D14C82F01C0D12C4C2F440F46
:10693000440F4C0F2D2D68E286E60E94C225CC2321
:1069400029F043E768E288E70E94C864C0937706AD
:1069500041E085E0E81240E080916D0660E383FB52
:10696000882780F90E948D2590916D0680FB93F910
:10697000ACC489EC94E10E942C2586E08093070941
:1069800063EA70E188E00E942565C0918306C95FD3
:10699000E11008C0DD2DD06467E08C2F0E942D141B
:1069A000C82F01C0D0E44C2F50E02D2F68E086E6C0
:1069B0000E942867C750C093830621E0E21220E0BE
:1069C00040916A06469546954695477065E770E1A1
:1069D00080E10E943F258770880F880F880F909173
:1069E0006A06977C982B90936A064091760644300D
:1069F00008F044E021E092E0E91220E06FE370E16A
:106A000088E10E943F25843008F087E08093760675
:106A1000E3E0EE120AC044E661E0809174060E9451
:106A20002A148093740621E401C020E44091740686
:106A300050E060E286E60E942867F4E0EF1209C0A9
:106A400065E0809175060E942D148093750621E4FF
:106A500001C020E44091750650E00DE210E168E2CB
:106A600086E60E943225C0916D06C695C1706DEE16
:106A700076E180E30E94256541E085E0E81240E090
:106A800060E38C2F0E948D2590916D0680FB91F91B
:106A90001CC482EE94E10E942C258AE080930709B1
:106AA00095E09E1508F4C3C00E94A12860EF7FE026
:106AB00088E00E94256541E0E11040E08091870672
:106AC00068E081700E948D259091870680FB90F987
:106AD00090938706C0916D06C17041E0E41240E0DA
:106AE00060E18C2F0E948D25817090916D0680FB56
:106AF00090F990936D068C130E949B1941E0E2E09F
:106B0000EE1240E08091730668E185FB882780F9EA
:106B10000E948D259091730680FB95F990937306E2
:106B2000F3E0EF12D12CE0917006F0E0EF5BFC4F48
:106B3000D491CCE6ED2FE370F0E0EF5AF94E44919A
:106B40002D2D60E28C2F0E943D64D695D695C650BF
:106B5000C43581F7DD2039F067E1809170060E942D
:106B60002D148093700614E2C0E0D0E02C2F46EB89
:106B700055E168E2812F0E94FC632091880630E095
:106B80000C2E02C0359527950A94E2F720FF06C027
:106B900020E042E168E2812F0E9461652196185E43
:106BA000143821F794E0E9120FC08091C60180FFEC
:106BB000FFC46FE0809188060E942D1480938806A0
:106BC0008091750D86FFF4C480916B06E5E0EE12AE
:106BD00013C090911E08992389F063E00E942D1440
:106BE00090916B06891761F0909173069F7790934F
:106BF000730680936B0604C020E003C021E001C04F
:106C000022E041E3480F60E382E10E943D64D4E268
:106C1000C0E08C2F0E94811020E0482F60E38D2F70
:106C20000E94AC10CF5FD85EC43099F7B2C4F9E0CF
:106C3000FE1528F489E08093E60869E0E62E83E0FB
:106C400080930509C9E8D6E010E058E0F52E00E091
:106C5000212F46EE52E06F2D8EE10E94EE6401E09E
:106C600086E0810FE81200E024E0AE016F2D8091F4
:106C7000F5070E94D92C88E0F80E1F5F2496143087
:106C800031F787C48BEE94E10E942C2586E0809337
:106C900007096CEC7FE088E00E942565E1100BC0DD
:106CA000CD2DC06448E768E2809156060E942A1400
:106CB0008093560601C0C0E42C2F4091560668E030
:106CC00086E60E94366791E0E91209C04EE666EF5B
:106CD00080916C060E942A1480936C0601C0D12C0E
:106CE00080916C06482F552747FD5095465F5F4FB2
:106CF0002D2D60E180E70E94286721E0E2E0EE129E
:106D000020E080916A0640EC5FE068E181700E94BB
:106D1000942590916A0680FB90F990936A0621E091
:106D2000F3E0EF1220E080916A0640E959E160E269
:106D3000869581700E94942590916A0680FB91F956
:106D400090936A0621E084E0E81220E080916A06D0
:106D50004FEA5FE068E282FB882780F90E94942571
:106D600090916A0680FB92F990936A0621E095E083
:106D7000E91220E080916A0687FB882780F941EAC2
:106D80005FE060E30E94942590916A0680FB97F98A
:106D900090936A06FEC38BEF94E10E942C2586E057
:106DA00080930709E11003C089E08093050901E0A1
:106DB000E11000E02AE048E756E068E08091F5073E
:106DC0000E94D92CC0916D06C2FBCC27C0F96EED94
:106DD00076E180E10E94256541E0E41240E060E157
:106DE0008C2F0E948D2590916D0680FB92F99093D7
:106DF0006D0621E0E2E0EE1220E080916D0641E9AF
:106E00005FE068E1829581700E94942590916D0603
:106E100080FB94F990936D0621E0F3E0EF1220E0FF
:106E20008091730646E85FE060E2829581700E947F
:106E300094259091730680FB94F99093730621E05A
:106E400084E0E81220E080916D064CE75FE068E2A4
:106E500085FB882780F90E94942590916D0680FB20
:106E600095F990936D06C0917306C7FBCC27C0F9C6
:106E700060E77FE080E30E94256541E095E0E9124C
:106E800040E060E38C2F0E948D259091730680FB7B
:106E900097F9909373067DC384E095E10E942C25B9
:106EA00063E677E080E105C18BE69FE00E942C2538
:106EB00010E0C0E0C43018F0D8EFD10F01C0D12FDE
:106EC0008091990601E00C0F82FF04C0C23011F4DA
:106ED00042E005C084FF07C0C63029F446E06D2FAC
:106EE00080E331DC0EC020E0402F6D2F8AE20E944B
:106EF00090118FE08C0F0E942569482F6D2F84E43C
:106F00005ED9C02F185F0930A9F667E47FE080E101
:106F10000E942565D8E3C0E08C2F0E942569482F88
:106F20006D2F80E24CD9CF5FD850C630A9F74FE320
:106F30005FE068E184E50E943B6516E0C0E2D0E0D6
:106F40002D2F46EB55E16C2F84E50E94FC63812FC9
:106F50000E942569482F6C2F8CE631D981E0810F82
:106F60000E942569482F6C2F88E729D9DF5FC85F09
:106F70001E5FD43029F78091990686FF0CC06AE322
:106F80007FE088E00E9425658BE20E943119482F3E
:106F900068E088E714D98091990687FFFAC265E313
:106FA0007FE080E10E9425658CE20E943119482F24
:106FB00060E188E704D9EDC281E39FE00E942C25BF
:106FC00081E08093070910925601D0E0C0E019E1FA
:106FD0000D2D006241E46D2F88E10E94C86441E3F9
:106FE0004C0F6D2F8EE10E94C8648C2F0E940616F4
:106FF000AC016D2F8AE20E943D65C43028F48C2FCD
:107000000E948110815003C0C730D9F08C2FE82F27
:10701000F0E0EE0FFF1FE05CF74F20813181129FFF
:10702000F001139FF00D1124F7FF02C0E150FF4F54
:107030005F2F550F550B4F2F6D2F8AE50E94566716
:1070400005C0402F6D2F8AE50E944A67CF5FD85F49
:10705000C83009F0BFCF6DE27FE088E20E9425656D
:10706000409100015091010160E388E70E9456675A
:1070700081E080931A0880911E08882309F489C250
:107080004FE761E8809157060E942A1480935706C3
:1070900080C28CE095E10E942C2586E08093070950
:1070A0008090F5078091630081FF06C066E27FE073
:1070B00088E10E9425656DC266E17FE088E00E945C
:1070C0002565C1E6D6E0A12C10E133E0732E9924AA
:1070D00093949A0C20E0492D612F80E00E94AC101F
:1070E000B12CEA1004C0709205098B1419F020E04D
:1070F000C12C02C0CD2C22E0E2E0BE16D1F1F3E0BB
:10710000BF1609F44DC081E0B81689F04981429557
:1071100046954695437069E07FE0812F0E943F25A8
:107120008295880F880F807C99819F731FC0098189
:10713000000F000F059505959DE00902F00111244F
:10714000F7FD3396AF0155954795559547952C2DED
:10715000612F82E40E942867C1FE3AC04FE161EED0
:10716000802F0E942A148F739981907C982B998389
:107170002FC06880E62DE7706E2E20E12E0F0C2DBB
:107180004AEE58E1612F88E40E94EE64C1FE20C0FF
:1071900063E0862D0E942D1487709881987F16C019
:1071A00008810595059505952C2D402F612F8AE5C1
:1071B0000E949011C1FE0CC04FE061EF802F0E9431
:1071C0002A14880F880F880F98819770982B9883BE
:1071D000B394F4E0BF1285CF185F2296103311F0FC
:1071E000A92C75CF84E0E8120BC0CD2DC06248E217
:1071F00066EF809171060E942A148093710601C087
:10720000C0E240917106552747FD5095465F5F4F9C
:107210000EEF1EE02C2F60E38EE40E94322504E284
:1072200011E0C9E5D6E090E3D92EF80141915191E2
:107230008F0129913991421B530B440F551F20E2B6
:1072400068E38D2D0E942867F8E1DF0E80E9D812EF
:10725000ECCF95E0E91215C0E0E6FE1214C01092E2
:107260001E0888E0E4E2F1E0A9E5B6E001900D92A5
:107270008A95E1F781E00E945E5E87E10E94AF742B
:1072800002C020E001C021E04AEF5EE068E380E058
:107290000E9400657EC182EF94E10E942C2588E067
:1072A00080930709E11014C00E94A12880916D0607
:1072B00021E04FEE5EE068E086FB882780F90E94BF
:1072C000942590916D0680FB96F990936D0661C1AF
:1072D00064EA7EE088E00E942565C0E008E0C09096
:1072E0009906C23051F0C33069F040919A06C1301E
:1072F00079F442954F7010E10DC040919C064F709B
:1073000010E408C040919C0642954F7010E802C0FE
:107310004F7014E0FF24F394FC0E21E0EF1020E006
:1073200060E87EE0802F0E943F25D82F812F809536
:107330008C21D11103C08093990603C0182B1093A0
:10734000990680919906C8120E94E010C23051F04F
:10735000C33069F0C130A1F4D295D07F90919A06E4
:107360009F7012C0DF7090919C06907F05C0D295EF
:10737000D07F90919C069F709D2B90939C0607C098
:10738000DF7090919A06907F9D2B90939A06085FEC
:10739000083211F0CF2DA3CFF5E0EF1611F040E049
:1073A00001C04D2D80919D0668E281700E948D255F
:1073B00090919D0680FB90F990939D0686E0E816DB
:1073C00011F040E001C04D2D80919D0660E386954F
:1073D00081700E948D2590919D0680FB91F990937C
:1073E0009D0697E0E912D12C80919D064D2D68E312
:1073F00082FB882780F90E948D2590919D0680FB55
:1074000092F990939D06C5C085ED94E10E942C25CC
:1074100081E0809307091092E608CAE7D8E010E0FF
:10742000812F0E9406162E853F85821793070CF444
:107430009C013F872E874C8D5D8D481759070CF4B2
:10744000AC015D8F4C8F143060F02E853F85240F8A
:10745000351F37FF02C02F5F3F4F35952795398382
:1074600028831F5F22961730D9F68091A408809355
:107470001A08E0E2FE1621F0FFEBFF120EC00BC06F
:107480008F5F8093A408833041F487E10E94AF743A
:1074900081E00E945E5E1092A4088091A408813071
:1074A00089F050F0823009F072C010925601E8E87D
:1074B000F8E0C8E2D6E01FC06EE67EE088E10E94F8
:1074C000256565C0CAE7D8E0D12C18E9E12E1AE39A
:1074D000F12E08E615ECFF86EE861D8F0C8F8D2DA4
:1074E0000E94061689939993D39487E0D812F3CF1C
:1074F00060E67EE043C061917191848595859B0132
:10750000281B390B37FF03C03195219531092333EF
:1075100031053CF1DF0150974D915C9159834883CF
:107520009A01261B370BB90137FF02C0615C7F4F00
:10753000B6E075956795BA95E1F7261B370B3F873F
:107540002E87841B950B9C0197FF02C0215C3F4F47
:10755000A6E035952795AA95E1F7821B930B9D8FA1
:107560008C8F229698E0E639F90729F60E941F5D74
:1075700090935306809352066EE47EE080E10E9471
:1075800025654CE155E168E182E10E943B650E947E
:107590005C28DF91CF911F910F91FF90EF90DF90CA
:1075A000CF90BF90AF909F908F907F906F900895F5
:1075B00029E04CE567E283E20E94CC6705CBCF93DC
:1075C000DF93C82FD62F462F60E2BDD841E04D0F84
:1075D00068E28C2FB8D842E04D0F60E38C2FDF912A
:1075E000CF91B1C81F93CF93DF93EC01862F11E0A9
:1075F000683008F410E00E940021FC019E013C5F0D
:1076000037FD0DC0211588E0380784F0112319F0EB
:1076100048E050E002C044E050E0E40FF51F8081F4
:10762000992787FD9095982F882723C0832F1123B2
:1076300021F03327220F331F02C086953170482F67
:1076400050E0E40FF51F608140E052E0421B530B15
:10765000559547956403C001659F900D1124618184
:10766000359527956203A001639F500D1124840F67
:10767000951F69E170E00E940C77CB01DF91CF91FB
:107680001F910895BF92CF92DF92EF92FF920F93D6
:107690001F93CF93DF93182F7B010E94FF24C82EE6
:1076A000812F0E940E18811104C001E01E141F04D6
:1076B0000CF400E08EE0189FE0011124CB50DC4F69
:1076C00084E0C89E60011124F601E00FF11DEC0F6B
:1076D000FD1FB080812F0E940E188823A1F08B2DF2
:1076E0000E940B18682F772767FD7095C7019C5F74
:1076F00097FD0196959587950E944B2C7C01EE0C89
:10770000FF1C00E00BC08B2D0E940B18682F772701
:1077100067FD7095C7010E944B2C7C01CC0DDD1DCF
:10772000C00FD11D8A8144E660E08C590E94F51794
:107730009701A82FBB27A7FDB0950E94A57624E648
:1077400030E040E050E00E944177E901812F0E9443
:107750000E188111D450CE01DF91CF911F910F915E
:10776000FF90EF90DF90CF90BF900895DF92EF925F
:10777000FF920F931F93CF93DF93D62E20EEF22E1E
:10778000F80EC0E0DCEF0FE730E2E32ED11005C0C9
:1077900060910409CE0126DF04C0BE018091030977
:1077A00071DF97FD4F969C0195E0359527959A9549
:1077B000E1F7122F0F3709F4022F412F552747FD0C
:1077C0005095401B510907FD539557FF03C0519534
:1077D00041955109423030F46E2D611B8F2D0E946E
:1077E0008D650CC001171CF09FEF940F01C090E055
:1077F0006E2D611B691B8F2D0E94DB65112321F00B
:1078000060E28F2D0E948D65F394A096C03284E0D3
:10781000D80711F0012FBACFDF91CF911F910F91AF
:10782000FF90EF90DF900895DF92EF92FF920F9319
:107830001F93CF93DF93D82E80910409EE24E39415
:10784000883008F4E12C0E940021EC0140E460E063
:107850008CE50E94DB65F12C0CE91FEF2F2D30E049
:10786000EE2019F049E050E002C045E050E0241756
:1078700035075CF5C90145E0880F991F4A95E1F786
:10788000EE2019F064E070E002C062E070E00E9457
:107890000C77E62FDE01A20FB31F2C9130E22302FA
:1078A000C0011124B8010E940C77DF1005C0625E90
:1078B00025E045E08AE304C0615E23E043E08BE31A
:1078C0008E0F0E94CC67F394C9CF60E08CE5DF9106
:1078D000CF911F910F91FF90EF90DF9047CF5F9274
:1078E0006F927F928F929F92AF92BF92CF92DF92D0
:1078F000EF92FF920F931F93CF93DF93882EAA24CA
:10790000A39480910409883008F4A12C87E796E1BC
:107910000E942C25AA2011F049E001C045E0682D05
:107920008CEF98E00E94CC258FEB881202C0109259
:10793000FB084091040950E04F5F5F4F21E060E099
:107940008AE20E942867809104090E940021EC01CC
:10795000B090FC0860901808AA2019F0F9E07F2E7A
:1079600002C0E5E07E2E5C2E0C2F1D2F65E0E62E7A
:10797000F12C70E1972ECB2CD12C802F8519B816C5
:1079800011F020E001C0262DF80141918F0155270B
:1079900047FD5095692D88E10E942867AA20A1F033
:1079A000F9E0EF1689F0CE14DF0411F020E001C0F9
:1079B000262DFE01EE0DFF1D4081552747FD5095F8
:1079C000692D80E30E94286788E0980EEFEFEE1A99
:1079D000FE0AF8E39F12D1CFB71411F020E001C0E6
:1079E000262D46E754E168E38CE00E940065B7105D
:1079F0003AC080911E088823F1F180920B02109109
:107A0000FB0820E044E06CEF812F0E942014082F37
:107A10008093FB08811779F1AA2011F024E001C0BE
:107A200022E0122F119530E059E1F52EE12FFF27CA
:107A3000E7FDF0952E173F0794F0EC0FFD1FE20FC6
:107A4000F31F1002A0011124F49EC001F59E900DB9
:107A50001124B9010E940C7760831F5FE7CF82E099
:107A60000E945E5E08C0CB0DD11D44E66CE98881A2
:107A70000E942A1488838B2DDF91CF911F910F9143
:107A8000FF90EF90DF90CF90BF90AF909F908F903E
:107A90007F906F905F90C8CEEF92FF920F931F93ED
:107AA000CF93DF93C62FD0E0FE01EE0FFF1FE95DFD
:107AB000F94F21813281821B930B9C01BC018827E5
:107AC00077FD8095982F0AE0660F771F881F991F12
:107AD0000A95D1F7121613061CF4258D368D02C0B7
:107AE000278530892436310514F424E630E0442714
:107AF00037FD4095542F0E944177790121308CEF5A
:107B0000380744F0211584E038073CF0E12CA4E06C
:107B1000FA2E03C0E12CBCEFFB2E0E94A21088239A
:107B200079F080916B06082F017010E082E090E000
:107B3000801B910BC817D90719F4F194E194F1084F
:107B4000C701DF91CF911F910F91FF90EF900895A2
:107B50002F923F924F925F926F927F928F929F925D
:107B6000AF92BF92CF92DF92EF92FF920F931F934B
:107B7000CF93DF93CDB7DEB7A1970FB6F894DEBFF2
:107B80000FBECDBF8F879B876D8B80916B06880F53
:107B9000880F9E012F5F3F4F4901E12CF12C1D8E74
:107BA0001C8E1B8E212C682E712CA3014A525D4F16
:107BB0003A0160726E8B5D8951705D876D8962706C
:107BC000562E3E2C8E2D0E9406166E2D65DF8C01E2
:107BD00073E07E1570F054E0959587955A95E1F71E
:107BE000F701E25BF74F8083F301EE0DFF1D449038
:107BF00001C04E2CC42CD12CC601880F991F9A8726
:107C00008987FC01E05CF74F11830083C80117FDF1
:107C10000F9634E0959587953A95E1F7282F87FDE3
:107C2000219522307CF481E090E00C2C01C0880F7B
:107C30000A94EAF7211102C0982F03C09091E5073A
:107C40009823292A93E0931508F473C0AD85A111F8
:107C500058C08091570281FF54C05601AA0CBB1C2A
:107C6000F501EF59F94F5F018181807C09F449C02A
:107C700080818595859585950E943119882309F421
:107C800040C0809115028823E1F1D501EC91E770A5
:107C9000F0E0DF01AA0FBB1FAC5DBE4FEE0FFF1F70
:107CA000E75AF94F8D919C9120813181821B930B72
:107CB00097FD0196AC0155954795F5012181322F2D
:107CC000330F330F359535953403C001359F900D33
:107CD00011246FE170E00E940C77660F771F660F2A
:107CE000771F2295269526952370213009F09DC691
:107CF000060F171FF2E04F1204C07C8F6B8F21E03C
:107D00002D8F3E89332339F0F601EE0FFF1FE3522A
:107D1000F84F11830083B801842DB4DC8C01632DEE
:107D2000809104070E941513880F991FD4018D9329
:107D30009C93BE89BB2339F0F601EE0FFF1FEB5376
:107D4000F84F118300835520E1F0E3E0E315C8F01C
:107D5000F2E04F16B1F0065F1F4F0531110538F004
:107D6000F601EE0FFF1FEB53F84F11821082E1E096
:107D7000F0E0EC0FFD1F29853A85E20FF31F118219
:107D800010823FEFE31AF30A42E0840E911C57E0A1
:107D9000E516F10409F015CF80915C0280FF27C041
:107DA00062E0809104070E941513182F0E94A21010
:107DB000012F81110195202F332727FD3095432F67
:107DC000532F23583F4F4F4F5F4FA0E0B4E08091B7
:107DD000C9079091CA07A81BB90B0E94CA7620E078
:107DE00034E040E050E00E9441773E832D836E896D
:107DF000662309F435C11091600212218091E507D4
:107E00008095812319F088E10E94AF741093E507F3
:107E100005EC17E0D8018D0180E094E0FD01978723
:107E20008687918B808B40916302442309F458C06C
:107E3000A281B381E680F7809D010E94A5764B0167
:107E40005C019701D7010E94A576860E971EA81E99
:107E5000B91E842F0E9418187C019C01DC010E942D
:107E6000A576681579058A059B05D0F580E1C82EB1
:107E7000D12C40E050E8E0E0F0E89A01DA010E94FD
:107E8000AB7686169706A806B90610F44E275F272C
:107E9000F695E79521E0C21AD108C114D104E9F49E
:107EA000F801228133814A01A12CB12CD7010E9413
:107EB000A576A50194010E944177F80133832283BE
:107EC00026813781D7010E94A576A50194010E94E1
:107ED0004177F8013783268303C04E2B5F2BCDCF2C
:107EE00060916102862F807E09F4BAC051100EC0E5
:107EF000F801228133818B819C81280F391F868173
:107F000097814F815885840F951F04C080E090E0D1
:107F100020E030E040916202442379F04150E42FA8
:107F2000F0E0EE0FFF1F443118F4E00FF11F02C024
:107F3000E850F84F4081518102C040E050E062FFBC
:107F400003C031952195310963FF03C09195819557
:107F5000910964FF03C05195419551096295669559
:107F60006770633009F463C0643009F469C062303B
:107F700059F1BC0197FF02C0695F7F4FF3E075952F
:107F80006795FA95E1F7DC01A61BB70BBC0197FFDB
:107F900002C061587F4F660F672F661F770BA61BC5
:107FA000B70B97FF02C081509C4F892F990F990BF7
:107FB00085958595A81BB90B7A01E21AF30A37FF5C
:107FC0002CC02F5F3F4F29C0B90137FF02C0695F46
:107FD0007F4FF3E075956795FA95E1F7D901A61BF8
:107FE000B70BB90137FF02C061587F4F660F672F8B
:107FF000661F770BA61BB70B37FF02C021503C4F03
:10800000232F330F330B25952595A21BB30B7A0134
:10801000E81AF90A97FD01969C0135952795240FDA
:10802000351FB9016A0F7B1F2A1B3B0B12C07A0157
:10803000E21AF30A240F351FB901680F791F07C030
:108040007A01E21AF30ABA01680F791F9A01281B14
:10805000390BF801F38AE28A758B648B378B268B98
:10806000FF85FB8B2B852C8B45EA53E05A8F498F7C
:108070001E861D86B5E62B2EB2E03B2E1F8A198A7E
:108080005D8559A3B101665F7F4F788B6F87C12CE7
:10809000D12C7601D1018C9190E00197ED85FE8580
:1080A0008E179F0709F059C3EF85F88938978081AB
:1080B0000E940B188A8B7F89672F70E07A87698707
:1080C0006B5F784F5B01FB01E056FF4F908040E013
:1080D00061E00F85188907501109D8018C910E9421
:1080E0002D18F8019081992359F0EF85F889399777
:1080F00090819D50983020F490911502992399F029
:10810000882391F0F10181858F7190E00090040740
:1081100002C0959587950A94E2F781709927F1E05E
:108120008F27817001C080E02F853889295031095F
:1081300038A32F8FD9011C91811131C0F501E05670
:10814000FF4F10821D32C9F4E985FA85EE0FFF1F3B
:1081500029853A85E20FF31FEB5BF84FAFE8B2E0F9
:10816000A70196010E94C076BB2797FDBA95A92F5B
:10817000982F872F80839183A28388EF810F82308D
:1081800008F0DEC2F10187818670843009F4D8C21C
:1081900080E0193009F0BCC000E01CEFBDC081E0F8
:1081A000911080E0982E2FEF210F2C30B0F4822F09
:1081B00090E0DC01AA0FBB1FAB53B84F0D911C918F
:1081C000243008F091C0F101278126FF8DC0FC0109
:1081D000EE0FFF1FE352F84F26C02431C0F483EFA7
:1081E000810FE82FF0E0DF01AA0FBB1FAC5DBE4F8F
:1081F0000D911C91843040F4EE0FFF1FE75AF94FA8
:1082000080819181081B190B000F111F6DC0243252
:1082100080F4F1018781E22FF0E0EE0FFF1F86FF6F
:1082200005C0E253F84F008111815EC0E850F84F5D
:10823000FACF243281F5F101918592959695977048
:10824000B1F08EE0890F823128F081E1890F85310C
:1082500049F01CC08131D1F49091990692FF16C06B
:108260001FE106C09091990694FDE4C30FC014E08D
:10827000812F0E946569811135C081E0810F0E94C4
:108280006569882361F100E010E02EC00E94256935
:10829000882341F124C02C3260F4E22FF0E0EE0F8D
:1082A000FF1FE854FB4F0081F8E00F02800111240A
:1082B0001BC02C3251F4C701B60124E630E040E087
:1082C00050E00E94417789010FC040E050E060E03B
:1082D00070E082ED810F0E94B2228C0105C000E0A7
:1082E00014E002C000E01CEFF1018781982F907329
:1082F00091F082958370815021E030E002C0220F1E
:10830000331F8A95E2F7C9013989382B398B03C0AD
:1083100000E010E001C081E0E985FA85EB55F84FF7
:108320008083F101878183FD0EC0EF85F889329744
:108330008081882341F04DE763E80E94F5170E9491
:108340001818080F191FF101F681FE8FF11105C0F1
:10835000F1018581882309F421C180915C0283FFAA
:1083600003C0F4E1F88F02C024E6288F49855A85BE
:10837000440F551FDA01AB5FB84F3C91FD012181DD
:10838000E985FA85E40FF51FEB5BF84F8081918159
:10839000A281AC016A2F772767FD70952A013B0106
:1083A000BB2777FDBA95A72F962F852FB801681B9D
:1083B000790BCB01AB01465F5F4F4531510550F062
:1083C000A32EB22EA114B10439F4F101258121119B
:1083D00008C002C0A12CB12C911003C09C878B87D0
:1083E00037C0F101878186708430D9F4E081F0E0F4
:1083F000EE0FFF1FE25EF74FA081B18120E034E66F
:108400000E94BA762B013C01FA89FF2351F02F2FED
:10841000332727FD3095432F532F0E9441772901A1
:108420003A01BB2777FCBA95A72D962D852D98018B
:10843000281B390B3C872B872115310549F0F101A9
:10844000858137FF82958F70F88DF89F5001112438
:108450001A141B04B4F480913C01882331F021E00C
:10846000A21AB108A114B10449F0332777FC3A9558
:10847000272D162D052D1C861B8603C0AA24AA9421
:10848000BA2CE985FA85EE0FFF1FEB5FF84FB1823A
:10849000A0824B855C85452B09F473C04801AA2452
:1084A00097FCA094BA2C5E8D552309F466C0809188
:1084B0003C01882309F440C06A89662379F0262F9D
:1084C00027FD219530E040E050E060E070E080E280
:1084D00093E00E944177CA01B90104C060E070E0F6
:1084E00080E293E0F10126814B855C851416150628
:1084F00044F090958095709561957F4F8F4F9F4F79
:1085000022952F7030E02115310591F0A88DA29FA2
:10851000A001A39F500D11249A01442737FD4095D7
:10852000542F0E944177420E531E641E751E04C0D4
:108530004424582C692C7A2CBB2777FCBA95A72D9C
:10854000962D852DEB85FC851E161F0634F48816A6
:108550009906AA06BB0634F009C088159905AA0534
:10856000BB0524F44424582C692C7A2C332777FC3F
:108570003A95272D162D052D04C04424582C692C1E
:108580007A2CE985FA85EE0FFF1F29853A85E20FDF
:10859000F31FEB5BF84F408251826282F1018781C9
:1085A000EF85F889369787FF26C080810E940B18D7
:1085B000A82FBB27A7FDB0951A161B0644F417FF7A
:1085C00062C024E630E02A1B3B0BD90109C010979A
:1085D00009F459C0101611060CF055C0AC59BF4F24
:1085E00098010E94A57624E630E040E050E00E9429
:1085F0004177890148C060818BE1860F873340F065
:108600006058772767FD7095C8010E944B2C34C0D5
:10861000862F992787FD9095A92FB92F873091052F
:10862000F8F4FC01E758FF4F0C945D7717FF2BC05F
:1086300010C0101611066CF026C017FF24C011954B
:108640000195110920C010161106C4F002C017FDD3
:1086500018C000E010E017C0101611067CF011C021
:1086600067FF06C011950195110936E0361B632F8F
:108670006750C8010E94F23A8C0105C000E014E086
:1086800002C000E01CEFF101478140FD12C0AF8D38
:10869000B8A18C919FEF980F943058F4FE01319659
:1086A000E80FF11DE80FF11D329780819181080FCD
:1086B000191F9801EA89AE2FBB27A7FDB0950E942C
:1086C000A5764B015C0143FF15C0EF85F889329711
:1086D0008081882379F04DE763E80E94F5170E94B6
:1086E000181824E630E0DC010E94BA76860E971E48
:1086F000A81EB91EF101878186958370813039F0FB
:108700008230E1F0C80CD91CEA1CFB1C19C0C50161
:10871000B40124E630E040E050E00E944177CA0115
:10872000B901A70196010E94D07620E034E040E034
:1087300050E00E94417769017A0102C0750164012D
:10874000FAE02F0E311C2F892F5F2F8B4F85588910
:10875000465F5F4F588B4F879DCC10925208809197
:10876000B506882309F441C08F01000F111F000FC7
:10877000111FF801EB54F94F87849088A188B288C3
:10878000FE89FF2319F0812C912C5401C701B601F9
:1087900024E630E040E050E00E944177E091040799
:1087A000F0E0EE0FFF1FEB54F94FA581B6810E9458
:1087B000C076680D791D8A1D9B1DF801EB54F94F99
:1087C0006787708B818B928B2D8926FFF9C0209152
:1087D000B8063091B90640E050E00E944177A4E627
:1087E000B0E00E94C0766B017C010D851E85000FF4
:1087F000111F005E174FC701B60124E630E040E0CC
:1088000050E00E944177D8012D933C93698C7A8C7B
:10881000F3013F01838194818090FB04912C8816A1
:1088200099063CF0919481949108881699060CF46D
:108830004C01F30121818401FAE02F02000D111D8A
:108840001124D3012C91F4014AE02402E00DF11D22
:1088500011249F01285E334008511C4F033E54E011
:10886000150714F002EE14E049012E316BEF3607C4
:1088700024F42EE1822E2BEF922E302F212F801701
:10888000910714F4382F292FA32EB22EA814B9045F
:108890000CF45401C114D104E104F104A9F0F7FE71
:1088A00004C0D501A819B90903C0D801AA19BB0988
:1088B000A70196010E94CA7620EA36E841E050E01E
:1088C0000E94417769017A01C5010E94DF175C01AE
:1088D000AC0CBD1CC8010E94DF178A159B050CF467
:1088E0005C01C4010E94DF17A816B9060CF45C01F4
:1088F000F3018281882319F0B194A194B108909179
:10890000C7049F7180E1891BF9A1F81708F052C0D4
:108910000D851E85000F111F08531B4FD8018D01B7
:108920008C91982F9F7309F445C0982F907C9034B8
:1089300009F440C09038F1F1880F880F859585952E
:108940000E943119F8019081907C903C39F5882380
:1089500019F01092E7081BC09091BC0520914408C3
:108960003091450895FF06C02D5E3F4F27323105F7
:1089700020F00DC024313C4F54F4AD8DAA2309F4EE
:108980005BC02B8D3C8D24313C4F0CF455C0909135
:10899000E708911101C081E080935208882351F0CB
:1089A000ED85FE85EE0FFF1FE753FB4F80810E9490
:1089B00018185C01F894AB89BC89AD92BC9278948C
:1089C000ED85FE853196FE87ED872B893C892E5FEC
:1089D0003F4F3C8B2B8B498D5A8D4B5F5F4F5A8F8E
:1089E000498F709709F04CCB1091750D798970FF04
:1089F00005C0111103C08EE10E94AF74898981FF07
:108A000007C0812F877F803419F48FE10E94AF74F3
:108A1000998992FF15C0812F877F803811F0103916
:108A200079F480E20E94AF740BC0223009F062C971
:108A30008B0160C915E21CCC91E09093E708A7CFA9
:108A4000A1960FB6F894DEBF0FBECDBFDF91CF91D8
:108A50001F910F91FF90EF90DF90CF90BF90AF905C
:108A60009F908F907F906F905F904F903F902F904E
:108A70000895FF920F931F93CF93DF930E94761A6E
:108A8000182F8093040763E68AE798E061D861E6CF
:108A90008AE998E05DD8CAE7D8E0E7EAF3E0218107
:108AA0003281499159918E8D9F8D481B590B808140
:108AB000811103C0519541955109240F351F293E5D
:108AC00083E038073CF428318CEF38072CF428E198
:108AD0003CEF02C028EE33E032832183359628E054
:108AE000CA39D207E1F600E0023071F40F5F0430BA
:108AF000D9F786E00E945E5E81E0DF91CF911F9101
:108B00000F91FF900C94AF74602F812F0E9415136A
:108B1000EC01F12C602F8F2D0E94D512853F21E0B2
:108B200092073CF4AC014C1B5D0B602F8F2D0E9413
:108B30002913F39484E0F812EDCFD8CF8F929F924F
:108B4000AF92BF92CF92DF92EF92FF920F931F935B
:108B5000CF93DF9390916906292F2F70F22E1092F8
:108B60005601209176082111A5C09077813809F42B
:108B70008BC088F4843209F441C038F4823209F49D
:108B800062C0833209F452C095C0853209F440C0F6
:108B9000803809F18FC0843841F160F4823809F4DB
:108BA00060C0833809F086C08CE091E30E9486198A
:108BB00083E85CC08E3879F08F3B09F46DC085384E
:108BC00009F078C081E080931A0883ED93E30E9456
:108BD000861985E828C092E090937608109277086D
:108BE0000E94F06910920B0265C081E080931A0820
:108BF00083EB9AE20E94861984E815C042E0F412E1
:108C000059C08091FE088F5F833054F080E008C027
:108C100052E0F5124FC08091FE08815087FD82E03E
:108C20008093FE0847C00E94F06944C0F39483E03B
:108C30008F1508F4F12C9F299093690681EA0E9410
:108C40005E5E83E126C0FF2011F0FA9402C0E3E0EB
:108C5000FE2E9F299093690681EA0E945E5E84E160
:108C600018C08CE091E30E94861982E8DF91CF91D1
:108C70001F910F91FF90EF90DF90CF90BF90AF903A
:108C80009F908F900C94F0690E94C3310E94C9316B
:108C900087E10E94AF740EC081E00E94F06983E01A
:108CA0000E94F06982E00E94F06981E08093E90807
:108CB0001092FE0880915F020E943119C82F88230C
:108CC00029F08091E908811101C0D3DEC093E90841
:108CD00090913D0180915606981710F4C6E001C0AE
:108CE000C4E080E00E9498334C2F406860E185E248
:108CF0000E944A6746E568E186E20E94C86424E073
:108D000040E060E18FE50E94CF2320E040E068E191
:108D100083E30E94E0110E94761A882361F0482FB5
:108D200060E186E20E943A2E29E046E26FE085E2A9
:108D30000E94CC6709C000E020915D0249E351E147
:108D400060E186E20E94EE64D0E07FE1E72E8D2FA5
:108D50000E948110E82FF0E0EC5CFE4EC4916D2F74
:108D6000809104070E941513AC0197FF02C04D5F6C
:108D70005F4F5595479555954795411108C0181671
:108D8000190614F441E003C0492F440F440B443E3C
:108D90000CF444EE142F4D310CF01CE18FEF8D0FCD
:108DA00046E38230C8F464E08C2F0E94DB65D1304A
:108DB00021F080915C0280FD0CC043E06EE18FEFFA
:108DC0008C0F0E94DB6543E06EE181E08C0F0E9416
:108DD000DB656E2D611B13C06BE385EE8C0F0E946B
:108DE000D9650FEF0C0F43E06AE3802F0E94D9652D
:108DF00043E06CE3802F0E94D965C10F6BE36350A1
:108E000027E047E08DEF8C0F0E94AC67DF5FD43026
:108E100009F09DCF91E09F1508F489C006EF17E097
:108E2000E12C29E1D22E3BE1C32EF801C191D19171
:108E30008F018E2D8370F1E0FF1639F18C9D802D0E
:108E4000112423E02E1510F068E201C060E39E01BA
:108E5000D7FF02C0215E3F4F95E0359527959A9543
:108E6000E1F7AE01421B530B9A01D7FF02C0C15874
:108E7000DF4FAE01440F452F441F550B420F531FC8
:108E800020E28F5D0E9428674DC053E05E1518F008
:108E9000A2E2AA2E02C0FEE5AF2EB82EBB0CBB0C80
:108EA000B80EE6E28E2E8B0C8091610281FF03C02A
:108EB00060E075E002C060E074E0AE01D7FF04C07E
:108EC000442755274C1B5D0BD49EF001D59EF00D19
:108ED0001124CF019E5F0E940C77962E89E18617A0
:108EE00014F479E1972E25E543E3682D87EE8A0D8A
:108EF0000E949E6545E064E26B0D8A2D0E94DB6551
:108F00001C161D0614F4A39401C0A91867E26B0D8A
:108F1000492D8A2D0E94D9656B2D6B5D492D8A2DB7
:108F20000E94D965E39498E0E9127FCF27C0E2E080
:108F3000FE1218C00E945C286091FE08C1E0C60FB6
:108F4000662329F0862F880F680F660F6D5F8AE011
:108F50000E94DF3A6C2F660F6C0F660F84E60E944A
:108F6000DF3A0CC024E041E068E289E30E94CF23AD
:108F700020E840E060E38FE00E94E01180917608F5
:108F8000882399F14EE06FE184EA96E10E941E2A5F
:108F900010927508813049F590917808911103C0BD
:108FA00083EB9AE220C0913039F490931A08109222
:108FB000540884E891E517C0923061F480937508F5
:108FC000E0914A01F0E0EE0FFF1FE35BFE4F80816E
:108FD000918109C0933019F483ED93E304C0943078
:108FE00021F48CE091E30E948619DF91CF911F91CB
:108FF0000F91FF90EF90DF90CF90BF90AF909F9038
:109000008F900895AF92BF92CF92DF92EF92FF922E
:109010000F931F93CF93DF936C01162FC5EBD6E010
:109020000E94761AF82E4091E8088417E1F1442353
:1090300061F0EFEFE40F8AE0E89FF0011124E75EB2
:10904000FA4F808182958F7001C080E0FF2061F02F
:10905000EFEFEF0D9AE0E99FF0011124E75EFA4F80
:1090600090819F70891718F08823D9F001C0892F4B
:10907000682F70E080E092E00E940C777A83698329
:1090800081E090E09C01042E01C0220F0A94EAF7CF
:109090003881322B0F2C01C0880F0A94EAF7382B45
:1090A0003883F092E8081062E12E8881882329F144
:1090B0001C821B828E01B12CAA24A39488818A2150
:1090C000A1F0BF1491F0B09204078B819C81F8014C
:1090D00025813681820F931F9C838B836E2DC60161
:1090E0000E94A83DFE2DFF7DEF2EAA0CB3940E5FCB
:1090F0001F4F85E0B812E2CF09C0FE01EF0DF11D50
:10910000EF0DF11D80E094E696838583FE01EF0D5F
:10911000F11DEF0DF11D8B819C8125813681820F20
:10912000931F9C838B83F09204076E2D6064C601AD
:109130000E94A83D8881882309F43EC080913C01AB
:109140008823D1F1FE01B0E0A1E080E094E6258122
:10915000368118814A2F412331F100913C01698108
:109160007A81069FA001079F500D1124BF1559F069
:109170004217530718F4241B350B17C02A2F2095CC
:109180002123288310C0BC01621B730B46175707AD
:1091900018F4240F351F09C02A2F20952123288376
:1091A00020E034E602C020E030E036832583AA0FB9
:1091B000BF5F3296B53059F6DF91CF911F910F9175
:1091C000FF90EF90DF90CF90BF90AF9008950F93F6
:1091D0009CEF940F9D3138F450E0425051098E5E5F
:1091E0000F910C942867413208F04D51022F242F23
:1091F00041E257E10E94EE640F910895CF92DF9211
:10920000EF92FF920F931F93CF93DF93C82E82E4C8
:109210009EE00E942C254091060950E04F5F5F4F71
:1092200060E08EE40E945667C091060989E0C89FFD
:10923000E0011124CC53DA4F8C81877011F04AE0A1
:1092400001C049E06C2D85EE98E00E94CC2510917C
:10925000E50816301CF469E17EE002C064EF7DE0B1
:1092600088E00E942565F090180816300CF0ACC01C
:109270000E94A128111107C06EE288810E942D145E
:1092800088832F2D01C020E0488168E080E60E949D
:10929000AC1088818823D9F081500E9430126C0173
:1092A0006FEE7DE088E00E9425654881453250F0F0
:1092B000455202E0E02E00E0960168E088E40E945A
:1092C000DD2305C0A60168E088E40E9456671130DE
:1092D00039F466E089810E942D1489830F2D01C025
:1092E00000E02981253018F447E357E103C02550F9
:1092F0004FED5DE060E18EE40E94EE64123081F497
:1093000084E680933E0122E040E05DE760E073E8A0
:109310008D819E810E945B139E838D832F2D01C0C2
:1093200020E048818D819E81453250F04552B2E85F
:10933000EB2E022F9C0168E188E70E94DD2305C027
:10934000AC0168E188E70E942867133051F440912E
:109350005701642F61958A810E942A148A832F2DD8
:1093600001C020E04A8160E280E60E949011143042
:1093700031F461E28B810E942D148B8301C0F12CAA
:109380002F2D4B8168E280E622DF21E0153009F0C5
:1093900020E04C8146954695469543706FEB7DE005
:1093A00080E30E943F258370880F880F880F9C817F
:1093B000977E982B9C83DF91CF911F910F91FF9007
:1093C000EF90DF90CF90089521E0163009F020E073
:1093D0004C8142954695437069EA7DE088E00E94A1
:1093E0003F2583708295880F807E9C819F79982B82
:1093F0009C8321E0173009F020E04C8147FB442793
:1094000040F96DE97DE080E10E943F254C8180FBC1
:1094100047F94C83042F077021E0183009F020E051
:10942000402F67E87DE088E10E943F2587709C819E
:10943000987F982B9C83801711F018861F828C814F
:10944000877009F465C06CE77DE080E20E942565C5
:109450008C818770813009F041C0193069F422E0B5
:109460004FEF51E060E070E08F8198850E945B13C0
:1094700098878F830F2D01C000E04F8158854C3FA6
:10948000E1E05E077CF0202F41E056E160E28CE6EF
:109490000E9400654F814B5C202F60E288E70E94AC
:1094A0003D6432C0453FF1E05F073CF0445F202F50
:1094B00060E28CE60E94982427C0202F60E288E7B3
:1094C0000E942867002301F180E8C81204C08F8140
:1094D00098850E946D1410921E0816C08230A1F467
:1094E000193051F46FE08F810E942D14482F50E005
:1094F00058874F830F2D01C000E02F814EEA57E1BE
:1095000060E28AE50E94EE64AAE0DA2E08E203C077
:10951000F9E0DF2E00E265E77DE0802F0E942565FF
:109520004D2D50E0E12FFF27E7FDF095E417F507FB
:1095300081F4E0E8CE120EC089E0FE0111928A9516
:10954000E9F710921E081A3029F488E08093E508A4
:1095500001C0F12C2F2D4BE65DE0602F88E4DF91F8
:10956000CF911F910F91FF90EF90DF90CF900C94CF
:109570000065CF93C62F20E04EE1682F80E00E9467
:10958000616580910B02803831F4C093AC0D87E2A5
:1095900091E20E94861910921E08CF9108951F93A0
:1095A000CF93DF93D82F162F237021F0223021F490
:1095B000C1E803C0C0E801C0CDE2612F8D2F0E9439
:1095C000C8644C2F612F86E08D0FDF91CF911F91E2
:1095D0000C94C86490911F08282F291B181644F476
:1095E000273014F0865005C027FD03C0892F01C025
:1095F00080E080931F080895CF92DF92EF92FF9250
:109600000F931F93CF93DF93C82F8DE796E10E94AE
:109610002C2540E16C2F8AEF98E00E94CC25F09039
:10962000FA088F2DD7DFD82EC03621F0C43611F0BE
:10963000CE3269F4F7FC0BC0F09204098C2F0E9423
:10964000F06910920B028FE69CE30E94861988E075
:10965000E82E0F2D112707FD1095CD2DD0E0CC243D
:10966000C3940C171D0709F0C12C2C2D43E754E1BE
:109670006E2D80E00E940065AE014F5F5F4F88E075
:109680008D1510F486E101C081E12C2D6E2D0E9414
:10969000286788E0E80ED39480E4E812DECFF7FC78
:1096A00005C0F092040984E60E94143CDF91CF913A
:1096B0001F910F91FF90EF90DF90CF9008956F92E0
:1096C0007F928F929F92AF92BF92EF920F931F93D0
:1096D000CF93DF9348E0682F89EF98E00E94CC2574
:1096E00061E076E180E00E942565C091060941E3D2
:1096F0004C0F60E08CE00E94C864A090F9088A2DAD
:1097000069DF782E45E24C0F92E0E92E00E020E080
:1097100030E060E080E30E94DD2340911F086FE2AB
:1097200074E188E00E942A6518E0BB24A7FCB0948D
:109730008BE0C89FE0011124C257DA4F4E01E7E0E9
:109740008E0E911C23E0622E472D50E0A416B50624
:1097500019F40091180801C000E0872D90E08930CD
:10976000910508F093C080589F4FFC010C945D77E1
:10977000202F4881612F82E40E94AC10002309F45D
:1097800085C06EE288810E942D1488837FC00111FC
:109790006092050924E0A401612F8091F5070E94E1
:1097A000D92C74C049815A81202F612F8EE40E94E8
:1097B0002867002309F46AC022E040E05DE760E02A
:1097C00073E889819A810E945B139A8389835EC0C2
:1097D000402F6B81812F0E94C5288B8357C0402F5B
:1097E0006C81812F0E94C5288C8350C0002329F0F2
:1097F00067E08D810E942D148D832D8147E056E115
:10980000612F88E40E94EE6441C0002349F08E81FC
:1098100061E081700E942D149E8180FB90F99E83EF
:109820008E8180FF02C04DE201C04BE2202F612FEC
:1098300088E40E943D642AC0002361F08E818695F1
:1098400062E083700E942D148370880F9E81997F3F
:10985000982B9E834E814695437050E0202F612FB8
:1098600084E50E94286712C021E0A416B50609F01D
:1098700020E04E8143FB442740F961E274E1812FEF
:109880000E943F259E8180FB93F99E837394185F0D
:10989000103409F059CFDF91CF911F910F91EF90C4
:1098A000BF90AF909F908F907F906F900895DF92C0
:1098B000EF92FF920F931F93CF93DF93C82F85EF03
:1098C00093E10E942C2548E06C2F87EF98E00E94DE
:1098D000CC250091F708802F7DDED82FC03861F4A9
:1098E00080E80E94F06989E180931C08802F0E9423
:1098F000876B81E00E94AF744D2F58E0F52E112741
:1099000007FD1095493051F1C42FD0E0EE24E394C7
:109910000C171D0709F0E12CDD24D394D40E2E2D55
:109920004D2D6F2D82E10E94586780911C0888237D
:1099300011F020E001C02E2DFE01EE0FFF1FE658B2
:10994000FF4D459154916F2D88E10E94006588E09C
:10995000F80E80E4F81611F04D2DD4CFDF91CF91A1
:109960001F910F91FF90EF90DF9008956F927F927B
:109970008F929F92AF92BF92CF92DF92EF92FF921F
:109980000F931F93CF93DF93C82E809102090E94FB
:109990009B10EC014FE06C2D86EF98E00E94CC25E7
:1099A00083EE93E10E942C2520E0488160E08A5FED
:1099B0000E94DA10A090F6088A2D0CDED82E409175
:1099C0001F086AE473E188E00E942A6568E0F62EC9
:1099D000BB24B39474E0972EE0E88E2EAD1003C044
:1099E000E090180801C0E12C0D2D10E000311105A8
:1099F00008F097C1F801E757FF4F0C945D77198184
:109A00002E2DAE016F2D84E50E943729153231F4D9
:109A100019851295169517701B5D03C0163208F054
:109A20001A5FEE2009F47DC147E361E0812F0E94B7
:109A30002A14853268F08C3210F0865009C08552A5
:109A40008295880F807E99859F71982B998785E2F2
:109A5000898367C12E2D4A816F2D80E60E94F624EE
:109A60008A835FC12E2D48856F2D80E60E94F624E3
:109A7000888757C18F814E2D6F2D83FB882780F9F2
:109A80000E948D259F8180FB93F909C199818F8167
:109A9000953080F486FB882780F94E2D6F2D9B2D05
:109AA000981B892F0E948D259B2D981B8F8190FBE1
:109AB00086F91FC086FB112710F96BE373E18F2D28
:109AC0000E9425654E2D6F2D812F0E948D259F812F
:109AD00080FB96F9E4C08F8181704E2D6F2D9B2DF8
:109AE000981B892F0E948D259B2D981B8F8190FBA1
:109AF00080F98F8316C18F8187FD08C08C81855EB8
:109B0000863340F410E047E756E107C011E04FE22A
:109B100053E103C012E045E353E12E2D6F2D86E0A3
:109B20000E940065EE2009F4FCC062E0812F0E94D3
:109B30002D14181709F4F5C0823011F48C8201C07D
:109B40001C829F8180FB97F9AAC08F8187FF09C083
:109B500004E62CE94C816F2D88E40E94B0248C83AC
:109B6000E0C04C818BE1840F8733B8F010E8140F0C
:109B70002E2D2064412F552747FD50956F2D86E6E9
:109B80000E942867EE2031F044E66CE9812F0E94A4
:109B90002A14182F10581C83C4C02E2D6F2D8CE052
:109BA0000E94A728EE2009F4BCC047E16FEE8C812B
:109BB0000E942A148C8390E6C912B3C087303CF00F
:109BC0008750809304098FE69CE30E9486198C815C
:109BD00087FFA7C08095809304098FE69CE30E94CD
:109BE00086199FC001E0E11001C000E02E2D4B81DD
:109BF0006F2D8EE40E94E2288B8393C0E110909237
:109C000005090FE310E07724739466246A946F0CBF
:109C100099859F71972121E009F020E040E3410FF1
:109C20006F2D802F0E943D64EE20E9F08091F507B2
:109C3000811319C029E048E0662D8FEF800F0E9444
:109C4000CC6780E2C81619F09EE2C9120CC0898563
:109C5000972D98279F71807E892B898782E00E94AB
:109C60005E5E10921E08770C1F5F095F153081F64B
:109C700058C01F81129513702E2D412F6F2D8EE429
:109C80000E94C225EE2009F44CC063E0812F0E949F
:109C90002D1483708295807F9F819F7C982B9F835A
:109CA00040C021E08BE0A81220E04F814695437030
:109CB0006DE073E18F2D0E943F258370880F9F8197
:109CC000997FECCF4D814F706E2D8F2D0E94B42166
:109CD0008F709D81907F0BC04D8142954F706E2D8E
:109CE0008F2D0E94B4218295807F9D819F70982B3B
:109CF0009D8317C04E8142954F706E2D8F2D0E940F
:109D0000B4218295807F9E819F7009C04E814F70E3
:109D10006E2D8F2D0E94B4218F709E81907F982B85
:109D20009E83D39498E0F90E80E4F81257CEDF9129
:109D3000CF911F910F91FF90EF90DF90CF90BF9048
:109D4000AF909F908F907F906F9008952F923F9249
:109D50004F925F926F927F928F929F92AF92BF923B
:109D6000CF92DF92EF92FF920F931F93CF93DF93E7
:109D7000A82E81E496E10E942C258091F10788238A
:109D800001F10E942025882331F01CF0A2E6AA2EC2
:109D900002C0F3E6AF2E2091F508211103C083E63F
:109DA000A81661F030E08091F307992787FD909520
:109DB0002817390721F4E2E6AE1201C0A12CA092C7
:109DC0000B0280917608811107C04091F3076A2D3C
:109DD00085EF98E00E94CC259090F50880910B02C9
:109DE000803641F08F3B19F08E32D1F403C01092CF
:109DF000F10716C09091F107992339F01092F107FD
:109E000010921E08109254080BC090917608911180
:109E100007C00E94F06910920B027724739401C06E
:109E2000712C892DD7DB582E8091760881111092E4
:109E30000B028091F1078823E1F080910B029EE9EB
:109E4000980F9230B0F401E0823609F000E01091F2
:109E50000209812F0E949B10EC0111119CC101117C
:109E6000A4C18881823010F08150888382E00E94F2
:109E70005E5E66246394B12C812CC52CD12C882D78
:109E80000E949B10EC01B51488F06B2D70E06C19EA
:109E90007D096730710554F46F5F7F4F660F660F61
:109EA000660F20E0462D81E00E94DA10FFE1F815F0
:109EB00008F4B8C028802610B5C02A96482C7E0128
:109EC0008AE0E81AF108B51408F49FC08B2D90E0E1
:109ED0008C199D09873091050CF088C00196382EA9
:109EE000330C330C330C8091F107811112C09B109D
:109EF00010C04092020920920009772031F01092A0
:109F00007708E1E0E0937608A12C11E080917608D3
:109F1000811110E0841459F0F701278126952370F0
:109F200000E043E952E1632D83E10E94EE6420E00A
:109F3000A701632D80E30E943729212F8E0108504D
:109F40001109F8014081632D8DE20E94F624F80189
:109F50008083FE0137974081442329F020E0632D60
:109F600088E40E949011FE01369740814423B1F0AD
:109F7000F701878187FF03C020E044E60BC08BE137
:109F8000840F20E0873328F4632D80E60E94A72801
:109F900005C045E4632D80E60E943D64F70186819B
:109FA000811102C040E201C04CE4F70185818823A1
:109FB00029F04C3411F44AE201C046E5632D89E7EB
:109FC0000E94C8648091F1078823F9F0809101090B
:109FD00084111BC020E046E6632D88E10E94616584
:109FE00040920209B092F5089B2C0FC0079769F4C4
:109FF0008091F107882349F080910109841105C0FF
:10A000008091F5088F5F8093F508B3944394F0E254
:10A010004F1671F12A96FE013A978081821509F454
:10A020004ECF26C09B1022C0609200098092020988
:10A03000692D6C19660F660F660F695F29E049E1AB
:10A0400080E00E94CC67772089F00E94632981110B
:10A050000DC060E0809102090E94D3211092F107A7
:10A0600086EB9CE40E948619B92C08C0B394482C56
:10A07000639481E1681611F0842C01CFB51428F1A6
:10A080008B2D90E0851991090797FCF464E872E143
:10A0900088E30E942565292D30E08091F3079927F8
:10A0A00087FD90952817390781F420E04EE768E393
:10A0B00080E00E946165E0E6AE1619F0FEE2AF12A4
:10A0C00004C087E59CE40E94861980917608882365
:10A0D00009F44CC0A0920B024BE06FE389E695E1D6
:10A0E0000E941E2A909178088130D1F5913079F440
:10A0F0000E94632981110DC0809102098F5F8093B6
:10A10000020960E00E94D3211092F10702C0923050
:10A1100018F486EB9CE40EC0943079F48091020927
:10A120008093F20780910B020E94F06910920B025B
:10A1300087E999E20E94861911C0953011F48FEFDA
:10A14000EFCF923041F4809102098F5F8093020932
:10A1500061E00E94D32181E08093F107109276089C
:10A16000809102098093010910921E08B092F307B2
:10A17000DF91CF911F910F91FF90EF90DF90CF90E3
:10A18000BF90AF909F908F907F906F905F904F9017
:10A190003F902F900895113208F06BCE103219F4D1
:10A1A000002329F066CE002311F01F5F01C011507B
:10A1B000812F0E949B10FC0198818FEF890F8031C5
:10A1C00008F057CE2081213108F053CE291302C068
:10A1D0008BE009C0002309F448CE903108F046CE48
:10A1E0009F5F988343CE815029F0908128812193ED
:10A1F0009993F9CF1093010939CE9F92AF92BF92F4
:10A20000CF92DF92EF92FF920F931F93CF93DF9342
:10A21000D82F85E69DE00E942C2547E06D2F84EE27
:10A2200098E00E94CC25C091E4088C2FD3D9A82EA9
:10A23000DE3211F0D03659F4C8304CF4C093060920
:10A240008D2F0E94F0698EEF98E40E948619B8E085
:10A25000BB2ECC2EDD24C7FCD094C9E09C2EEA2C6A
:10A26000F12C9E9CE0019F9CD00D1124CC53DA4F21
:10A27000A7014F5F5F4F02E61DE020E06B2D81E1FB
:10A280000E94322520E048816B2D8EE10E94AC10A7
:10A2900020E04A816B2D86E30E94901120E04B81E3
:10A2A0006B2D8EE40E94E7489C819770913021F0DD
:10A2B000923039F441E401C043E26B2D82E70E9401
:10A2C000C8648C81887129F048E46B2D88E70E946E
:10A2D000C864CE14DF0431F420E048E76B2D80E041
:10A2E0000E94616588E0B80EA39480E4B812B7CFED
:10A2F000DF91CF911F910F91FF90EF90DF90CF9062
:10A30000BF90AF909F9008953F924F925F926F924F
:10A310007F928F929F92AF92BF92CF92DF92EF92F5
:10A32000FF920F931F93CF93DF9392E090931708C0
:10A3300047E063EE78E00E944B21E82E4091070948
:10A340004150682F83EE98E00E94CC2580917308DD
:10A350008630A1F038F4813071F08530C9F48EE494
:10A360009EE214C08A3069F08B3071F0883081F43D
:10A3700087E59CE40BC086EA9EE408C08CEF9AE473
:10A3800005C089E597E202C08DEF90E50E9486192D
:10A39000F090E308C09118080091730810E00F30A6
:10A3A000110510F00C94EB5CF801E756FF4F0C948C
:10A3B0005D7781EB96E10E942C258EE08093070962
:10A3C00041E04F0D67E086E49DE00E9411220C946D
:10A3D000EB5C8BEF94E10E942C252AE02F1510F006
:10A3E0000E94A12880E18093070985E08F1508F479
:10A3F000E6C0F11003C089E08093050901E0F11087
:10A4000000E02AE04BE452E068E08091F5070E940A
:10A41000D92C91E0F91210C0E0E6EE1204C0809150
:10A4200055020E94831461E3809155020E942D140D
:10A43000809355022C2F01C020E04091550250E03E
:10A440004C5F5E4F08E31DE060E188E50E94322525
:10A4500061E07DE088E10E94256511E0D0E0809117
:10A46000990682FF20C08EEF8D0F8430E0F440917A
:10A47000FA04D23051F4242F30E0359527953595E4
:10A48000279545E468E18EE40CC0D43071F4242FA4
:10A4900030E044E0359527954A95E1F749E468E1D5
:10A4A0008AE57DD802C081E001C080E090919906E4
:10A4B00094FF0CC0D63039F420910C0641E468E1D9
:10A4C00086E66DD818C0D73009F4D8E0882399F013
:10A4D0008091FA04812301E009F400E04D2F50E05F
:10A4E0004A5E574E8D2F880F8D0F880F21E068E14F
:10A4F0008E5B0E94CA64110FDF5FD83008F4AFCFC3
:10A50000F2E0FF121DC029E048E367E181E40E9408
:10A51000CC6720E6E21619F08EE2E81211C08E2D0B
:10A520000E94F0690E94AD128093FA0485E20E94B5
:10A53000CF6980930C0610921E0882E00E945E5E36
:10A5400041E093E0F91240E08091BC0560E2829521
:10A5500081700E948D259091BC0580FB94F99093A9
:10A56000BC05E4E0FE1209C0C06264E68091FB0411
:10A570000E942D148093FB0401C0C0E24091FB04B3
:10A5800050E02C2F68E288E70E94286721E0F5E080
:10A59000FF1220E04091C70442954695477065EE52
:10A5A0007CE080E30E943F258295880F807E909119
:10A5B000C7049F71982B9093C7040C94EB5C2AE01E
:10A5C0002F1508F487C065EA7CE088E00E942565C5
:10A5D00041E086E0F81240E08091610268E08695F3
:10A5E00081700E948D259091610280FB91F990937A
:10A5F000610291FF1BC0C091BC05C5FBCC27C0F90F
:10A6000021E097E0F91220E04C2F65E97CE080E141
:10A610000E943F2581709091BC0580FB95F9909335
:10A62000BC058C1791F00E949B190FC0E5EAF3E07E
:10A63000808187FD1082818118160CF41182359675
:10A6400023E0E53FF207A0F3D6CFC091BC05C6FBDF
:10A65000CC27C0F941E088E0F81240E068E18C2F97
:10A660000E948D2581709091BC0580FB96F9909396
:10A67000BC058C130E949B190E94A210882311F024
:10A6800041E801C040E860E280E60E94C86441E021
:10A6900099E0F91240E080915C0268E281700E94CA
:10A6A0008D2590915C0280FB90F990935C0241E0D3
:10A6B000EAE0FE1240E080915C0260E382958170E6
:10A6C0000E948D2590915C0280FB94F990935C022E
:10A6D0000C94EB5C60E67CE088E00E94256521E05C
:10A6E000FBE0FF1220E040915D026EE37CE088E039
:10A6F0000E943F2580935D022CE0F21204C001E02D
:10A70000C11103C001C0C0E000E02C2F40915F02E6
:10A7100060E186E60E94E22880935F0241E08DE0DE
:10A72000F81240E080915C0268E183FB882780F9A1
:10A730000E948D2590915C0280FB93F990935C02BE
:10A7400041E09EE0F91240E08091570260E2869578
:10A7500081700E948D259091570280FB91F9909312
:10A76000570286E3C82E8CE0D82EE6011FE301E0F5
:10A7700096E0B92EAC2EAC18FE0144918091600297
:10A78000802321E009F420E068E2812F0E943D64EB
:10A79000FFE0FF121DC0B09205098091F5078A11F4
:10A7A00017C029E048E067E28FEF810F0E94CC6775
:10A7B00020E2E21619F08EE2E8120AC080916002EF
:10A7C00080278093600282E00E945E5E10921E08E5
:10A7D000000F2196195F103769F60C94EB5C80E14D
:10A7E00098E10E942C258AE08093070994E09F1548
:10A7F00028F00E94A128E12C10E003C0EE24E3948D
:10A8000015E0E5E0EE9EE0011124C050DE4FD0904F
:10A8100018086CE578E088E00E94256541E34E0D5C
:10A8200068E08EE10E94C864F11202C02D2D01C0C3
:10A8300020E048815981022F68E087E40E94666722
:10A84000F11214C08CE380933E014CE364EC80E091
:10A850000E942A1448815981480F511D87FD5A953D
:10A860005983488357FF02C01982188281E0810F03
:10A87000F81207C063E18A810E942D148A8341E0A7
:10A8800001C040E0E11002C021E001C021E860E128
:10A890008CE30E94E01182E0810FF81205C0DD20F8
:10A8A00019F02D2D03E002C020E002E04B8168E1A9
:10A8B0008AE50E94E2288B8321E083E0810FF81271
:10A8C00020E04C8164E478E080E20E943F258C83A4
:10A8D0001C5FF112D12CE11003C04091BA0502C0F7
:10A8E0004091BB05DD2011F003E001C002E02D2DF9
:10A8F00068E28FE40E94E228E11003C08093BA0569
:10A9000002C08093BB05E0E0F2E0808191819093EA
:10A9100059028093580282818093560283818093EA
:10A92000C60480915702948190FB80F9809357026E
:10A93000858196819093F7048093F60487818093B4
:10A94000F80480858093F9048091BC05918590FB83
:10A9500087F98093BC050C94EB5C81E996E10E9439
:10A960002C2586E080930709C091180865EF7BE0ED
:10A9700088E00E94256521E0F11020E0409161020D
:10A980004295469547706DED7BE088E00E943F253B
:10A990008295880F807E909161029F71982B909391
:10A9A0006102F1E0FF1209C064E2809162020E943C
:10A9B0002D14809362022C2F01C020E0409162028E
:10A9C00060E186E60E94AC1022E0F21208C064E664
:10A9D000809163020E942D148093630201C0C0E045
:10A9E0002C2F4091630268E184E50E94C22541E07A
:10A9F00083E0F81240E08091610260E282FB8827E8
:10AA000080F90E94AC259091610280FB92F99093AD
:10AA1000610241E094E0F91240E08091610268E255
:10AA200083FB882780F90E94AC259091610280FB0E
:10AA300093F99093610241E0E5E0FE1240E08091DD
:10AA4000610260E3829581700E94AC259091610261
:10AA500080FB94F990936102BEC789E896E10E9459
:10AA60002C2585E08093070910925601D0910309A7
:10AA700020E0F11009C043E060E08D2F0E94201417
:10AA8000D82F8093030921E041E04D0F68E080E07A
:10AA90000E94AC108D2F0E94FF24182F00E0282F59
:10AAA00042EC5BE068E08AE20E94EE6461EA7BE0EF
:10AAB00088E00E942565ED2FF0E0EE0FFF1FE05CBF
:10AAC000F74F40815181453651052CF44C395F4F89
:10AAD00024F0C2E003C0C0E001C0C1E08D2F0E949D
:10AAE0000E18811106C0CC2329F081E0F81202C0B3
:10AAF00002C0C0E080E0EE24E39400E0212F48E1B2
:10AB000068E10E94782CC13011F081E0F81280E0F9
:10AB1000E12C00E0212F48E160E30E94782CCC2357
:10AB200019F081E022E0F21280E0EE24E39401E0EB
:10AB3000212F48E268E10E94782CC13019F081E0B1
:10AB400092E0F91280E0E12C01E0212F48E260E37D
:10AB50000E94782C81E0E3E0FE1280E0E12C00E02E
:10AB600023E640E36EE10E94782C81E0F4E0FF12DE
:10AB700080E0E12C00E022E648E36EE10E94782CC0
:10AB8000809103090E940E18882311F08CE301C004
:10AB90008CE540E460E00E94DB6581E08093610920
:10ABA00061E08CE50E94B63B80910309E82FF0E05C
:10ABB000EE0FFF1FE05CF74FC081D181BE010E9404
:10ABC000423B8C0189E18C9F90018D9F300D1124B7
:10ABD00037FF02C021503F4F532F550F550B432FC6
:10ABE00060E382E70E94566789E1809F9001819F20
:10ABF000300D112437FF02C021503F4F532F550F06
:10AC0000550B432F68E084E50E945667CE014096BD
:10AC100097FF02C0CE018F967C01C5E0F594E794C2
:10AC2000CA95E1F7E8016096D7FF02C0E801AF9648
:10AC3000B5E0D595C795BA95E1F7D195C195D109FC
:10AC40006C2F635E47E08CE58E0D0E94DB656C2FF8
:10AC5000605E47E089E58E0D0E94D965109261091A
:10AC6000BAC6E0905A022E2D2F70E22ED22E81E02D
:10AC7000281751F092E0291729F0E5E02E1721F06E
:10AC8000C4E003C0C3E001C0C7E086E596E10E94CE
:10AC90002C25C0930709D0911808C091F50762E9E7
:10ACA0007BE088E00E942565F11013C080915C0272
:10ACB00067E08295869587700E942D148295880F93
:10ACC000807E90915C029F71982B90935C0221E0B2
:10ACD00001C020E040915C024295469547704F5C70
:10ACE00068E082E70E943D64EE2049F08DE08E0D21
:10ACF0008F70CC24C394823020F0C12C02C0CC24AD
:10AD0000C394F1E0FF1202C0CC2311F000E001C0B7
:10AD10000D2F2E2D46E65BE060E184E20E94EE649A
:10AD2000CC2079F162E67BE080E10E94256521E09C
:10AD3000F21202C0C13011F000E001C00D2F2091CD
:10AD40005B022E5F44E45BE060E188E40E94EE6415
:10AD500081E0F81202C0C23011F020E001C02D2FB6
:10AD600040915E0292E34902A0011124445D5E4FCE
:10AD700060E180E70E942867E1E0FE126AC082E09D
:10AD80001AC040915B02F5E0EF1201C04F7021E064
:10AD9000F21202C0C13011F020E001C02D2F552762
:10ADA00047FD50950DE31BE060E18EE70E943225E0
:10ADB00081E0F81287C08093050980911D088823DF
:10ADC00009F454C0C13051F018F0C23029F12EC03E
:10ADD00066E08E2D0E942D14D82E28C0CC2019F0AC
:10ADE00044E06EEF12C095E0E9120DC080915B0265
:10ADF0006FE08F700E942D1490915B02907F980FEE
:10AE000090935B0213C04CE760E080915B020E946C
:10AE10002A1480935B020AC0CC2041F04AE06CEF18
:10AE200080915E020E942A1480935E0280915A02F1
:10AE3000982F9F70807F2D2D2F70822B80935A0228
:10AE40009D1110925B02809157028B7F8093570275
:10AE50000DC0E2E0FE120CC044E16CEE8091640291
:10AE60000E942A148093640221E203C0CC2051F195
:10AE700020E240916402F5E04F02A00111244F51FD
:10AE80005F4F0DE21BE068E18CE40E94322563E233
:10AE90007BE080E20E94256521E083E0F81220E05B
:10AEA00040916102417069E17BE080E20E943F25B0
:10AEB0009091610280FB90F990936102A4E0EA2EE8
:10AEC00018E203C0F2E0EF2E18E195E0D9121EC19E
:10AED0006DEE7AE0812F0E942565C0903C05EC2D37
:10AEE000EF73DE2EFE1007C06EE38E2F0E942D142E
:10AEF000D82E0D2F01C000E0FBE1FD1540F02D2DF7
:10AF000043E45AE0612F8CE30E94EE6409C04D2DAA
:10AF100050E04F5F5F4F202F612F8EE70E94286720
:10AF200090913C05907C9D0D90933C05D0905B02E8
:10AF3000492F552747FD50952C2D30E042175307D8
:10AF400049F44D2D50E0E4E055954795EA95E1F739
:10AF5000477001C040E088E0810F31E03E0D9F73F3
:10AF6000D9F09E30E1F09330E9F09530F1F0973070
:10AF7000F9F0983001F1993009F19B3011F19C30D2
:10AF800019F1903121F1913129F1993131F19B3150
:10AF900039F563EF78E026C067E27AE023C069E123
:10AFA0007AE020C06BE07AE01DC06BEE79E01AC059
:10AFB00064EC79E017C064EB79E014C062EA79E0F0
:10AFC00011C066E679E00EC063E579E00BC067E486
:10AFD00079E008C06AE279E005C064E179E002C086
:10AFE0006BEE78E021E0F31220E00E943F259D2DDA
:10AFF0009F7820E1829F900D112490935B0260E185
:10B00000B62EB10E72E0C72ECE0CAD2CAA1CAA240F
:10B01000AA1CFC1002C0CC2311F000E001C00D2FCF
:10B020002A2D41EE58E06B2D84E20E94EE64FC1064
:10B0300002C0C13011F020E001C02D2F40913D052C
:10B04000552747FD50956B2D8EE70E94286769EDC7
:10B0500078E08B2D0E942565FC1022C081E0809352
:10B060000509C1110FC080911D088823C9F061E056
:10B070008A2D0E942D149D2D9F77811190689093A9
:10B080005B020EC0C13061F480911D08882341F03D
:10B090004FE761E880913D050E942A1480933D05A9
:10B0A00048E1B42EB10E53E0A52EAE0CD0903C0575
:10B0B000D6FACC24C0F8FA1002C0C13011F000E07A
:10B0C00001C00D2F2C2D45ED58E06B2D88E70E9417
:10B0D000EE64FA107BC081E080930509C11103C0C2
:10B0E00061E08B2D71C0C13009F070C080911D08E6
:10B0F000882309F46BC061E08C2D0E942D149D2DD6
:10B100009F7B8111906490933C0560C082E0D812CF
:10B1100012C06DEC78E0812F0E94256521E0FE10C1
:10B1200020E040913C056EEA78E0812F0E943F25A7
:10B1300080933C0550C491E0D9124DC46DE878E08D
:10B14000812F0E94256521E0FE1020E040913C0502
:10B150006EE874E1812F0E943F2580933C0521E039
:10B1600081E08E0DF81220E04091570242FB442707
:10B1700040F965E878E088E0810F0E943F259091D2
:10B18000570280FB92F99093570221E082E08E0DE6
:10B19000F81220E040915A02429543706AE974E146
:10B1A00080E1810F0E943F2583708295807F90917E
:10B1B0005A029F7C982B90935A0283E08E0DF812CE
:10B1C00005C061E088E1810F0E94B94A84E08E0DDC
:10B1D000F81201C460E280E2810F0E94B94AFBC309
:10B1E00086E398E00E942C258CE08093070983E099
:10B1F00080930509B090F5078F2D0E94EA4A982E9A
:10B2000038E0D32EF91003C08090180801C0812CBB
:10B210004CE46D2D80E00E94C864E8E0E91510F46C
:10B2200048E301C041E3490D6D2D85E00E94C864EB
:10B23000F1E0BF1629F022E0B21629F0712C01C00E
:10B24000782CA12C02C0A82C712C492D50E0EA01C9
:10B25000CC0FDD1FC40FD51FCF55DB4FBB2011F026
:10B2600000E001C0082D2A812F7047E357E16D2DC2
:10B270008DE00E94EE648A818F700E949510C82E26
:10B2800081111CC0188115327CF015526981812F03
:10B290000E942E239C0192E8E92E0A2D412F6D2D4C
:10B2A00084E60E94DD2323C04981552747FD509540
:10B2B0002A2D6D2D83E60E94286719C081E0C812EF
:10B2C0000DC0272D48816D2D86E30E9490112A2DF7
:10B2D00049816D2D8DE40E94901134C092E0C91215
:10B2E0000DC02A2D49816D2D80E50E94AC10272DBF
:10B2F00048816D2D86E30E94AC1024C0488147FF31
:10B3000004C04095E72DE0627E2E552747FD5095FD
:10B310004F5F5F4F02E318E0272D6D2D89E40E94F7
:10B320003225498147FF04C04095FA2DF062AF2EC7
:10B33000552747FD50954F5F5F4F2A2D6D2D8BE6AA
:10B340000E9428674A8142954F7049300CF04F5F48
:10B3500023E0B21611F020E001C0282D6D2D88E603
:10B360000E94901180911D08882309F462C08820F2
:10B3700009F45FC081E0B81631F1B81698F092E098
:10B38000B916D9F1E3E0BE1254C08A816FE082950C
:10B390008F700E942D148295807F9A819F70982BC8
:10B3A0009A8347C08A816EE08F700E942D148F703F
:10B3B0009A81907F982B9A830E949510C816C9F1A4
:10B3C0001882198236C0F1E0CF1659F0CF1690F0EE
:10B3D00022E0C21679F083E0C8122BC043E66EEC7F
:10B3E00004C040915701642F619588810E942A14FE
:10B3F00088831FC04EE260E0F8CF91E0C91671F07B
:10B40000C91648F0E2E0CE1671F0F3E0CF1211C099
:10B4100043E66EEC0AC04DE763E807C04091570170
:10B42000642F619502C04EE260E089810E942A1477
:10B430008983939428E0D20E80E4D812E3CECBC265
:10B440008CE996E10E942C2581E18093070983E035
:10B4500080930509A090F5078F2D0E94EA4A982E47
:10B460009FE09F15A0F0EF2DF0E0EE0FFF1FEA50D8
:10B47000F84F4081518157FF02C04F5F5F4F559594
:10B48000479544525A4F60E08EE40E94566780917F
:10B490000B02803819F5EFE0EF1540F14F2D50E029
:10B4A000FA01E919F109EE0FFF1FEA50F84F208168
:10B4B0003181A11013C085E0849FF001859FF00DBC
:10B4C0001124EB55FC4F8281882319F03195219589
:10B4D00031093483238382E0F1D3ECD4B8E0EB2E3E
:10B4E000C5E05C2EDAE0CD2ED12C8EC0F0E1FF124B
:10B4F000F5CF89E180931C0880E80E94F0690E94E2
:10B500003945ECCFE92DF0E05E9EE0015F9ED00D65
:10B510001124CB55DC4FEE0FFF1FEA50F84F80810E
:10B5200091814A812B813C81442319F031952195E9
:10B530003109821B930B833391050CF069C08E3C5B
:10B540009F4F0CF468C01DE266246394690C20E0F0
:10B55000462D6E2D80E00E94DA10412F6E2D8BE477
:10B560000E94C8648091610281FF59C0EDE77E2E80
:10B57000B12C472C419433243A943E0CF91052C01C
:10B58000AB1050C02091180880911D08882309F441
:10B590004BC0222309F448C010925601822E80919C
:10B5A000FB04882309F44EC00B811C810115110591
:10B5B00009F03CC0C801B6010E940C77F1E0BF164B
:10B5C00009F449C0BF1608F042C020624B815C817B
:10B5D0006E2D8DE20E942867882059F022E048EE07
:10B5E00053E068E17CEF8B819C810E945B139C831C
:10B5F0008B83B394E4E0BE12C1CF88E08E0D80341B
:10B6000009F482C0E82E962C20E192127BCF6EC006
:10B61000411103C0F2C14111F0C11FE795CF74E69B
:10B62000772EA6CF20E0B0CF812CB9CF90E0801745
:10B6300091075CF0919581959109081719070CF015
:10B64000B9CF03C000E010E0B5CF8C01B3CF82E0EA
:10B65000B816E9F040C018811456AB01410F511DD6
:10B6600017FD5A9543389FEF590714F443E85FEFED
:10B670006E2D88E40E942867882009F4BACF49E13A
:10B68000642D812F0E942A148C598883B2CF89811E
:10B690008C59AB01480F511D87FD5A954E37510506
:10B6A00014F04DE750E06E2D86E60E942867012BCE
:10B6B00031F029E048E3632D82E30E94CC678820C3
:10B6C00009F497CF8981472D67EE8C590E942A147F
:10B6D000845689838ECF422F6E2D8A810E94AC259D
:10B6E00091E0811101C090E09A8383CF21E080E155
:10B6F000F81220E080911C08811181C140E258E0DD
:10B700006E2D82E10E94006566C180E198E00E9492
:10B710002C2589E180930709C090F5078F2D0E94A1
:10B72000EA4AD82E58E0E52E60E1B62E8091C70493
:10B73000D11021C0F11010C010920509C091180855
:10B7400060E18F710E942D148F719091C704907EDB
:10B75000982B9093C70401C0C0E04091C7044F717B
:10B7600050E0485F5F4F01E018E02C2F6E2D8CE613
:10B770000E9432252AC18F719B2C981ACD2DD0E0C2
:10B78000FD1003C082E080930509C131D1052CF47E
:10B79000CC0FDD1FCA53DB4F04C0CC0FDD1FC65DCD
:10B7A000DA4F10E0FD1009C0C11207C0009118085F
:10B7B000002321F022E0A22E02C000E0A12C9D1463
:10B7C00008F49EC0111118C020E04D2D6E2D80E0B0
:10B7D0000E94DA10488142954695469543702A2D7D
:10B7E00069EF77E08E2D0E943F258295880F880FA4
:10B7F000807C98819F7331C08881113089F5809059
:10B800005701982F907C903811F499E1892E482F98
:10B81000440F440F4595459547314CF029EE240FD0
:10B8200042EE57E06E2D85E40E94EE6405C0202FA5
:10B830006E2D85E40E949011AA2009F4C2C0609187
:10B84000570161958881880F880F482D85958595CA
:10B850000E942A148F739881907C982B9883B1C092
:10B86000982F907C4981903491F447FD03C04F306C
:10B8700024F401C040E0242F01C02FE029834EEAC8
:10B8800057E16E2D88E70E94EE644FE015C09038B6
:10B8900031F5880F880F89358CF047FD04C0493099
:10B8A0001CF049E001C040E049834F5F202F6E2D1E
:10B8B00080E60E947B2249E060E01BC04F360CF01E
:10B8C0004FE64983552747FD509540585F4F202F3D
:10B8D0006E2D88E70E9428674FE660E80AC055276A
:10B8E00047FD5095202F6E2D88E70E9428674DE771
:10B8F00063E8AA2009F465C089810E942A1460C007
:10B90000111122C06FED77E08E2D0E94256520E099
:10B910004D2D6E2D86E10E945867AA2069F0409156
:10B9200057014150888160E08F710E942A148F7105
:10B930009881907E982B988348814F71202F6E2D8F
:10B940008EE10E9490113DC08881113081F4482F12
:10B950004295469547702A2D61EB77E08E2D0E9427
:10B960003F258295880F807E98819F7176CF829542
:10B970008695877090E04981069764F0493008F019
:10B9800049E049834F5F202F6E2D80E60E947B2285
:10B9900069E010C04B3F38F450E0202F6E2D86E652
:10B9A0000E94286706C0485F202F6E2D84E50E9404
:10B9B00098246FEFAA2029F0898190E00E94321428
:10B9C00089831F5F133009F0EDCED394F8E0EF0EBA
:10B9D00020E4E212ABCEDF91CF911F910F91FF9047
:10B9E000EF90DF90CF90BF90AF909F908F907F901F
:10B9F0006F905F904F903F9008951EE7A5CD20E097
:10BA00007DCE1F93CF93DF93EC011AE088810E94D3
:10BA1000BF2C0E94CF2C89931150C1F7DF91CF9199
:10BA20001F9108959C01265F3F4FFB014491DC016B
:10BA30004D93CD013196A217B307C1F70895E8E2FF
:10BA4000F6E080E090E021913191820F931F26E093
:10BA5000E034F207C1F7089587E7E7E2F6E0DF0197
:10BA60001D928A95E9F78BE08093270689E1809300
:10BA700055068AE58093560681E080936B0686E141
:10BA800080935806E8E2F6E020E032E080E093E0C0
:10BA90002193319395878487938F828FB6E0E63325
:10BAA000FB07B1F769E07AE188E796E0BBDFC7DF23
:10BAB00090935306809352060895EF920F931F932D
:10BAC00061E0680F88ECE82E0CED13E02BE432E027
:10BAD00042E082E199E002D621E08C3D934009F0FA
:10BAE00020E0822F1F910F91EF900895CF93C82FE0
:10BAF0002CED33E0EBE4F2E0DF01C9011D92019788
:10BB0000E9F76EEF79E1CF018DDF8C2F90E06AE0ED
:10BB100070E001960E940C77605D60935002805D3A
:10BB20008093510284E080933B0582E080935D0224
:10BB300080E00E94876BEDE6F6E080818062808382
:10BB40008C2FCF91BACF0F931F93CF93DF93EB013D
:10BB5000042F803120F561E0680F82E199E00FD475
:10BB600010E0A80160E270E0CE010E947D774AE01B
:10BB700050E0BE0182E199E085D40A9781F482E128
:10BB800099E0EFD3C00FD11F009749F06AE070E051
:10BB90000E940C77805D8A93862F972FF5CFDF91D7
:10BBA000CF911F910F9108958F5F93C361E0680F4C
:10BBB00082E199E0E4D38CED93E0EBE4F2E0DF0185
:10BBC0009C011D9221503040E1F74CED53E0BF0144
:10BBD00082E199E057C4FF920F931F93CF93DF93B5
:10BBE000CDB7DEB768970FB6F894DEBF0FBECDBFF6
:10BBF00001E0080F102F1031B0F4FF24F394F10E80
:10BC00008F2D67D381110DC0602F82E199E0B7D3EA
:10BC100061E0610F28E532E042E0CE0140960ED5AA
:10BC200006C01F2DE8CF103179F780E017C04FE034
:10BC300050E0BE016F5F7F4F82E199E0BDD3882362
:10BC400049F0482FBE016F5F7F4FCE0140967DD4F3
:10BC5000A895EDCFCE01409617D581E068960FB636
:10BC6000F894DEBF0FBECDBFDF91CF911F910F9132
:10BC7000FF900895EF920F931F9361E081EC99E19B
:10BC80000E9451198FEA99E10E949F12E6D298EC26
:10BC9000E92E07E710E027E236E041E060E082E1CC
:10BCA00099E01CD58737910521F081EA99E10E943E
:10BCB000841980E01F910F91EF9018CFCF93C82F78
:10BCC0008770A1F090911D09982B90931D090E94F7
:10BCD0008E1090931C0980931B098C2F90E024E018
:10BCE000959587952A95E1F780931E09CF91089540
:10BCF000CF93DF93D4D2811102C080E02EC04DD209
:10BD000087FDFBCF60E082E199E039D387E7E7E286
:10BD1000F6E0DF011D928A95E9F747E750E0BF01A1
:10BD200082E199E0AFD388E796E06BDE8091270649
:10BD30008B3040F481E08093C7018BE0809327062D
:10BD400081E0BCDFC0915206D091530678DE21E03D
:10BD5000C817D90709F020E0822FDF91CF9108950D
:10BD6000EF920F931F93CF93DF9310926009C091CE
:10BD70001D09CC2309F498C090911E099F5C9093F3
:10BD8000600981111CC00E948E1020911B09309106
:10BD90001C09821B930B883C910508F485C0809197
:10BDA0001E09882361F0815080931E09882339F091
:10BDB0000E948E1090931C0980931B0975C01092ED
:10BDC0001E098091080981116FC0DC2FD470C2FD5B
:10BDD00002C081E001C083E080930809C0FF2CC04D
:10BDE00082E38093600980911D098E7F80931D09F5
:10BDF00044E1E42E07E710E027E236E041E061E1AC
:10BE000089E099E06BD48737910519F461E180E00E
:10BE10002FC080910F09823051F480911D098160FB
:10BE200030C080910F09823029F1D1113BC084E1EB
:10BE30009AE10E94841936C0C1FF34C083E3809325
:10BE4000600980911D09897F80931D0934E1E32EEB
:10BE50000CED13E02BE432E042E061E189E099E08F
:10BE60003DD48C3D9340E9F68091540661E18F5FAB
:10BE70003ED218C080911D09D11102C0826001C05C
:10BE8000866080931D090E948E10885C91099093B2
:10BE90001C0980931B098091AE0D833019F4A8957D
:10BEA0001092AE0D10920809DF91CF911F910F9162
:10BEB000EF90089580911D09882351F081E050DFB3
:10BEC0008091AE0D8330B1F7A8951092AE0DF2CFF0
:10BED0000895EF92FF920F931F93CF93DF93C82F94
:10BEE000803108F0BFC062DE8F3F910509F010F489
:10BEF0008C2FFCDD8BE492E084DD8091F3048111D2
:10BF000007C080915C02869583708E5F8093F304F6
:10BF100080915A02982F92959695969593709330AA
:10BF200029F090933C05806C80935A0280913B05E8
:10BF3000823008F062C010E0812F0E949B10EC015B
:10BF400089818150843018F40E94811089831F5F99
:10BF5000103291F7C1EAD4E000E010E08A818F70DE
:10BF60000E949510882389F08230C1F4C8018E5553
:10BF70009B4F7C01FC018081882339F085302CF4B3
:10BF800081500E948110F70180838881882331F0DD
:10BF9000853024F481500E948110888323960D5FA0
:10BFA0001F4F04321105D1F688E3E5EFF3E0AAE76D
:10BFB000B8E001900D928A95E1F7CAE7D8E010E069
:10BFC0000EE0812F0E9481108150089FD001112422
:10BFD000AB50BC4FFE01802F01900D928A95E1F786
:10BFE0001F5F2E96143069F789EE99E10E9484193B
:10BFF00082E080933B0562DE5DDF80913B0583300C
:10C00000F8F480E090E0FC01EF55FB4F2281322FE5
:10C010003F703C3019F4207F2A6022832281322F26
:10C020003F703D3019F4207F2B60228303968432C9
:10C03000910549F783E080933B0582E03FDE3ADFDC
:10C0400080913B05843070F4809182068093FA04DD
:10C0500086ED99E10E94841984E080933B0582E09B
:10C060002DDE28DFE0E0F2E08091560282838091AD
:10C07000C6048383809158029091590291838083F2
:10C0800080915702817084838091F8048783809126
:10C09000F90480878091F6049091F7049683858354
:10C0A0008091BC0587FB882780F981870E94C33176
:10C0B0000E94C931DF91CF911F910F91FF90EF90B6
:10C0C000089540E450E060E070E08FE199E00C9466
:10C0D000816841E050E062E070E081E299E00C9418
:10C0E0008168CF93DF931F92CDB7DEB7698390E16C
:10C0F000899FB001112441E050E0CE0101960E94D9
:10C1000081680F90DF91CF910895CF93DF931F92B5
:10C11000CDB7DEB790E1899FB001112441E050E036
:10C12000CE0101960E94847789810F90DF91CF9193
:10C130000895CF93DF93D82FC82F8C2FE6DF882365
:10C1400021F08C2FE2DFC82FF8CF609121098C2FCE
:10C15000C8DFD0932109DF91CF91BBCFCF93C0919E
:10C160002109CC2341F08C2FD0DF80932109B1DF4E
:10C1700060E08C2FB6DF8C2FCF910895CF93DF93A3
:10C1800080912109C0E0D0E0882319F02F96BDDF0F
:10C19000FBCFCE01DF91CF910895DF92EF92FF9216
:10C1A0000F931F93CF93DF9380E8EBE4F2E0DF017E
:10C1B0001D928A95E9F7C3E2D9E0F12CB4E1FB12B4
:10C1C00005C08091210901E219E002C08E01888139
:10C1D00090E0E12CDD24D394DF0C0097E9F09C0182
:10C1E000245031092C37310530F4FC01E55BFD4F5B
:10C1F0002081222361F0EE2021F060E08E2D71DF9E
:10C2000003C0F80110825DDF80E090E0E6CFD082CD
:10C21000E82E7BDF90E0E1CFF3942396F5E1FF1267
:10C22000CDCFC4E0D0E0FE01E55BFD4F8081811100
:10C2300007C0609121098C2F54DFC093210949DF89
:10C240002196C038D10579F780E0DF91CF911F9119
:10C250000F91FF90EF90DF900895CF9380E4EFE18E
:10C26000F9E0DF01982F1D929A95E9F794E09093F9
:10C270001F098093200980E18093220984E0C1E0B6
:10C28000C80F6C2F2EDFCF3711F08C2FF8CF60E066
:10C290008FE727DF84E080932109CF9112CF40E41C
:10C2A00050E060E070E08FE199E00E948477809137
:10C2B0002009811103C080E48093200980911F0927
:10C2C000843029F481E090912009903409F080E0D5
:10C2D000089590E0FC01EE0FFF1FE80FF91FE15EEB
:10C2E000F64F81E09481911101C080E00895CF93D1
:10C2F000DF9390E0EC01CC0FDD1FC80FD91FC15EAA
:10C30000D64F8C819D81AE8170E0FB01EE0FFF1F47
:10C31000E60FF71FE15EF64F2481358146812C83BD
:10C320003D834E8384839583A683DF91CF91C9CECD
:10C33000CF9390E09C01220F331F280F391FF90182
:10C34000E15EF64FC481F901ED5DF64F1082118276
:10C350001282B7DECC2319F08C2FCF91EACECF9189
:10C360000895FC01808190E0FC01EE0FFF1FE80FB3
:10C37000F91FEC5DF64F918180819F700895CF93F6
:10C38000DF93FC0160831282118270E0CB01880F81
:10C39000991F860F971FEC01C15ED64F2C81238316
:10C3A000148215821682FC01EB5DF64F8081829526
:10C3B0008F70DF91CF910895AF92BF92CF92DF92AD
:10C3C000EF92FF920F931F93CF93DF931F92CDB7FE
:10C3D000DEB78C01FC01808190E0FC01EE0FFF1FB5
:10C3E000E80FF91FEC5DF64F80812181922F9F703D
:10C3F000F80121813281821B930B7A018417950702
:10C4000008F47C015B016701C114D10421F1F8013A
:10C410008381882301F164816F5F648370E0F0E1C0
:10C420008F9F600D711D112441E050E0CE010196F7
:10C430000E9484778981F50181935F01F8018481ED
:10C440008F3028F01482838160DEF8018383F1E06D
:10C45000CF1AD108D9CFF801818192818E0D9F1D0D
:10C460008C199D09928381838E2D8C190F90DF91F9
:10C47000CF911F910F91FF90EF90DF90CF90BF90E1
:10C48000AF9008957F928F929F92AF92BF92CF927A
:10C49000DF92EF92FF920F931F93CF93DF934C01A4
:10C4A0006B018A01C0E0D0E05C0125E0A20EB11C66
:10C4B000C017D107D8F5F40185818F7781F0F40199
:10C4C0004581F42FFF777F2E2F2F30E0C8018C1B82
:10C4D0009D0B8217930758F4702E7C1A08C041E018
:10C4E00050E0B501C40168DF813049F31FC0E72C7B
:10C4F000F12CC6018C0F9D1F47FF06C0A70160E00D
:10C5000070E00E947D770BC0A701BC01C40154DF1D
:10C51000871529F0FE01E80FF11DCF0108C0CE0DEF
:10C52000DF1DF401858187198583C2CFCE01DF919C
:10C53000CF911F910F91FF90EF90DF90CF90BF9020
:10C54000AF909F908F907F900895AF92BF92CF92BF
:10C55000DF92EF92FF920F931F93CF93DF93EC0143
:10C560008B01D42E8B81811110C089819A81892BF6
:10C5700061F4E880F12CF2DD8B83F701EE0FFF1FF1
:10C58000EE0DFF1DE15EF64F8483CD2C8FE0A82ECB
:10C59000CC2009F43CC0EF80F8840E948E10E81A89
:10C5A000F90AF7FE02C082E004C08B81811103C04A
:10C5B00081E08E832CC09C819F3058F01C82A5DDC9
:10C5C000811104C0CBDD682F8B818BDD8B819DDDDC
:10C5D0008B838B81882361F36C819A2D961BBC2CF5
:10C5E0009C1508F4B92EEB2CF12C70E090E1899F9A
:10C5F000600D711D11246F5F7F4FA701C80181D5A8
:10C600000E0D1F1D8C818B0D8C83CB18C1CF6D2D12
:10C6100070E06C19710929813A81260F371F3A831E
:10C6200029838D2D8C19DF91CF911F910F91FF9050
:10C63000EF90DF90CF90BF90AF900895EF92FF9270
:10C640000F931F93CF93DF93EC01F62EE42E890115
:10C6500096DE6F2D70E0FB01EE0FFF1FE60FF71F58
:10C66000EC5DF64F1082E29430EFE322E1820E940B
:10C670008E10800F911F98878F83DF91CF911F912C
:10C680000F91FF90EF9008951F93CF93DF93EC01EC
:10C69000888190E0FC01EE0FFF1FE80FF91FEC5DB1
:10C6A000F64F898180839A819F708181807F892B59
:10C6B00081838B81882321F028DD182F81110AC006
:10C6C00010E0FFDC112311F0812F33DDDF91CF91DA
:10C6D0001F91089560E08B8104DDF3CF7F928F92EC
:10C6E0009F92AF92BF92CF92DF92EF92FF920F9301
:10C6F0001F93CF93DF931F92CDB7DEB76C01590123
:10C700002E2D30E09BDF19824501E12CF12C77249E
:10C710007394F40181914F019981811108C07110C6
:10C720004CC08081811105C0772473941BC07110A7
:10C730000AC080E09F3718F4E016F10661F5772013
:10C7400081F0782E01C0712C992329F1906899838A
:10C7500041E0BE016F5F7F4FC601F7DE8130D1F04F
:10C7600026C0782E9923B9F041E0BE016F5F7F4F5C
:10C77000C601EBDE8130D9F44981B701641B710930
:10C780006A0D7B1DC601E1DE9981891719F0981B9E
:10C7900099830DC0198289818F5F8983A895FFEFE6
:10C7A000EF1AFF0A0E151F0508F0B3CF08C08981E4
:10C7B0008F778701081B110902C0872DBBCFC601E7
:10C7C00063DFC8010F90DF91CF911F910F91FF9010
:10C7D000EF90DF90CF90BF90AF909F908F907F9021
:10C7E000089580E094E0E2E6F9E0DF019C011D920B
:10C7F00021503040E1F70895FF920F931F93CF939C
:10C80000DF93FA01149131967491795F769576955C
:10C810007695DA011396FA0132964491249FA00D81
:10C82000B11D112466956695669590E0F0E86F9FBE
:10C83000800D911D112420E030E060E08E59964F6C
:10C84000412F50E0671799F00A2FEC01C20FD31F58
:10C85000FD01FE2EF01AF11620F4F490F9923196B3
:10C86000F8CFA40FB51F6F5F20583F4FEBCFDF917C
:10C87000CF911F910F91FF900895CF93DF93382FA1
:10C88000463128F4842F880F840F880F7EC086E0FD
:10C89000830F20FD08C021FD02C090E005C09091EB
:10C8A000750D96FFFACF91E0687FA32FB0E050E1BD
:10C8B000659FA00DB11D1124AE59B64F22FF3DC09A
:10C8C0004E3211F088E0830F24ED240F2F3010F446
:10C8D0004B5211C02FEB240F2A3110F441530BC0DF
:10C8E0002FE9240F2A3110F4465305C04F3511F4B7
:10C8F0004AE201C040E06EE0469FA0011124455D80
:10C90000554E27E0FA0134913796E491211102C087
:10C91000E0E030E04F5F5F4F992311F03095E095F4
:10C92000FCE0A13EBF0730F43C93ED01C058DF4F5F
:10C93000E8831196215030F728C023FF07C0892FC4
:10C9400081958D9385E0830F31E001C030E025E0D3
:10C95000429FF0011124EF5AF24E25E04491332317
:10C9600011F0243041F05DE0A236B50718F49111C2
:10C9700040954C931196215031962111EFCF6DE0E7
:10C98000A236B60710F491959C93DF91CF9108954C
:10C9900020E073CFEF92FF920F931F93CF93DF931B
:10C9A000F62E122F902F9071E92EFA01112379F0B3
:10C9B000EE2011F0408101C04491EF012196442303
:10C9C00031F0202F6F2D59DF1150FE01EFCFDF9195
:10C9D000CF911F910F91FF90EF9008950F93FA015F
:10C9E00094914F5F5F4F929F400D511D1124292F4D
:10C9F000D1DF0F9108950F9300E0CCDF0F910895E0
:10CA0000FF920F931F93CF93DF93162F022F922F36
:10CA10009071F92EEA01FF2011F0488102C0FE0159
:10CA20004491442361F04F3131F4185F103438F4ED
:10CA300080E02196F0CF202F612F1FDFFACFDF910A
:10CA4000CF911F910F91FF900895AB0120E0682FC7
:10CA500080E0D6CFFB01442341F09491992351F01B
:10CA60009F3109F441503196F6CF20E0AF01682F95
:10CA700080E0C6CF089520E0C3CFFF920F931F93AD
:10CA8000CF93DF93082FF62EEA0114E1180F15500B
:10CA90004C2F4F704A301CF0495C28E002C0405DCA
:10CAA00020E06F2D812FE9DE84E0D695C7958A9529
:10CAB000E1F71013ECCFDF91CF911F910F91FF9011
:10CAC0000895222321F09091750D96FD0895480F49
:10CAD000687FE82FF0E090E1699FE00DF11D1124DF
:10CAE000EE59F64F8E1B982F9E0F941720F49081CD
:10CAF00090959193F8CF08952DE08236920760F4D7
:10CB0000FC01208130916109332319F0262B31304B
:10CB100009F02627FC0120830895262F287F6770BF
:10CB2000E62FF0E0E052F04E649190E030E1239F78
:10CB3000800D911D11248E59964FDECFEF92FF92FA
:10CB40000F931F93CF93DF93F42E47FF02C0840F00
:10CB5000F194962F987FC82FD0E080E1989FC00D68
:10CB6000D11D1124CE59D64F6770E62FF0E0E05268
:10CB7000F04EE490FF20B1F08DE0C236D80790F47B
:10CB8000022F10E020FF08C06E2DCE01B5DF1595F5
:10CB90000795202F206803C015950795202FFA943C
:10CBA0002196E8CFDF91CF911F910F91FF90EF90E9
:10CBB00008952FEFC3CF1F93CF93DF93142F47FF19
:10CBC00002C0640F1195962F987FC82FD0E080E1A6
:10CBD000989FC00DD11D1124CE59D64F862F877036
:10CBE00099F0E82FF0E0E052F04E64916195180F53
:10CBF000185017FF0DC0E12FFF27E7FDF095E85112
:10CC0000F04EE4916E0F04C018303CF018506FEFF6
:10CC1000CE0172DFC058DF4FF7CF111654F4E12F69
:10CC2000FF27E7FDF095E052F04E64916150CE0190
:10CC300063DFDF91CF911F9108953F924F925F92F2
:10CC40006F927F928F929F92AF92BF92CF92DF921C
:10CC5000EF92FF920F931F93CF93DF93182FB62E6F
:10CC6000802F05FF04C004FF04C002E003C000E001
:10CC700001C001E0982F9F77C92EE7FE04C0E19420
:10CC80006624639401C0612C57FF0AC050954095FB
:10CC9000309521953F4F4F4F5F4F7724739401C0DC
:10CCA000712C82FF06C098E09093620DE8E0DE2EC2
:10CCB00005C096E09093620D75E0D72E86FF28C0E0
:10CCC00071101D0D283E83E038074105510514F011
:10CCD0001D0D05C0243631054105510514F01D0D0B
:10CCE00005C02A303105410551050CF01D0D00230A
:10CCF00081F0023031F424363105410551054CF400
:10CD00001D0D2A303105410551051CF41D0D01C0D2
:10CD10001D198091620D810F8093620D023011F414
:10CD200090EFC90E8824839452E0A52E912CFF2405
:10CD3000E7FCF09466E0562E5B0CE82DF0E0EE1672
:10CD4000FF060CF45DC06AE070E0C9010E940C7738
:10CD5000382EEB0140E3442E480E2C2D442D6B2D34
:10CD6000812F8BDD08112FC0C2FE1AC08FEF830DFB
:10CD7000833008F4A394CE016AE070E00E940C773F
:10CD8000823011F08430D9F484E3481204C099242D
:10CD90009394910E15C099249A94910EA39410C067
:10CDA0003EEF432E410E8FEF810FC0FE04C047E0DF
:10CDB0006B2D01DF02C0652DB0DE142D01C0912E58
:10CDC000209709F000E09E01442737FD4095542F3D
:10CDD000211531054105510581F4002331F0023060
:10CDE00059F491E0981540F008C0C4FE09C06110E4
:10CDF00004C080EFC80E01C000E01D1983949DCFD0
:10CE0000992059F09A944A2D6CE06B0D892DD1DE52
:10CE10004A2D6DE06B0D892DCCDE772031F02C2D65
:10CE20004DE26B2D812F8D1928DD80E0DF91CF91B0
:10CE30001F910F91FF90EF90DF90CF90BF90AF9038
:10CE40009F908F907F906F905F904F903F9008954C
:10CE5000EF920F93022F9A01442737FD4095542FEC
:10CE6000F5E0EF2EEADE0F91EF900895CF93DF9378
:10CE7000D62FC22F206250E0EBDFC7FD08C02C2F59
:10CE800046E76D2F8091620DDF91CF91F6CCDF9157
:10CE9000CF91089590913D0120915606921710F47C
:10CEA00022E001C020E0242B492FE0CF20E0D0CFAA
:10CEB000EF920F93022F005F242F30E040E050E00C
:10CEC000A2E0EA2EBADE0F91EF900895DF92EF9282
:10CED000FF920F931F93CF93DF93182FE62EEA0153
:10CEE000F22E822F8470D82E22FF05C01D5F57FFBF
:10CEF0000FC087E103C057FF0BC08FE02F2D4DE21D
:10CF00006E2D912F981B892FB8DCD195C195D10931
:10CF10002F2D20234AE36E2D812FAFDC6CE370E0D0
:10CF2000CE010E940C77462FC82FD1101E5F2F2DE7
:10CF30006E2D812FBDDFDD2011F085E101C08FE076
:10CF4000810F202F4C2F6E2DDF91CF911F910F91CC
:10CF5000FF90EF90DF90ACCF0F931F93CF93DF93B1
:10CF6000C82FD62F142F022F422F25DE123030F07B
:10CF7000402F6D2F8FEF810F8C0F1DDE6FEF6D0F28
:10CF8000600F412F8C2F15DE412F6D2F8C2FDF91DD
:10CF9000CF911F910F910DCECF93C091610991E078
:10CFA00090936109D9DFC0936109CF9108950F93E0
:10CFB0001F93CF93DF93182FC62FD22FE42FF0E0CB
:10CFC0003297053608F004E60E9FC0010F9F900DC2
:10CFD000112464E670E00E940C77062F2D2F6C2F31
:10CFE000812FDADF002361F0D150DC0FCF5F1F5FAC
:10CFF000CD1730F4402F6C2F812FDBDDCF5FF8CFC2
:10D00000DF91CF911F910F910895A998AB988BBB99
:10D01000AD9AAD98AB9AA99A0895CF93C82F81E0A5
:10D0200080935F0981E8F1DF8C2FEFDF10925F09B9
:10D03000CF91089580915506F0CFCF93DF9381E093
:10D0400080935F09AA982AE02A95F1F700C0AA9A6E
:10D050008CED95E0E5E0EA95F1F700000197009787
:10D06000C9F7AC98C1E2DAE1FE018491CEDF2196E6
:10D07000FAE1CB32DF07C1F7DF91CF91DBCF1F930E
:10D08000CF93DF9340916009442321F08091750D87
:10D0900086FD32C081E080935F0910EBC2E6D9E0E3
:10D0A00084E0B3DF80E1B1DF812FAFDFA998AB9AD5
:10D0B000FE019E0120583F4F80818BBBAD9AAD98F9
:10D0C00081818BBBAD9AAD9882818BBBAD9AAD98B7
:10D0D00083818BBBAD9AAD983496E217F30761F765
:10D0E000EF01AB9AA99A1F5F183BD1F610925F0926
:10D0F000DF91CF911F9108954A5260E080E059DDA1
:10D10000C9CFBF92CF92DF92EF92FF920F931F93FE
:10D11000CF93DF937B018A01080F191FEC01E81AF6
:10D12000F90A6701CC0EDD1EC017D107C1F0B99016
:10D13000809108098270E19B05C08823E1F30E9479
:10D14000011CF6CFDFBACEBAE09A8DB3B81649F318
:10D15000BDBA8FB7F894E29AE19A8FBFE2CFDF9120
:10D16000CF911F910F91FF90EF90DF90CF90BF90E4
:10D1700008958091A60D1092A60D0895FC0180815E
:10D180008F70880F611181608F709081907F982BD4
:10D19000908381818F5F81838281882351F09F708A
:10D1A00041F4833621F0842F80628093A60D118292
:10D1B00012828281883069F148F4813091F188F0DF
:10D1C000823039F1843009F03FC023C08F35C1F07F
:10D1D00018F48031F1F00895813649F0823671F10A
:10D1E000089580818F708F3079F581E62BC040667D
:10D1F0004093A60D10923601109235018FE522C0A2
:10D200008181803211F4406816C08832E9F480E1EF
:10D2100019C09181903328F090E09595879582838D
:10D220001182828190E00197218130E08223932353
:10D23000892B51F440644093A60D08958181803478
:10D2400018F088E08283118208955091630041B103
:10D25000282F30E02F3031056CF4F901EE0FFF1F5D
:10D26000E20FF31FE758F24F90819F7081E09F30EB
:10D2700051F52AC090E0FC013F97E930F10518F51F
:10D28000E855FF4F0C945D77942F947019C091B1BD
:10D29000927016C0952F10C0952F9095987010C061
:10D2A00053FF11C091B102C0942F9095907408C0A3
:10D2B000942F907105C0942F917002C0942F90729A
:10D2C00081E0911101C080E008958D3208F062C0C4
:10D2D0009FEF980F993010F4825FB7CF51EE580F3F
:10D2E0005330D8F491B1909594705523C9F0409182
:10D2F0009A064F70415021E030E0042E01C0220F09
:10D300000A94EAF73091780D3223523041F0932B92
:10D3100021E009F020E0922F03C090E001C0932F9C
:10D3200085528330F0F491B19695917021E0922767
:10D33000882369F140919A0642954F70415021E04F
:10D3400030E0042E01C0220F0A94EAF73091780DE4
:10D350003223823009F1932B81E009F080E0982F8D
:10D3600016C0863019F420919C0605C0873079F4E8
:10D3700020919C0622952F70215081E090E0022E92
:10D3800001C0880F0A94EAF79091780D982381E004
:10D39000911104C080E00895932FF9CF0895CF93A1
:10D3A000C82F93DF811107C081E08C0F8EDF8823A7
:10D3B00021F081E003C080E001C082E0CF910895B8
:10D3C0008F7090E08F30910551F0FC01EE0FFF1F40
:10D3D000E80FF91FE758F24F82E682831182089521
:10D3E0008F7090E08F30910549F0FC01EE0FFF1F28
:10D3F000E80FF91FE758F24F83E682830895EF9212
:10D40000FF920F931F93CF93DF938091760D9091AE
:10D41000770D01969093770D8093760D8093750D1F
:10D4200096B390958091A70D882321F0282F287717
:10D43000292349F4892F807609F07DC093FD77C0B8
:10D4400094FF77C080E1182F166019238093A70DF1
:10D45000C9E7DDE000E011FB662760F9402FCE014F
:10D460008DDE0F5F169523960630A9F780910A028C
:10D4700081110EC0F0B2F0948091870686FF09C03A
:10D480008F2D837FF82E80917D0E8C70F82A01C03D
:10D49000F12CC8EEDFE100E010E076E0E72EEC1AB8
:10D4A000FE0184914C2F4E0D8F2161E009F460E064
:10D4B000C8018557924F62DE21960D5F1F4F0831DC
:10D4C000110571F79091100261E0C92FC07295FFAC
:10D4D00060E04EE083EA9DE051DE86B390E0809507
:10D4E00090958E7799278C2B19F089E080935501C0
:10D4F00080917D0E86FD02C0817402C081708260C1
:10D500009091630092FF88609091630095FF806224
:10D51000989B84609C9B8064B79B80618093780D0E
:10D52000DF91CF911F910F91FF90EF90089588E0C8
:10D530008ACF80E088CF80E686CF929A10929800BA
:10D5400089E18093990080919B008D7F80939B005F
:10D5500086E080939D0080919B0087FF03C08091AF
:10D560009C00F9CF88E980939A00089581E0809328
:10D57000AB0D80930A028091870686FFDECF089567
:10D580008091870686FF10929A0010920A026CC75B
:10D5900090919B0095FFFCCF80939C000895E3E65B
:10D5A000FDE091898089891749F0DF01A90FB11D3C
:10D5B0008C919F5F9F70918B90E008958FEF9FEF0C
:10D5C00008951F920F920FB60F9211242F938F93ED
:10D5D0009F93EF93FF9380919A008F7780939A00A7
:10D5E0007894E091730D81E08E0F8F7090919C0084
:10D5F0002091740D821731F0F0E0ED59F24F9083D5
:10D600008093730DF89480919A00806880939A00BB
:10D61000FF91EF919F918F912F910F900FBE0F90DF
:10D620001F90189595E0899FD0011124AF5CBB4FE6
:10D63000CB010596FB0124912D933196E817F9074C
:10D64000D1F708950F931F93CF93DF93182FC5E65B
:10D65000D2E090E08881181738F0882329F09032C2
:10D6600001F19F5F2A96F6CF9032D9F02FE130E09A
:10D67000291B31090AE0029FA001039F500D1124CC
:10D68000BE01CE010A960E946C77FE0111920A95A6
:10D69000E9F7188384E68A838F8188608F83CE01BF
:10D6A00002C085E692E0DF91CF911F910F9108951E
:10D6B00080E491E0E5E6F2E0DF019C011D9221505B
:10D6C0003040E1F7089588E2E1E3F4E0DF011D92E4
:10D6D0008A95E9F788E4E9E5F4E0DF011D928A958F
:10D6E000E9F7089590E00197FC01EE0FFF1FE80FA6
:10D6F000F91FEF55FB4F6F706283408321830895BC
:10D70000CF93C62F9FDFFC01C183CF9108959F92D5
:10D71000AF92BF92CF92DF92EF92FF920F931F933F
:10D72000CF93DF9300D000D0CDB7DEB7182FE091B4
:10D730007006F0E0EF5BFC4FE49184E09E2F937065
:10D74000A1E0B0E0AC0FBD1FA90FB11D8C93E69511
:10D75000E695815099F7111108C0AADF61E089812F
:10D76000CFDF62E08A81CCDF3AC0113041F4EB8137
:10D77000F0E0EE0FFF1FEA53FB4F10830AC0123098
:10D7800089F4EB81F0E0EE0FFF1FEA53FB4F81ECD1
:10D7900080838091BC0585FF02C080E001C08CE9D8
:10D7A000818309C1133009F583DF0981802F4ADFA6
:10D7B000FC01EE24E394E1821EEC1283802F42DF11
:10D7C00002E0FC0101831283FA808F2D3BDFFC0114
:10D7D000E18212838F2D36DFFC010183128363E027
:10D7E0008B818EDF64E08C8121C0143009F560DF0D
:10D7F000FA808F2D27DFFC0122E0E22EE1820EEC81
:10D8000002838F2D1FDFFC0111830283FC808F2D8B
:10D8100019DFFC01E18202838F2D14DFFC011183EB
:10D82000028361E089816CDF63E08B8169DFC3C0C3
:10D83000153009F092C03CDF46DF81E003DF4AE0AB
:10D84000C42EFC01C18282E0FDDE5BE0D52EFC012E
:10D85000D18283E0F7DE6CE0F62EFC01F18261E01C
:10D8600084E04EDF85E0EEDEFC0103E0018374E03E
:10D87000B72EB38287E0848387818160878385E0C8
:10D88000E1DEFC0101831383A8E09A2E9482878154
:10D890008160878385E0D6DEFC010183B6E0EB2E54
:10D8A000E38289E0A82EA48287818160878385E056
:10D8B000C9DEFC0191828CE9828381E083838781C8
:10D8C000897F8460878386E0BDDEFC01A1828EE1D2
:10D8D000828388EF83838BE0B5DEFC01018396E4CD
:10D8E000A92EA282B382C4828781816087838BE064
:10D8F000A9DEFC010183A2821383D4828781816027
:10D9000087838BE09FDEFC010183A282E382F482A5
:10D91000878181608783809161028F7180628093AB
:10D9200061028FE18093620264E070E280E07ADE5F
:10D930006FEF7FE181E076DE6AEF7FE182E072DE09
:10D9400065EF7FE183E06EDE60EF7FE184E06ADE19
:10D9500060EF7FE185E066DE2EC0163099F486E048
:10D9600071DEFC01118382E3828398EF93838087C9
:10D9700086E068DEFC0111838EEC828398E093835D
:10D98000808719C0173021F01830A9F488E001C051
:10D9900080E158DEFC0189E0818384E6828384E1B2
:10D9A000838387E786838EE08093C10488E0809339
:10D9B000BF048093C00482E00E945E5E0F900F90CF
:10D9C0000F900F90DF91CF911F910F91FF90EF90EB
:10D9D000DF90CF90BF90AF909F900C945A5F80E4FF
:10D9E0009CE99BBD8ABD87B7806187BF1FBC8AE069
:10D9F0008EBD08950F931F93CF93DF9310915C0218
:10DA0000129516951770882331F0A0E0BEE08330A0
:10DA100021F420E103C0A8EBBDE028E090915B0277
:10DA2000990F910F920F60915E0224E66202B0019D
:10DA30001124685A7D4F0091640248EE53E00403BC
:10DA40009001059F300D112428533045261B370BBC
:10DA5000FD0132966D937C934091610241FF03C0BA
:10DA600040E055E002C040E054E0833011F418EF8C
:10DA7000190FCC27DD27C41BD50B1917F0F4A12FE4
:10DA8000B0E0AA0FBB1FAA50B84F0D90BC91A02DBB
:10DA90004A175B070CF4DA01AC17BD070CF4DE0182
:10DAA000A854B44F2A1B3B0BA61BB70BB183A08312
:10DAB000738362831F5F3496E0CF283293E2390785
:10DAC00010F428E233E231832083882331F0285E8A
:10DAD00033403093A90D2093A80D13821282DF9159
:10DAE000CF911F910F9108951F920F920FB60F9231
:10DAF00011242F933F934F938F939F93EF93FF9313
:10DB000088B391E0892788BBE0910E01F0910F0165
:10DB10008081982F9F709F3039F040914A0E949FDA
:10DB2000402D1124415001C04FEF242F30E037BD6C
:10DB300026BD90E024E0959587952A95E1F700971A
:10DB400031F43196F0930F01E0930E0101C0808310
:10DB5000493C40F080915A028F70863011F4C09891
:10DB600001C0C09A8091AE0D81608093AE0DFF918F
:10DB7000EF919F918F914F913F912F910F900FBEF9
:10DB80000F901F9018951F920F920FB60F921124AD
:10DB90002F933F938F939F93EF93FF9388B391E0DD
:10DBA000892788BBE0911001F0911101808128B58F
:10DBB00039B580FD03C0205E3F4F02C0205F3F4F5C
:10DBC00039BD28BD90E095958795009769F4CF0100
:10DBD000019690931101809310018181811105C0FC
:10DBE00087B7877F87BF01C080838091AE0D81603A
:10DBF0008093AE0DFF91EF919F918F913F912F9167
:10DC00000F900FBE0F901F901895EDE7F0E0808108
:10DC1000857E808317981F9AAAE8B0E01C92109224
:10DC20008B0082E88C938081806280830895EDE789
:10DC3000F0E080818F7D8083179AAAE8B0E01C9283
:10DC400010928B008AE08C93808188618083089594
:10DC50001F920F920FB60F9211248F939F93EF9301
:10DC6000FF938091480E882321F01F9A1092480E4E
:10DC700004C01F9881E08093480EE0910A01F09162
:10DC80000B01808191819093870080938600809121
:10DC9000A80D9091A90D90938500809384008281B6
:10DCA0009381892B11F0329608C080916102809592
:10DCB00081708093480EE0E0FEE0F0930B01E0936A
:10DCC0000A018091AE0D81608093AE0DFF91EF91BE
:10DCD0009F918F910F900FBE0F901F901895EFEAB4
:10DCE000FDE09081969596952781222311F09695D7
:10DCF0009695982B908321812F5F2183808528170B
:10DD000050F0A281B3819D012F5F3F4F3383228367
:10DD10009C93108211820895FF920F931F93CF93CB
:10DD2000DF93C82F80915A028F70823069F09C2F48
:10DD300088E0D0E0292F2078D20F990F8150D1F7B9
:10DD4000D07859E0F52E03C048E0F42ED0E810E07A
:10DD500080E190E00C2F0170901302C0805F02C040
:10DD6000BEDF80E1C695CD2B1F5FF11618F0D0E81D
:10DD7000902FF0CF805FDF91CF911F910F91FF9097
:10DD8000AECF882339F08091B50D8F5F8093B50DAC
:10DD900080E803C01092B50D80ECA1DF8091B50D35
:10DDA0008530C0F70895CF93DF93C82F8091B40DCD
:10DDB0008C27E82FEF70F0E0EE0FFF1FE457FF4DC8
:10DDC0006591749182958F7041E850E1849F900134
:10DDD000859F300D11245091B30D40E02427352745
:10DDE000262737273093B40D2093B30DD8E08C2F1E
:10DDF0008078C7DFCC0FD150D1F7DF91CF91089554
:10DE0000CF9380EC6CDFC6E080E869DFC150E1F7BA
:10DE100080ECCF9164CF8031E0F4E82FF0E0EE0F9A
:10DE2000FF1FEA50F84F20813181C901880F991FE7
:10DE3000820F931F97FD03969595879595958795E6
:10DE40009C5F1816190644F48E3F27E092073CF4B5
:10DE5000089580E094E0089581E090E008958EEFC9
:10DE600097E008956F927F928F929F92AF92BF92A8
:10DE7000CF92DF92EF92FF920F931F93CF93DF9396
:10DE80001F92CDB7DEB77FEA672E7DE0772EF301D4
:10DE90003F0188EB9DE0938382831082118215827B
:10DEA000148281E0878382E080871091AA0DF09030
:10DEB0005A02FF2DFF70FF2EF81357C080E18093A8
:10DEC0004A0E16FF0CC080913C05882321F081305A
:10DED00021F410E906C010E804C018E902C017FFD9
:10DEE00005C087E1B2D9882309F4F9C017FDF9C04C
:10DEF00085E10E943119882309F4F3C01062812F53
:10DF00000BDF1093AA0D80915B0206DF06EF17E08E
:10DF1000F12C6DE0D62EF801819191918F01D89E60
:10DF20009001D99E300D112455E0359527955A95CD
:10DF3000E1F73E5F37FD07C02F3FF3E03F0734F4C2
:10DF4000E22E832F06C0E12C80E003C0EE24EA9489
:10DF500083E09F2D990F990F892BDEDE8E2DDCDE5D
:10DF6000F39426E0F212D7CF97C084E180934A0E53
:10DF700086E0F81302C08FE021C080913C0599270C
:10DF800087FD909501968F739927809714F084E50B
:10DF900001C085E5C1DE10913C051F5F1F758091B2
:10DFA000AC0D80FD106885FD1062812FB5DE1093E9
:10DFB000AA0D80915B02B0DE80913D05ADDE00E0F0
:10DFC00010E0C12CD12CE12C912C35E0A32EB12CEA
:10DFD00048EF842E80915C02829586958770F801C7
:10DFE000E80FF11DEE0FFF1FEA50F84F808191817D
:10DFF000880F991F880F991F181619061CF424E022
:10E0000030E002C02CEF3FEF820F931FB50104D721
:10E01000E5E0CB01FE1202C09C5F02C080529C4F23
:10E0200097FD07C08115F8E09F072CF08FEF97E070
:10E0300002C080E090E0AA2797FDA095092C03C0BC
:10E04000880F991FAA1F0A94DAF7C82AD92AEA2A40
:10E050002BE0290D29838C2D5FDECD2CDE2CEE24C8
:10E060008981885089838830B0F793E0990D892F92
:10E07000869586958695992E889D900C11240F5F24
:10E080001F4F0031110509F0A5CFE6E0FE1204C0D4
:10E0900080E042DE80E040DEF3018181A281B38135
:10E0A000882319F08FE08C9304C0FD018291806F6A
:10E0B000808388EB9DE090930F0180930E010F9079
:10E0C000DF91CF911F910F91FF90EF90DF90CF9054
:10E0D000BF90AF909F908F907F906F9008951F7723
:10E0E00005CF1F7D0CCFCF92DF92EF92FF920F935F
:10E0F0001F93CF93DF93C0915A02CF708091730624
:10E1000085FF04C0809147028111C4E08091AB0D6E
:10E110008111CFEF8091AD0D8C1709F467C0C093CA
:10E12000AD0D1EBC1DBC1CBC87B7837C87BF809116
:10E130007D008E7F80937D008CE386BF8FE380938C
:10E140007C008C2F90E08730910508F04FC0FC01D7
:10E15000EF54FF4FB2C659DD42DC0CC156DD88E5F5
:10E160009BE199BD88BD80EA9FE090937900809300
:10E17000780087B7886087BF80917D008160809339
:10E180007D001FBC82E08EBD44C03FDD88EC90E086
:10E1900090937900809378008CE291E09DBD8CBDD6
:10E1A00080EE9BEA97BD86BD87B7806287BF80916E
:10E1B0007D00816080937D001FBC8AE18EBD16C00A
:10E1C000C43021F484E016DCC09803C008DC83E08E
:10E1D00011DC80E593EC909387008093860088E8BB
:10E1E00093E1909385008093840021DDC23009F48F
:10E1F000BEC038F4CC2309F4BDC0C13009F0BCC0A6
:10E2000008C0C33009F4B6C0C550C23008F0B4C06D
:10E21000AEC07894F0904A0E87B7877F87BF809111
:10E220007D008E7F80937D00EFEAFDE088EB9DE02E
:10E23000909311018093100189EB9DE09383828379
:10E2400015821482108211821682178284E08087E0
:10E250008FEF8093B80DD4DD80915B02A4DD4091F7
:10E26000AC0D80913C0540FF0CC090E48902900108
:10E27000112480915A028695869586958670822B08
:10E2800004C020E48202C0011124842B8CDD80E0D4
:10E290008ADDE0905C02E294E694A7E0EA228F2D0A
:10E2A0008170D82EF0FE02C098E0E90EF8E0CF2E83
:10E2B000CE0C8E2DB0DD8C01D110185F802F73DD58
:10E2C00081E08E0DA8DDEC01D110D85FE394E394DA
:10E2D0009C2F9295907F812F8F70892B64DDCE01CA
:10E2E000E4E096958795EA95E1F75DDDEC10E1CFE6
:10E2F00080E059DDC091B30D8091B40D54DD8C2FB9
:10E3000052DD7EDD8091B00D882319F080E0E7DCDE
:10E31000F9CFE091B10DF091B20D1082E8E7F0E095
:10E32000808191819C012854344F39BD28BD805B88
:10E33000994B91838083C09A88E086BF81E0809367
:10E340007C0087B7886087BF80917D008160809363
:10E350007D0080913C05813031F08091570282FD33
:10E3600002C0F39401C0F12CF0924A0E05C07894DB
:10E3700079DD02C080E03EDBDF91CF911F910F91EC
:10E38000FF90EF90DF90CF9008951F920F920FB6FD
:10E390000F9211242F933F934F935F936F937F932B
:10E3A0008F939F93AF93BF93CF93DF93EF93FF939D
:10E3B0008CB59DB52091490E222321F0C09A109270
:10E3C000490E04C0C09821E02093490EC0910C0171
:10E3D000D0910D01FE01219131913BBD2ABDF093F9
:10E3E0000D01E0930C01E6E0F1E0282F31813817B0
:10E3F00008F481833081231708F480838A819B810C
:10E40000892BD1F488EB9DE090930D0180930C0152
:10E4100080916102809581708093490E87B78F7ECD
:10E4200087BF61DE80915A028F7011F0833021F432
:10E4300087B7806187BF78948091AE0D81608093AB
:10E44000AE0DFF91EF91DF91CF91BF91AF919F9171
:10E450008F917F916F915F914F913F912F910F908D
:10E460000FBE0F901F90189580916102809581706A
:10E470008093490E8093480E811101C0C09A80910B
:10E480005A028F70865F8093AD0D1092AB0D2BCE2C
:10E490001F920F920FB60F9211242F933F934F9319
:10E4A0005F936F937F938F939F93AF93BF93EF93FC
:10E4B000FF9380915A028F70813011F1863029F0DC
:10E4C000853031F080E492EA05C080E89EE302C026
:10E4D00080E99DE397BD86BD209178003091790059
:10E4E0002F3F310538F488589341909379008093F9
:10E4F000780007C088EC90E09093790080937800D2
:10E50000F2DDFF91EF91BF91AF919F918F917F913C
:10E510006F915F914F913F912F910F900FBE0F9090
:10E520001F9018951F920F920FB60F9211242F93E0
:10E530003F934F935F936F937F938F939F93AF938B
:10E54000BF93EF93FF9380915A028F7078949091CC
:10E55000AD0D981769F0943059F4809147028823E3
:10E5600021F08091730685FD02C0BDDD02C084E00C
:10E5700041DAFF91EF91BF91AF919F918F917F9180
:10E580006F915F914F913F912F910F900FBE0F9020
:10E590001F90189580919D0680FD05C080916500B3
:10E5A0008B7F809365000895CF93DF93EC01F2DFBA
:10E5B0001C821D82188219821EA61FA6DF91CF9190
:10E5C0000895F2CF21E0FC018481811101C020E097
:10E5D000822F0895FC0121818081281B277098E0FB
:10E5E000921B81E0933008F480E00895CF93DF938D
:10E5F000EC018C818823F1F081508C838A819B818E
:10E60000890F8A838EA58823D1F18FA59FEF980F5C
:10E610009FA7882351F080919D0680FD30C0809196
:10E6200065008460809365002AC0B4DF8091750620
:10E630008FA725C01B98AEDF8D81882319F08150EC
:10E640008D831DC0888199818917C9F090E0FE01F2
:10E65000E80FF91F26812A8326892C8326852B83A0
:10E66000268D2D8320A92EA71FA626A13FEF320FAE
:10E6700036A3211104C00196877099278883DF9102
:10E68000CF910895EF92FF920F931F93CF93DF9353
:10E69000EC01F62E142FE22E9DDF882309F453C0DF
:10E6A0008091C60181FD4FC080916A06887309F48C
:10E6B0004AC0302F3295369536953370402F4F70C3
:10E6C000333009F43FEFFF2021F090917406965FFC
:10E6D000F90E803129F48BEA189F112D112402C004
:10E6E000883111F4169509C0883211F4110F05C054
:10E6F000803319F4812F880F180F288104FF0DC073
:10E70000FA821C83ED8205FB882780F98EA71FA65D
:10E710003B8329834423B9F001C04F5FE981F0E0D6
:10E72000CF01019687709927281769F0EC0FFD1F1C
:10E73000F682168BE68E05FB002700F900AB4150F0
:10E7400046A336878983DF91CF911F910F91FF9068
:10E75000EF9008950F931F93CF93DF93EC01062F53
:10E76000642F80916A068695869586958770388194
:10E7700029813213EFC010E00332110508F0EAC01E
:10E78000F801E854FF4F99C300E326C000E321E0FD
:10E79000C0C002EA22E04AE064E6DAC00AE222E00F
:10E7A00045E06FE5CE016EDF01E22AE045E06FE56E
:10E7B000CE0168DF0AE222E045E06FE5C9C002EC65
:10E7C00023E04AE060E5CE015DDF02E423E04AE0B9
:10E7D0006CE3CE0157DF00E221E065C001E221E0F9
:10E7E00045E066E4CE014EDF22E04FE062E3CE0179
:10E7F00049DF22E04FE062C002E221E045E06EE640
:10E80000CE0140DF03E221E045E097C000E025E0D3
:10E8100045E062E3CE0136DF25E045E06AE5CE0162
:10E8200031DF02E024E043E06EE692C003E22AE03A
:10E8300045E060E5CE0126DF01E224E145E060E548
:10E84000CE0120DF03E22AE045E038C002E625E001
:10E8500044E16AE07DC002E22AE044E062E3CE01E6
:10E8600011DF01E224E148E066E4CE010BDF02E2C1
:10E870002AE048E062E3CE0105DF01E224E144E062
:10E880004DC00AE22AE002C002E222E345E04BC0AA
:10E8900001E203C002E201C003E22AE044E160E0D9
:10E8A00057C002E122E04AE039C002E423E044E13B
:10E8B0006CE3CE01E7DE02EE23E044E160E548C010
:10E8C00000E321E048E22AC0813009F443C000E1BE
:10E8D00021E04AE06BE43CC08130E1F100E121E05D
:10E8E0004AE061E435C000E121E046E031C000E3E8
:10E8F000D9CF813079F100E1D5CF00E112C003E337
:10E9000003C002E301C001E323E04FE00CC001E3D8
:10E9100029E144E103C000E321E04EE166E418C0D0
:10E9200001E321E04AE068E713C002E321E04AE0A6
:10E930006AE70EC003E321E04AE06CE709C000E5A6
:10E9400020E04AE062E804C000ED20E04AE062E333
:10E95000CE0198DEDF91CF911F910F91089546E48B
:10E96000682F88EC91E0F6CE462F682F88EC91E076
:10E97000F1CE9091760691FF03C0862F0C948714F8
:10E98000EECFCF92DF92EF92FF920F931F93CF9330
:10E99000DF93EC01062F142F47FF03C0842F0E9442
:10E9A0008714D7FF06C0D195C195D1098AE10E948D
:10E9B0008714002369F0023019F464E670E002C0A5
:10E9C0006AE070E0CE0128D2262FC22FD72FF82E72
:10E9D00064E670E0CE0120D29B01FB01EC016115E1
:10E9E000710591F16A307105C4F06AE070E0C90107
:10E9F00013D26B017C01653171051CF48EE68C0D20
:10EA000005C08CE88C0D0E9483148EE60E9487144A
:10EA1000F701309769F001E001C000E084E68E0F55
:10EA20000E948714011104C0209741F18C2F0AC065
:10EA3000209721F1CE016AE070E0EED19E01281B03
:10EA4000390BC901845713C084570E9483140023D3
:10EA5000A9F0023079F46AE070E08F2D90E0DCD10B
:10EA6000C82F86E0860F0E9487148CE88C0F0E94C6
:10EA7000831404C086E08F0D0E94871411161CF4C5
:10EA8000812F0E948714DF91CF911F910F91FF90EA
:10EA9000EF90DF90CF90089586B380958E7708959C
:10EAA0008FEF8ABB1BBA91E897BB9EE798BB9EE3AA
:10EAB00094BB91EC95BB11BA82BB98E092B997EFE9
:10EAC00093B9109261001092620094E190936400F7
:10EAD0009BEF909365008093AA0DD4B780E884BF24
:10EAE00084BF80E487B985E886B987E083BF8CE975
:10EAF00081BF82E085BD83E487BF1FBC8AE08EBDF5
:10EB000010928B0082E880938A0080E280937D00DF
:10EB100078948EE995E490934C0180934B010E9488
:10EB2000785E882319F00E941D6806C00E942C5D43
:10EB30000E941D680E943A5E91E080B38095837CBC
:10EB4000803419F49093C601F8CF823849F4F894D0
:10EB500064E172E088E00E9425650E943F68FFCF73
:10EB6000D09054068D2D0E94695F96DF982F967085
:10EB7000963031F48091C60182608093C60125C031
:10EB8000C0E081FD05C08695CF5FC630D1F71DC0BE
:10EB90008C2F0E94D45D8823C1F0C09354068C2F23
:10EBA0000E94695F81E00E945E5E0E94F16324E042
:10EBB0004EE052E060E086E10E94006588E10E943C
:10EBC00098330E943F680E9468120E94E010809172
:10EBD000870686FD0E949D6A81E0809339010E942C
:10EBE000581A1092390180918306895F0E94891416
:10EBF000D3FD76C080916D0684FF05C080916A06C2
:10EC000082FD47C03DC080917606882319F06CE1F3
:10EC100087E0AFDE0E9434190E94F16320E040E6F5
:10EC200053E060E080E00E94FC638091730684FD05
:10EC300008C000E12AE048E756E068E380E00E946F
:10EC4000CA640E943F680E9468120E9459160E947E
:10EC50002A168C010E948E10EC01C057DE4F0E94D4
:10EC60003F680E9434190E9459160E942A167C019E
:10EC700013DF8111C3CFE016F10609F45CC0BECFEB
:10EC80000E94BE60883C910520F488EF91E00E94CC
:10EC900084190E94591680912101909122016EE001
:10ECA00070E0A6D060933D010E949B190E94B619A6
:10ECB00090916A06987B21F482EE91E00E9484197B
:10ECC0008091C701882331F086EB91E00E9484197E
:10ECD0001092C7010E946812809155020E9483140D
:10ECE000909105019260909305011092040760E0F5
:10ECF00086EF97E00E940248B7DB8DE028E130E024
:10ED00000FB6F894A89521BD0FBE81BD23EB3AE262
:10ED100030934E0120934D0180915406D81629F06E
:10ED200081E00E945E5E0E945A5F81E0809348020B
:10ED30000E94011CFDCF0E948E10C817D90709F050
:10ED40008ECF5CCF88EC91E03CCC05D0332312F41D
:10ED50008A1B9B0B10C0A29FB001B39FC001A39F51
:10ED6000700D811D1124911DB29F700D811D112404
:10ED7000911D0895F0DFB7FF0895821B930B08954E
:10ED8000EADFA59F900DB49F900DA49F800D911D6B
:10ED900011240895B7FFF4CFF3DF821B930B08957E
:10EDA000DB018F939F93ECDFBF91AF91A29F800D0A
:10EDB000911DA39F900DB29F900D11240895991B52
:10EDC00079E004C0991F961708F0961B881F7A9562
:10EDD000C9F78095089587FB082E062687FD819543
:10EDE00067FD6195ECDF0EF4919507FC8195089520
:10EDF000AA1BBB1B51E107C0AA1FBB1FA617B70761
:10EE000010F0A61BB70B881F991F5A95A9F780957C
:10EE10009095BC01CD01089597FB072E16F4009440
:10EE200006D077FD08D0E4DF07FC05D03EF49095CE
:10EE300081959F4F0895709561957F4F0895A1E248
:10EE40001A2EAA1BBB1BFD010DC0AA1FBB1FEE1F64
:10EE5000FF1FA217B307E407F50720F0A21BB30BAF
:10EE6000E40BF50B661F771F881F991F1A9469F72B
:10EE700060957095809590959B01AC01BD01CF0187
:10EE80000895052E97FB16F400940FD057FD05D07A
:10EE9000D6DF07FC02D046F408C050954095309567
:10EEA00021953F4F4F4F5F4F0895909580957095F6
:10EEB00061957F4F8F4F9F4F0895EE0FFF1F059075
:10EEC000F491E02D0994FB01DC0102C001900D9248
:10EED00041505040D8F708956817790768F4FB014E
:10EEE000DC01E40FF51FA40FB51F02C002900E92C3
:10EEF00041505040D8F70895E6CFDC0101C06D9332
:10EF000041505040E0F70895DC01CB01FC01E1994C
:10EF1000FECF06C0FFBBEEBBE09A31960DB20D925C
:0CEF200041505040B8F70895F894FFCF1E
:10EF2C00F00064000A02FF000000000EB80DB80DDE
:02EF3C00B80D0E
:00000001FF
